:10000000FCFB0220D101000059F3000011F30000B5
:1000100011F3000011F3000011F3000011F30000D0
:1000200011F3000011F3000011F3000059F3000078
:1000300059F3000011F30000A9120100F9140100A6
:1000400059F3000059F3000059F3000059F3000080
:1000500059F3000059F3000059F3000059F3000070
:1000600059F3000059F3000059F3000059F3000060
:1000700059F3000059F3000059F3000059F3000050
:1000800059F3000059F3000059F3000059F3000040
:1000900059F3000059F3000059F3000059F3000030
:1000A00091EF0000A5EF000059F3000059F30000A4
:1000B000651CFF1F59F3000059F300009916010059
:1000C00059F30000B518010059F30000D11A0100DE
:1000D00059F30000D11B010059F3000069EF000043
:1000E00059F3000059F3000059F3000059F30000E0
:1000F00059F3000059F3000059F3000059F30000D0
:1001000059F300003107FF1F59F3000059F30000B5
:1001100059F30000F500010059F3000059F3000005
:1001200059F3000059F3000059F3000059F300009F
:1001300059F3000059F3000059F3000059F300008F
:1001400059F3000059F30000D11C010059F30000DD
:1001500059F3000059F3000059F3000059F300006F
:1001600059F300007DEF0000B9EF000059F30000E3
:1001700059F3000059F3000059F3000059F300004F
:1001800059F30000EDEF000059F3000059F30000AF
:1001900059F3000059F30000D11D010059F300008C
:1001A00059F3000059F3000059F30000CDEF0000AF
:1001B00059F3000059F3000059F3000059F300000F
:1001C00059F3000059F3000059F3000059F30000FF
:1001D000614B4CF220524DF6281010B51A80188051
:1001E00000BF00BF5D4C0FF0BBF84FF030612160E5
:1001F0005B4B5C49A3604FF470005B4A5B4BE26071
:1002000008605B4C5B481C6090F800C05FEA0C71B2
:1002100004D590F800E04EF008020270564C574AA0
:10022000574BAA212170574CA34204D252F8040F15
:1002300043F8040BF8E7544954480024814202D2A1
:1002400041F8044BFAE75249524A002352F823007E
:1002500041F823000133742BF8D14F4C4F498023D0
:1002600004F8013B8C42FBD14D4B4E48484A02609A
:10027000A3F5805C8A242421A0221C708CF8011034
:100280008CF800209CF806008207FBD59CF80640FD
:10029000E406FBD4444991F806E00EF00C03082B69
:1002A000F9D142486022027002300478802CFCD1DF
:1002B0003D4B01215D2219715A7198798006FCD558
:1002C00093F806C0384C5FEA4C61F9D5384B394990
:1002D0001960002220205A602070A17901F00C03DF
:1002E0000C2BFAD1344A354C354814600168354C32
:1002F00011F4807303D14FF4A85223600260324995
:10030000324808600023072231484B6041F8042C32
:10031000C1F80C0D62B60FF019F92468E20705D593
:100320002C480FF001F92C4B2C4919602C4A1078FD
:10033000430609D5284C294B2168994204D1254808
:100340000FF0F2F80022226012F0CEF90FF00EF852
:100350000EF03EFFFEE700BF0E2005403080044057
:10036000823F040088ED00E00100002B002008E03F
:100370000300008502D0074000E007401018040089
:100380003007FF1F5030FF1F5030FF1F20E30120B8
:100390000002FF1F0000000000E400E064E400E051
:1003A0000050064008ED00E00040064001E0074034
:1003B000448004400000060204800440C01007008E
:1003C00010D0034014D0034014E000E01FBF02002F
:1003D0000000202071D46A681CE00340A5C3945A31
:1003E00000F00740FFFFFFFFFFFFFFFFFFFFFFFFE2
:1003F000FFFFFFFFFFFFFFFFFFFFFFFFFFFFFFFF0D
:10040000FFFFFFFFFFFFFFFFFFFFFFFFDEF9FFFF23
:1004100010B5054C237833B9044B13B10448AFF33E
:1004200000800123237010BD5030FF1F000000002A
:100430000C180400084B10B51BB108490848AFF36D
:1004400000800848036803B910BD074B002BFBD0A0
:10045000BDE81040184700BF000000005430FF1FE7
:100460000C1804005030FF1F00000000704700BF50
:10047000704700BF30B40246836842F21070DC78E7
:10048000240625D4DD782D0622D493F803C05FEA34
:100490000C651DD4DC7824061AD4DD782D0617D41B
:1004A00093F803C05FEA0C6412D4DC7825060FD4FD
:1004B000DD782C060CD40838E1D1987000BF936821
:1004C00080219970507300BF0124147330BC7047B1
:1004D0000220D8709468A37843F01005A570906846
:1004E0000171936842F21071DC78A40707D4DD78BB
:1004F000A80704D493F803C05FEA8C7513D5D978A4
:100500005FFA81FC0CF01004022504F0FF00DD709E
:10051000002C33D15FEACC7323D4012095680222EA
:10052000EA7030BC7047D8788407E8D4DC78A0073C
:10053000E5D4DD78AD07E2D493F803C05FEA8C74AC
:10054000DDD4D8788007DAD40839CDD1997000BFCE
:10055000936880249C70517300BF01250846157371
:10056000DFE793680121D97000BF936815739C7011
:1005700000BF95688021A9705473CFE7906810245C
:10058000C47000BF9568032100231173AB7000BFD6
:1005900094688020A07018465373BFE770B483B08E
:1005A00000238DF8073005469DF80730836842F236
:1005B0001070DC78260626D4DE78340623D493F82F
:1005C00003C05FEA0C661ED4DC7824061BD4DE78F8
:1005D000360618D493F803C05FEA0C6413D4DC78B1
:1005E000260610D4DE7834060DD40838E1D1987090
:1005F00000BFAE688022B270687300BF01242C7304
:1006000003B070BC7047987800F0E7049C70AE6847
:100610003379012AD8B28DF8070035D00224F4705E
:10062000541E002A39D00226AB6842F2107093F8AB
:1006300003C05FEA8C7217D4DA78920714D493F867
:1006400003C05FEA8C720FD4DA7892070CD493F867
:1006500003C05FEA8C7207D4DA78920704D493F867
:1006600003C05FEA8C7209D5FCB11B7901F8013B2C
:10067000012C14D0A868013CC670D5E7DA7892073F
:10068000F2D40838D3D1B2E7B27842F00803B3709D
:10069000AE680220F0700024C5E70120B0E7A8682A
:1006A000827842F008038370E4E79E7806F0C70280
:1006B0009A70AA6842F2107392F803C05FEA8C64E1
:1006C00029D5D078800626D5D478A60623D5D67825
:1006D000B40620D592F803C05FEA8C601BD5D078B1
:1006E000860618D5D478A40615D5D678B00612D5C6
:1006F000083BE1D1937000BFAA68802090706B73B3
:1007000000BF0124AA682C73184613790B70A968DE
:100710000225CD7074E70120F7E700BF034690F88B
:10072000640008B10020704770B49C6842F21076F3
:10073000E578AD060DD594F803C05FEA8C6508D561
:10074000E578AD0605D594F803C05FEA8C6500F145
:100750009B80B026A6709C6842F21076E578AD06C4
:1007600007D494F803C05FEA8C6502D4E578AD063F
:1007700048D5E678B60663D5A57845F03006A6706C
:100780009C6842F2107694F803C05FEA8C6507D447
:10079000E578AD0604D494F803C05FEA8C6554D5BF
:1007A00042EA4102D1B221719A6842F21074D678BD
:1007B000B50724D4D578A90721D492F803C05FEAFD
:1007C0008C751CD4D178890719D4D678B60716D47D
:1007D000D578AD0713D492F803C05FEA8C710ED4BC
:1007E000D1788E070BD4083CE1D1947000BF9A6891
:1007F000802696705C7300BF01241C7300E001200A
:1008000070BC704794F803C05FEA8C65B1D4E5789A
:10081000AD06AED494F803C05FEA8C65A9D4E57840
:10082000AD06A6D494F803C05FEA8C65A1D4083E57
:1008300094D1A67000BF9C688025A5705E7300BF30
:1008400000BF04261E7370BC7047E578AD06A7D4C0
:1008500094F803C05FEA8C65A2D4E578AD069FD416
:1008600094F803C05FEA8C659AD4E578AD0697D416
:10087000083E88D1A67000BF9D688021A9705E7374
:1008800000BF01221A73BBE7E578AD067FF561AFC3
:1008900094F803C05FEA8C657FF55BAFE578AD0641
:1008A0007FF557AF94F803C05FEA8C657FF551AFD1
:1008B000083E7FF43DAFBCE7034B586810B10168B8
:1008C0000A681047704700BF84DD0120034B986819
:1008D00010B101680A681047704700BF84DD01202D
:1008E000034BD86810B101680A681047704700BF11
:1008F00084DD0120034B186910B101680A681047B4
:10090000704700BF84DD0120034B586910B10168B6
:100910000A681047704700BF84DD0120034B9869C7
:1009200010B101680A681047704700BF84DD0120DC
:10093000034BD86910B101680A681047704700BFBF
:1009400084DD0120034B186A10B101680A68104762
:10095000704700BF84DD0120034B586A10B1016865
:100960000A681047704700BF84DD0120034B986A76
:1009700010B101680A681047704700BF84DD01208C
:10098000034BD86A10B101680A681047704700BF6E
:1009900084DD0120034B186B10B101680A68104711
:1009A000704700BF84DD0120034B586B10B1016814
:1009B0000A681047704700BF84DD0120034B986B25
:1009C00010B101680A681047704700BF84DD01203C
:1009D000034BD86B10B101680A681047704700BF1D
:1009E00084DD0120034B186C10B101680A681047C0
:1009F000704700BF84DD0120034B586C10B10168C3
:100A00000A681047704700BF84DD0120034B986CD3
:100A100010B101680A681047704700BF84DD0120EB
:100A2000034BD86C10B101680A681047704700BFCB
:100A300084DD0120034B186D10B101680A6810476E
:100A4000704700BF84DD0120034B586D10B1016871
:100A50000A681047704700BF84DD0120034B986D82
:100A600010B101680A681047704700BF84DD01209B
:100A7000034BD86D10B101680A681047704700BF7A
:100A800084DD0120034B186E10B101680A6810471D
:100A9000704700BF84DD0120034B586E10B1016820
:100AA0000A681047704700BF84DD0120034B986E31
:100AB00010B101680A681047704700BF84DD01204B
:100AC000034BD86E10B101680A681047704700BF29
:100AD00084DD0120034B186F10B101680A681047CC
:100AE000704700BF84DD0120034B586F10B10168CF
:100AF0000A681047704700BF84DD0120034B986FE0
:100B000010B101680A681047704700BF84DD0120FA
:100B1000034BD86F10B101680A681047704700BFD7
:100B200084DD0120034BD3F8800010B101680A680E
:100B30001047704784DD0120034BD3F8840010B1C7
:100B400001680A681047704784DD0120034BD3F821
:100B5000880010B101680A681047704784DD0120E1
:100B6000034BD3F88C0010B101680A681047704736
:100B700084DD0120034BD3F8900010B101680A68AE
:100B80001047704784DD0120034BD3F8940010B167
:100B900001680A681047704784DD0120034BD3F8D1
:100BA000980010B101680A681047704784DD012081
:100BB000034BD3F89C0010B101680A6810477047D6
:100BC00084DD0120034BD3F8A00010B101680A684E
:100BD0001047704784DD0120034BD3F8A40010B107
:100BE00001680A681047704784DD0120034BD3F881
:100BF000A80010B101680A681047704784DD012021
:100C0000034BD3F8AC0010B101680A681047704775
:100C100084DD0120034BD3F8B00010B101680A68ED
:100C20001047704784DD0120034BD3F8B40010B1A6
:100C300001680A681047704784DD0120034BD3F830
:100C4000B80010B101680A681047704784DD0120C0
:100C5000034BD3F8BC0010B101680A681047704715
:100C600084DD0120034BD3F8C00010B101680A688D
:100C70001047704784DD0120034BD3F8C40010B146
:100C800001680A681047704784DD0120034BD3F8E0
:100C9000C80010B101680A681047704784DD012060
:100CA000034BD3F8CC0010B101680A6810477047B5
:100CB00084DD0120034BD3F8D00010B101680A682D
:100CC0001047704784DD0120034BD3F8D40010B1E6
:100CD00001680A681047704784DD0120034BD3F890
:100CE000D80010B101680A681047704784DD012000
:100CF000034BD3F8DC0010B101680A681047704755
:100D000084DD0120034BD3F8E00010B101680A68CC
:100D10001047704784DD0120034BD3F8E40010B185
:100D200001680A681047704784DD0120034BD3F83F
:100D3000E80010B101680A681047704784DD01209F
:100D4000034BD3F8EC0010B101680A6810477047F4
:100D500084DD0120F8B50646044690F85870002559
:100D60002DE0042B00F0C080022B00F0B18008348D
:100D7000A069013540B1227F032A00F09D80042A3A
:100D800000F08F80022A7CD0206A6A1C38B194F867
:100D90002430032B69D0042B5CD0022B4CD0A06AEA
:100DA000AA1C38B194F82C1003293AD004292DD06C
:100DB000022917D00335082D04F1180425D0A069A5
:100DC0000028D4D0237F032BCBD147FA05F1CB07E2
:100DD000CDD496F858202A41D107C8D503681968A0
:100DE0008847C4E747FA02FC5FEACC71E2D596F87F
:100DF000583043FA02F2D307DCD4036819688847F5
:100E00000335082D04F11804D9D1F8BD96F858100F
:100E1000794041FA02F3DB07CCD5036819688847AB
:100E2000EEE747FA02F1C907C4D496F858C04CFA65
:100E300002F2D207BED5E0E747FA02F1C907AED504
:100E400096F858C04CFA02F2D307A8D401680B6890
:100E50009847A4E796F858307B4043FA02F1CB0755
:100E60009DD501680B68984799E747FA02FC5FEA4D
:100E7000CC7194D496F8583043FA02F2D2078ED54A
:100E8000E4E747FA05FC5FEACC727FF57DAF96F8A0
:100E900058302B41DB073FF577AF01680A68904770
:100EA00072E796F8581079402941C9077FF56CAF71
:100EB00001680A68904767E747FA05F2D2073FF5ED
:100EC00063AF96F858302B41DB077FF55DAFE4E761
:100ED00047FA05F1CA077FF54AAF96F858202A412C
:100EE000D3073FF544AF79E796F858307B402B4164
:100EF000D9077FF53CAF03681968884737E700BF1B
:100F000030B48369164C027F93F858302568016924
:100F100082B01341019503F00103019A81B1446845
:100F2000551AA54209D3A3B9826895424FF001032F
:100F300034BF002501254575037502B030BC7047EC
:100F4000002BFAD124680094009D056102B030BCEA
:100F50007047002101610175417502B030BC7047D6
:100F6000B4DE0120F8B5D0F890328269064600EB75
:100F7000C3001469D0F8CC12A7B2032B0F8035DD63
:100F8000A3F10802032A4BD90133122BA8BF002377
:100F900003F15907C6F8903216F8377006F529752F
:100FA00000242B6847FA04F228469B6802F00101EE
:100FB00001349847042C05F10805F2D11A48377D11
:100FC0004D2101FB070E9EF8435005F01F041F2C16
:100FD0000BD0B66915F0800F16BFF168102121F013
:100FE000100144F04002F1603260F8BD1A46B018BA
:100FF000D6F88C1290F8C4425CB1002440F2555CE3
:1010000067450A4494BF00270127147780F8C4720B
:10101000BAE740F25554A74294BF00240124EDE7FB
:10102000D0F88C522F88E2E798110400F8B500241C
:1010300090F8C872C0F89042064600F529752B68F2
:1010400047FA04F128469A6801F0010101349047FB
:10105000042C05F10805F2D1377D154BB06906EB7C
:10106000870C4D26DCF80C20046806FB073E55096A
:10107000A9009EF8437001F1604302F01F0603F5DA
:10108000614C012207F01F0144F0400402FA06F50A
:101090001F290460CCF8005009D03F064ABFC7683A
:1010A000102727F0100741F04003C7600360F8BD28
:1010B00098110400D0F8A012027D4B1C03F003032A
:1010C000F0B41C4C856900EB83064D27D6F88C6282
:1010D00007FB024C2A691CF80640C0F8A03204F055
:1010E0001F031F2B92B209D026064ABFEC681024BA
:1010F00024F0100443F04007EC602F60D0F89C020D
:101100000D4D06683368AB4212D1C768FC0708D59D
:10111000456880687E10AC592358A8199C46F0BCDD
:1011200060474668836806EB67009C46F0BC6047F2
:10113000F0BC184798110400A1120000037D194962
:1011400070B4D0F8A052846900EB830200EB8500F4
:10115000D268D0F88C5220684D2606FB031C51093A
:101160008B001CF8055003F1604606F5614C02F057
:101170001F02012105F01F0640F0400001FA02F3B2
:101180001F2E2060CCF8003009D02D064ABFE5683C
:10119000102525F0100546F04002E560226070BC85
:1011A000704700BF9811040010B4384B196883B021
:1011B00029B10B6FC2785C782CB9162A42D003B0E3
:1011C0005DF8044B7047197829B9162A3DD003B051
:1011D0005DF8044B704702F1FF3C0179BCF1160F3A
:1011E000EDD801A050F82CF0731200005912000045
:1011F000BF110000BF110000BF110000BF110000AF
:10120000BF110000BF110000BF110000BF1100009E
:10121000BF110000BF110000BF110000BF1100008E
:10122000BF110000BF110000BF110000BF1100007E
:10123000BF110000BF110000BF1100004B120000E1
:10124000531200001C78002CC5D10121597019706F
:10125000B5E700201870B2E70D4A0E4814680094F4
:1012600045F6E44C009A5A6000249C7040F80C103B
:10127000A5E7074A07481468019445F6E84C019A27
:101280005A6000249C7040F80C1098E70871FF1F0A
:10129000B4DE01201071FF1F704700BF704700BF10
:1012A00030B4C368DC0708D5456880685B10EC582B
:1012B0002458E818A44630BC604784684568A446B2
:1012C00005EB630030BC6047C368DA0706D55B10E6
:1012D00041688268C8588258C818104741688268B7
:1012E00001EB6300104700BF4368074AD8B211F012
:1012F000FF0F52F830304FF0010014BF83F8800028
:1013000083F80001704700BF14130400C9B20079CC
:101310000EF078BD10B5102104460EF081F820467D
:1013200010BD00BF08B500790EF05EFD08BD00BF1E
:10133000427B012A03460AD0826D416D8A4204D263
:10134000501C1A449865107D70470020704700B506
:10135000036883B0DB680DF10701984708B19DF879
:10136000070003B05DF804FB836830B4044642F222
:101370001075D87880060CD593F803C05FEA8C60AE
:1013800007D5D878800604D593F803C05FEA8C604F
:101390003BD4B0259D70A36842F21075D8788006C2
:1013A00007D493F803C05FEA8C6002D4D878800633
:1013B00060D5DD78A80641D5987840F030059D705D
:1013C000A36842F2107093F803C05FEA8C6507D4FB
:1013D000DD78AD0604D493F803C05FEA8C6533D59D
:1013E00042EA4102D1B21971A36842F21070DD786D
:1013F000AA0707D493F803C05FEA8C7502D4DA78A1
:10140000950750D5012030BC7047D8788006C0D5EC
:1014100093F803C05FEA8C60BBD5D8788006B8D556
:1014200093F803C05FEA8C60B3D5083DA1D19D70ED
:1014300000BFA06880218170657300BF00BF0423D6
:101440002373002030BC7047DD78AD06C8D493F814
:1014500003C05FEA8C65C3D4DD78AD06C0D493F8D1
:1014600003C05FEA8C65BBD4DD78AD06B8D408381C
:10147000A9D12BE093F803C05FEA8C6099D4D878A7
:10148000800696D493F803C05FEA8C6091D4D87834
:1014900080068ED493F803C05FEA8C6089D4083D3F
:1014A0007FF47CAFC3E7D9788907ABD4DD78AA078E
:1014B000A8D493F803C05FEA8C75A3D4DA789107B7
:1014C000A0D4D9788A079DD4083890D1987000BFED
:1014D000A36880259D70607300BF0122227330BC19
:1014E000704700BF10B50446D4ED007A007A2DEDA8
:1014F000028BB8EEE70A9FED0A8A20EE080A0EF08A
:101500007BFB6168207A012303FA01F202EBD271BE
:1015100019410EF067F984ED038ABDEC028B10BD12
:1015200000007A4510B50446D4ED007A007A2DED1E
:10153000028BB8EEE70A9FED0A8A20EE080A0EF049
:101540005BFB6168207A012303FA01F202EBD2719E
:1015500019410EF047F984ED038ABDEC028B10BDF2
:1015600000A00C4690F8643063B310B48268284C35
:1015700092F802C027490CF0FE039370026E1379B3
:101580002370046E22790A70816891F803C05FEAC3
:101590000C63FAD5046E204B22791A7081680224FC
:1015A000CC70826892F802C00CF0C7039370836815
:1015B00042F21071DC78A40605D400225DF8044BD9
:1015C00080F864207047DA789206F6D5DC78A406B5
:1015D000F3D593F803C05FEA8C62EED5DA7894060F
:1015E000EBD5DC78A206E8D593F803C05FEA8C64FB
:1015F000E3D5DA789206E0D50839DBD1997000BFDF
:10160000836880249C70417300BF01210173D4E77B
:101610001F8000401A8000401C800040B5EEC00AC8
:10162000F1EE10FAF0B500F1B980FDEEC07A451E7A
:10163000F8EEE70A17EE903A002130EE600A5A4EB3
:1016400000E0214686FB0324DA17C2EBA40707EB70
:10165000870CA3EB4C03303305F8013F4C1C3B4691
:10166000002FEED166107FD00219034612F801CD8B
:10167000077803F801CB751E06449E42177005F0EB
:10168000070771D0BFB3012F2DD0022F25D0032F14
:101690001DD0042F15D0052F0DD0062F05D01D7895
:1016A00012F801CD03F801CB15701D7812F8017DF9
:1016B00003F8017B15701D7812F801CD03F801CBFA
:1016C00015701D7812F8017D03F8017B15701D78E7
:1016D00012F801CD03F801CB15701D7812F8017DC9
:1016E00003F8017B157012F801CD1D7803F801CBCA
:1016F0009E42157038D01D4612F8017C93F800E028
:1017000005F8017B02F801EC5F7812F802CC83F84F
:1017100001C002F8027C6F7812F803EC85F801E052
:1017200002F8037CDD7812F8047CDF7002F8045CB8
:1017300093F804C012F8055C1D7102F805CC93F80B
:1017400005C012F8067C5F7102F806CC9D7912F88C
:10175000077C9F7102F8075C12F8087DDD79DF7164
:1017600008339E421570C6D1B2EE041A60EE011A1B
:101770000D4EBDEEE12A014412EE103A86FB03271E
:10178000DA17C2EBA70C0CEB8C05A3EB4506303641
:101790002E23002703558E70CF70F0BD2D230370CC
:1017A000B1EE400A013040E76766666638B5437BB4
:1017B00085689C1E012CEA78A97902D90223EB7076
:1017C00038BD5FFA82FC5FEACC642AD45FEA4C63DE
:1017D0002DD4CBB213F0500F044612D0A87940F0AC
:1017E0005002AA71A568A97901F0DF03AB71A06866
:1017F0000222C27025690DB1606DA8470221A5685B
:101800006173636D3F2B04D8581C606523442A79AB
:101810001A75A97941F05003AB71A4680225E570EF
:1018200038BD1022EA705FEA4C621CD58568002141
:101830004165816595F806C04CF02003AB71846862
:10184000C025A57081680A79530880F85C308C79CE
:1018500044F050058D7181684222CA708468032368
:10186000A279437338BD8568A97941F05002AA7105
:1018700080680224C47038BD0FB400B5C3B044AB57
:10188000FF2153F8042B019302A811F001FC02A8D8
:1018900011F056FB014602A80FF054FA43B05DF870
:1018A00004EB04B0704700BF437B012B0AD0816D6D
:1018B000426D914204D24B1C01448365087D704700
:1018C0000020704782B000218DF807109DF8073086
:1018D000836842F2107193F803C05FEA0C6227D468
:1018E000DA78120624D493F803C05FEA0C621FD49E
:1018F000DA7812061CD493F803C05FEA0C6217D49E
:10190000DA78120614D493F803C05FEA0C620FD49D
:10191000DA7812060CD40839DDD1997000BF8368DB
:1019200080229A70417300BF01210173002071E091
:10193000997801F0E7029A70836819795FFA81FC5F
:101940008DF807C09A7842F00801997083680222E6
:10195000DA70836842F2107193F803C05FEA8C7208
:101960001DD4DA7892071AD493F803C05FEA8C7218
:1019700015D4DA78920712D493F803C05FEA8C7218
:101980000DD4DA7892070AD493F803C05FEA8C7218
:1019900005D4DA78920702D40839DDD1BDE7997809
:1019A00001F0C7029A70826842F2107392F803C085
:1019B0005FEA8C612BD5D178890628D592F803C0CF
:1019C0005FEA8C6123D5D178890620D592F803C0CF
:1019D0005FEA8C611BD5D178890618D592F803C0CF
:1019E0005FEA8C6113D5D178890610D5083BDDD12B
:1019F000937000BF826880219170437300BF012102
:101A000082680173022118461379D17002E0022323
:101A10001079D37002B070472DE9F041AD4B1C68CE
:101A20008CB074B1617D01290ED0256EE26D9542B6
:101A30006ED26E1C254426662A7F1546461EAE428F
:101A40006BD00CB0BDE8F08100278DF806709DF8D2
:101A50000630236942F21071DD782F0616D493F810
:101A600003805FEA086611D493F803C05FEA0C654F
:101A70000CD4DA78120609D4DE78370606D4DF787B
:101A80003E0603D4DD782D0640F16581997801F09A
:101A9000E7029A7023691E79F7B28DF806709D7877
:101AA00045F00801997023690222DA70236942F235
:101AB0001071DE78B50700F10F81DF78BA0700F109
:101AC0000B81DD78AF0700F1078193F803C05FEA6F
:101AD0008C7600F1018193F803805FEA887500F14C
:101AE000FB80DA78920700F1F780DE78B70700F123
:101AF000F380DF78BE0700F1EF800839D9D1997003
:101B000000BF25698027AF70617500BF0121217575
:101B10000025461EAE422A4693D104F10808074626
:101B200040468DF80820FFF7BFFE8DF809004046BB
:101B3000FFF7BAFE8DF80A004046FFF7B5FE042F06
:101B40008DF80B0002A81DD041190DF10B020027E2
:101B500002264FF0800C4FF0010E07E05D1C23447D
:101B600025661B7F02F8013F8A420BD0637D012B63
:101B70000DD0236EE56DAB42F0D3002302F8013F98
:101B80008A42F3D16468A0470CB0BDE8F0818DF8BB
:101B900007709DF80730236942F21078DD782D0632
:101BA00024D4DD782D0621D4DD782D061ED4DD78F1
:101BB0002D061BD4DD782D0618D4DD782D0615D41E
:101BC000DD782D0612D4DD782D060FD4B8F1080883
:101BD000E4D183F8028000BF256985F802C084F84B
:101BE000158000BF002384F814E0C7E793F8028053
:101BF00008F0E7059D70236993F804805FFA88F583
:101C00008DF8075093F8028048F008059D7023690D
:101C1000DE70236942F21078DD78AD0718D4DD78E4
:101C2000AD0715D4DD78AD0712D4DD78AD070FD43C
:101C3000DD78AD070CD4DD78AD0709D4DD78AD07CC
:101C400006D4DD78AD0703D4B8F10808E4D1C0E7C5
:101C500093F8028008F0C7059D70D4F8108042F216
:101C6000107598F803309B062FD598F803309B0623
:101C70002BD598F803309B0627D598F803309B06A0
:101C800023D598F803309B061FD598F803309B06A0
:101C90001BD598F803309B0617D598F803309B06A0
:101CA00013D5083DDDD188F8025000BF236983F8C1
:101CB00002C0657500BFD4F8108084F814E02B468C
:101CC00098F8045088F803604CE798F8043088F8D6
:101CD000036047E778DC0120997801F0C7059D7023
:101CE000236942F2107193F803C05FEA8C672CD528
:101CF00093F803805FEA886627D5DA78950624D5BD
:101D0000DE78B20621D5DF78BF061ED5DD78AE06B7
:101D10001BD593F803C05FEA8C6516D593F8038052
:101D20005FEA886211D50839DDD1997000BF236957
:101D300080279F70617500BF0126236926750D46B7
:101D400002221979DA702A4678E6197902260D46B8
:101D50000A46DE7072E693F803805FEA08623FF598
:101D600095AE08397FF478AEC9E600BFD0ED047AAD
:101D700090ED067A90ED056AD0ED036AD0ED025A37
:101D800030EE670AB0EE675AA7EE005AF6EE004A48
:101D900075EE671A36EEE51A31EEC62AA2EE246A0F
:101DA00076EE052A80ED056AF4EEC12AF1EE10FA0E
:101DB000C0ED042A24D572EEA56AC0ED036AD0ED09
:101DC000003A90ED074A90ED010AF0EE007AB0EE8D
:101DD000637AA5EEA77AF0EE635A76EEC76AE6EE6E
:101DE000845AF4EEC05AF1EE10FA08D5F4EEE53A52
:101DF000F1EE10FA54BFB0EE630AB0EE650A704718
:101E000036EEA53AF4EEC32AF1EE10FAC4BF72EE34
:101E1000E56AC0ED036AD2E72DE9F04F002A9DF88C
:101E2000244069DB002B67DB7F2865DC7F2963DCCE
:101E30007F2AA8BF7F2220EAE07E7F2BA8BF7F23D6
:101E4000724521EAE1789C4656DB5F1CC8EB07002F
:101E5000DFF8A8A002F10109C7014FEAC81BC44579
:101E600044DB0EEB0B028023A7F18001BB420AF892
:101E70000240C1F3C215524438D0EDB1012D17D044
:101E8000022D13D0032D0FD0042D0BD0052D07D01C
:101E9000062D1CBF4FF4807382F88040D4548033E9
:101EA000D4548033D4548033D4548033D4548033C6
:101EB000D4548033BB4219D003F1800103F58076FE
:101EC00003F5C075D45403F500705454945503F5CC
:101ED0002071545503F5407603F5607503F5806372
:101EE000BB421454545494555455E5D10EF1010E8F
:101EF000CE45B4D1BDE8F08FBDE8F08F0831FF1FAB
:101F000001380B463A2800F25C82DFE810F05302F9
:101F10004C0245023E0237023002290222021B0215
:101F2000AE01A701A001990192018B0184017D01FD
:101F300076016F01680161015A0153014C014501AD
:101F40003E0137013001290122011B0113010B0160
:101F50000301FB00F300EB00E300DB00D300CB0048
:101F6000C300BB00B300AB00A3009B0093008B0039
:101F700083007B0073006B0063005B0053004B0029
:101F800043003B00BC48BD49C0F8EC201A463B204A
:101F90000DF04ABAB848BA49C0F8E8201A463A20C3
:101FA0000DF042BAB448B749C0F8E4201A463920C7
:101FB0000DF03ABAB048B449C0F8E0201A463820CB
:101FC0000DF032BAAC48B149C0F8DC201A463720CF
:101FD0000DF02ABAA848AE49C0F8D8201A463620D3
:101FE0000DF022BAA448AB49C0F8D4201A463520D7
:101FF0000DF01ABAA048A849C0F8D0201A463420DB
:102000000DF012BA9C48A549C0F8CC201A463320DE
:102010000DF00ABA9848A249C0F8C8201A463220E2
:102020000DF002BA94489F49C0F8C4201A463120E6
:102030000DF0FAB990489C49C0F8C0201A463020EB
:102040000DF0F2B98C489949C0F8BC201A462F20EF
:102050000DF0EAB988489649C0F8B8201A462E20F3
:102060000DF0E2B984489349C0F8B4201A462D20F7
:102070000DF0DAB980489049C0F8B0201A462C20FB
:102080000DF0D2B97C488D49C0F8AC201A462B20FF
:102090000DF0CAB978488A49C0F8A8201A462A2003
:1020A0000DF0C2B974488749C0F8A4201A46292007
:1020B0000DF0BAB970488449C0F8A0201A4628200B
:1020C0000DF0B2B96C488149C0F89C201A4627200F
:1020D0000DF0AAB968487E49C0F898201A46262013
:1020E0000DF0A2B964487B49C0F894201A46252017
:1020F0000DF09AB960487849C0F890201A4624201B
:102100000DF092B95C487549C0F88C201A4623201E
:102110000DF08AB958487249C0F888201A46222022
:102120000DF082B954486F49C0F884201A46212026
:102130000DF07AB950486C49C0F880201A4620202A
:102140000DF072B94C486949C2671A461F200DF05C
:102150006BB94948664982671A461E200DF064B97A
:102160004548644942671A461D200DF05DB9424852
:10217000614902671A461C200DF056B93E485F4976
:10218000C2661A461B200DF04FB93B485C49826677
:102190001A461A200DF048B937485A4942661A467D
:1021A00019200DF041B93448574902661A461820E3
:1021B0000DF03AB930485549C2651A4617200DF05E
:1021C00033B92D48524982651A4616200DF02CB9B4
:1021D0002948504942651A4615200DF025B9264870
:1021E0004D4902651A4614200DF01EB922484B498C
:1021F000C2641A4613200DF017B91F48484982647B
:102200001A4612200DF010B91B48464942641A467E
:1022100011200DF009B91848434902641A461020EC
:102220000DF002B914484149C2631A460F200DF05F
:10223000FBB811483E4982631A460E200DF0F4B8EF
:102240000D483C4942631A460D200DF0EDB80A488E
:10225000394902631A460C200DF0E6B806483749A2
:10226000C2621A460B200DF0DFB80348344982627F
:102270001A460A200DF0D8B884DD0120410D000077
:102280002D0D0000190D0000050D0000F10C0000DF
:10229000DD0C0000C90C0000B50C0000A10C000012
:1022A0008D0C0000790C0000650C0000510C000042
:1022B0003D0C0000290C0000150C0000010C000072
:1022C000ED0B0000D90B0000C50B0000B10B0000A6
:1022D0009D0B0000890B0000750B0000610B0000D6
:1022E0004D0B0000390B0000250B0000110B000006
:1022F000FD0A0000E90A0000D50A0000C10A00003A
:10230000AD0A0000990A0000850A0000710A000069
:102310005D0A0000490A0000350A0000210A000099
:102320000D0A0000F9090000E5090000D1090000CC
:10233000BD090000A90900009509000081090000FD
:102340006D0900001F48204942621A4609200DF01D
:102350006BB81C481D4902621A4608200DF064B88B
:1023600018481B49C2611A4607200DF05DB8154890
:10237000184982611A4606200DF056B811481649D0
:1023800042611A4605200DF04FB80E48134902610C
:102390001A4604200DF048B80A481149C2601A468E
:1023A00003200DF041B807480E4982601A4602200A
:1023B0000DF03AB803480C4942601A4601200DF06E
:1023C00033B8704784DD0120590900004509000039
:1023D000310900001D09000009090000F50800008E
:1023E000E1080000CD080000B908000008B5134658
:1023F00040680A461946FFF783FD08BD2DE9F04FF6
:10240000C14C0F78236895B005460A930A9E22684E
:102410000B920B9B40696B61013F032F00F2F3822B
:10242000DFE817F031022602030204009FEDB77ABD
:102430000023361A01EE106ADFEDB56AF8EE411A94
:10244000A1EEE67A85ED047AA8682F7B002B40F098
:10245000D482012390F8599003FA07F729EA070676
:10246000236880F859600693069E91F809A02068B9
:102470000790079F686E6F660AF1FF3BBBF1030F81
:1024800000F2C782DFE81BF0C601BB01980104001F
:102490009FED9E2A0023361A04EE106A9FED9C5A87
:1024A000F8EE444AA4EEC52A85ED182AA86D95F8E1
:1024B0005C70002B40F09B82012390F859E003FAF6
:1024C00007F72EEA0706236880F859600293029EF8
:1024D00091F80A8020680390039F686F6F6708F186
:1024E000FF39B9F1030F00F29682DFE819F05A01C3
:1024F0004F012C010400DFED855A0023361A00EE4F
:10250000106A9FED831AF8EE400AE0EEC15AC5ED5D
:102510001C5AA86E95F86C70002B40F06282012363
:1025200090F859B003FA07F72BEA0702DFED786A53
:10253000DFF8E0C180F859200E1D2B460020F2EE96
:102540000E4A01274FF08C0E22681292DDF8488067
:1025500011F801BFD4F80090CDF84C90DDF84CA0F4
:10256000D3F82490C3F824A00BF1FF32032A00F221
:102570004C82DFE812F0DC00D100A9000400DFED9E
:10258000631A0022C9EB080B03EE10BAF8EE433AC7
:10259000E3EEE61AC3ED081AD3F8189093F81C80FE
:1025A000002A40F07A8199F859A007FA08F22AEA3D
:1025B0000208226889F859800E92DDF8389016F8E2
:1025C00001BFD4F80080CDF83C80DDF83CA0D3F802
:1025D0008480C3F884A00BF1FF32032A00F2178233
:1025E000DFE802F0665B3C029FED484A0022C8EB40
:1025F000090B06EE10BAB8EE467AA7EE664A83EDEE
:10260000204AD3F8789093F87C80002A40F04E81DD
:1026100099F859A007FA08F22AEA020201300428C0
:1026200089F8592003F110038ED12C68206894F8A2
:102630005A10036800225E68B047002840F0878186
:102640006D68286895F85A10066800227768B847C0
:10265000002840F0338115B0BDE8F08F22680C925D
:10266000DDF830A04FEA9A0BACFB0BB2D2080EFBA0
:1026700012A2462A8CBF0022012293ED204AB5EE19
:10268000C04AF1EE10FABCDD24EE245AFDEEC55A24
:1026900015EE90AA0AF00102A9E722680D920D9AA0
:1026A000C2F30802B2F5807F8CBF00220122E4E76A
:1026B00093ED204AB5EEC04AF1EE10FAE4DCD3F80F
:1026C000789093F87C80A3E722681092DDF840A010
:1026D0004FEA9A0BACFB0BB2D2080EFB12A2462AB1
:1026E0008CBF00220122D3ED081AF5EEC01AF1EEDC
:1026F00010FA7FF751AF21EEA42AFDEEC22A12EEA6
:1027000090AA0AF001023DE7B4DE0120CDCCCC3E18
:102710006F12833A3BA8833A22681192119AC2F34E
:102720000802B2F5807F8CBF00220122DBE7D3EDE7
:10273000081AF5EEC01AF1EE10FADCDCD3F81890A6
:1027400093F81C802FE722680092009FB34BBA08D1
:10275000A3FB0232D2084FF08C0A0AFB1273462BFD
:102760008CBF00230123D5ED1C5AF5EEC05AF1EEC3
:1027700010FA7FF7CEAEB2EE0E6A25EE867AFDEE47
:10278000C77A17EE902A02F00103B7E6276801978F
:10279000019BC3F30803B3F5807F8CBF00230123A3
:1027A000E1E7D5ED1C5AF5EEC05AF1EE10FAE2DC85
:1027B000A86E95F86C70B2E622680492049F974B5D
:1027C000BA08A3FB0232D2084FF08C0C0CFB127338
:1027D000462B8CBF0023012395ED182AB5EEC02AA5
:1027E000F1EE10FA7FF762AEF2EE0E2A22EE223AF6
:1027F000FDEEC33A13EE902A02F001034BE6276880
:102800000597059BC3F30803B3F5807F8CBF0023B6
:102810000123E1E795ED182AB5EEC02AF1EE10FA92
:10282000E2DCA86D95F85C7046E622680892089F85
:102830007A4BBA08A3FB0232D2084FF08C0808FB8F
:102840001273462B8CBF0023012395ED047AB5EE5D
:10285000C07AF1EE10FA7FF7F7ADF2EE0E7A27EEBE
:10286000270AFDEEC00A10EE902A02F00103E0E50F
:1028700027680997099BC3F30803B3F5807F8CBFD2
:1028800000230123E1E795ED047AB5EEC07AF1EE7D
:1028900010FAE2DCA8682F7BDBE599F859B002FA60
:1028A00008FA4BEA0A025FFA82F882E699F859B010
:1028B00002FA08F84BEA0802D2B2AFE6286895F8A7
:1028C00059100468A268904700283FF4C4AE2968F4
:1028D000886890F802C00CF0C70383708B6842F2DE
:1028E0001070DD78AF067FF5B6AEDE78B6067FF500
:1028F000B2AEDF78BD067FF5AEAEDC78A4067FF51C
:10290000AAAE93F803E05FEA8E627FF5A4AE93F877
:1029100003905FEA89677FF59EAE93F803A05FEAB4
:102920008A667FF598AE93F803B05FEA8B657FF512
:1029300092AE0838D5D1987000BF8B6880229A700B
:10294000487300BF0120087315B0BDE8F08F206800
:1029500094F859100768BA68904700283FF470AEA1
:1029600021688868847804F0C70383708B6842F21A
:102970001070DE78B4067FF563AEDF78BA067FF5B7
:102980005FAE93F803C05FEA8C647FF559AE93F8AD
:1029900003E05FEA8E627FF553AE93F803905FEA3F
:1029A00089677FF54DAE93F803A05FEA8A667FF5ED
:1029B00047AE93F803B05FEA8B647FF541AE93F8BE
:1029C00003805FEA88627FF53BAE0838D1D198700A
:1029D00000BF8C688022A270487300BF01230B7374
:1029E0002EE690F85960BB403343DAB29EE590F88A
:1029F0005920BB401343DEB265E590F85920BB4037
:102A00001343DEB22CE501231FE701226BE601220E
:102A100033E60123E0E60123A5E600BF3BA8833AA5
:102A200010B504464068134A03681B6893421DD1E1
:102A3000007901210DF0E6F9606801688A680121DA
:102A4000904732200DF03EFA6068036800219A68D2
:102A5000904732200DF036FA606804680121A368BF
:102A600098473220BDE810400DF02CBA012198475C
:102A7000E2E700BF0D130000F8B504460068294ADC
:102A80000368277B5D6895420E4645D190F8642027
:102A9000002A3BD09A680021904720680768314699
:102AA000BD68A84721688868847804F0C7068670E6
:102AB0008B6842F2107093F803C05FEA8C6500D413
:102AC000F8BD93F803E05FEA8E64F9D5DA789206F0
:102AD000F6D5DF78BF06F3D5DD78AE06F0D5DC7825
:102AE000A506EDD5DE78B406EAD593F803C05FEA13
:102AF0008C62E5D50838DED1987000BF8B688022E3
:102B00009A70487300BF01200873F8BD3946FEF77C
:102B10002BFC20680368BDE739460022A8472068DF
:102B20000368B7E71D0700002DE9F041044600687F
:102B30009D4F0368217B5D68BD4240F0168190F88F
:102B40006420002A7CD09A68984D0021904705F1B6
:102B50001B0820682E46036816F8011B9A689047E8
:102B60002068697803689A689047206871780668D9
:102B7000B36898472068E97802689668B04720688B
:102B8000297903689A689047206869790668B3686C
:102B900098472068A97902689668B0472068E97963
:102BA00003689A6890472068297A06680935B368EF
:102BB00098474545CDD121688868857805F0C702DA
:102BC00082708B6842F21070DE78B60611D44FF432
:102BD00000520021A06810F00DF9227D002A34D0A7
:102BE00064200DF06FF92046AF21FFF745FFBDE8E7
:102BF000F081DD78AD06EAD593F803C05FEA8C6614
:102C0000E5D593F803E05FEA8E65E0D593F803809D
:102C10005FEA8862DBD5DA789606D8D5DE78B50625
:102C2000D5D5DD78AA06D2D50838CDD1987000BFA9
:102C30008B6880229A70487300BF01200873C6E732
:102C4000FEF792FB206803687DE72068217B05681A
:102C50006E68BE4240F0978090F86420002A00F031
:102C60008980AF684021B847256895F8641000292D
:102C7000B6D1A0682169AB68E866296742F2107690
:102C800093F803C05FEA0C622AD493F803E05FEA8A
:102C90000E6725D493F803805FEA086220D4DA78BF
:102CA00017061DD4DF783A061AD493F803C05FEAFA
:102CB0000C6715D493F803E05FEA0E6210D493F822
:102CC00003805FEA08670BD4083ED9D19E7000BF2D
:102CD000AB68802098706E7300BF01262E737FE76B
:102CE0009E7946F050029A71AB681227DF70AE6889
:102CF000B278012942F01003B37048D02B6E1A68E5
:102D00000026D671D3F800C0471C176001279780B2
:102D1000CCF808701F6801391FFA81FEA7F81EE081
:102D20001B684A42FA60A3F816E0296EAF680B6888
:102D300004379E71B7F1804F1F619E820F681ED2CB
:102D40000122BA600F68296E194A0023BB610E790F
:102D50001670AF68B97841F00102BA70AB680078BC
:102D60001871012685F864603AE70022A8472068B8
:102D70000368E8E6FEF7F8FA2068056871E7BE68C0
:102D8000002EE0D1DCE7B0472068056869E72F68CE
:102D90000178BA6828469047A86E00283FF420AF13
:102DA0000568296888471BE71D0700001C6F0100A4
:102DB0001B8000402DE9F04F42F296038046C05C34
:102DC00083B0002840F0388108F501513C31019171
:102DD000DFF8F492A8F1020A09F5804BD9F80470E3
:102DE000D9F80860D9F80C50D9F8104009F1140C42
:102DF0009CE807004FEA172E4FEA174C0CF4706C52
:102E00002EF47F6E4CEA0E0E07F0F0074FEA164CD8
:102E10004EEA07074FEA162E0CF4706C2EF47F6E04
:102E20004CEA0E0E06F0F0064FEA154C4EEA060686
:102E30004FEA152E0CF4706C2EF47F6E4CEA0E0ED9
:102E400005F0F0054FEA144C4EEA05054FEA142E42
:102E50000CF4706C2EF47F6E4CEA0E0E04F0F0044D
:102E60004FEA104C4EEA04044FEA102E0CF4706C3A
:102E70002EF47F6E4CEA0E0E00F0F0004FEA114C7B
:102E80004EEA00004FEA112E0CF4706C2EF47F6EA7
:102E90004CEA0E0E01F0F0014FEA124C4EEA01012D
:102EA0004FEA122E59F8203FAAF802700CF4706C09
:102EB0002EF47F6E4CEA0E0E02F0F0024FEA134C35
:102EC0004EEA02024FEA132E0CF4706C2EF47F6E61
:102ED0004CEA0E0E03F0F0034EEA030CCB45AAF8C1
:102EE0000460AAF80650AAF80840AAF80A00AAF84E
:102EF0000C10AAF80E202AF810CF7FF46FAF019FB4
:102F00003A7D42F27C0912B103B0BDE8F08F58F867
:102F100009006B4E0468397B6568B54240F0BB80A0
:102F200090F86420002A00F0A780A2684021904712
:102F300042F27C0058F8004094F864100029E3D174
:102F4000019B98681969A368E066216742F21075D1
:102F5000DF783E062AD4DE78320627D493F803B011
:102F60005FEA0B6722D493F803E05FEA0E661DD494
:102F700093F803C05FEA0C6218D493F803905FEAF9
:102F8000096713D493F803A05FEA0A660ED4DA78CF
:102F900012060BD4083DDBD19D7000BFA3688026CC
:102FA0009E70657300BF01202073ADE79D7945F0E9
:102FB00050079F71A3681226DE70A26895780129D8
:102FC00045F0100797706BD0236E1A680025D571F5
:102FD0001F68461C166001269680BE601F68013976
:102FE0001FFA81F8A7F81E801B684A42FA60A3F80E
:102FF0001680266EA768316804378D71B7F1804F4F
:103000000F618D82336842D201229A603368266E46
:103010002C4F0021996135793D70A26892F802B079
:103020004BF0010393700078A6680127307184F893
:10303000647003B0BDE8F08F08F5015242F29406C7
:1030400014463C3418F8067001942046812142F25F
:103050009509FFF711FD39462046FFF70DFD18F8D9
:1030600009307BB9A7210198FFF706FD42F29600CF
:10307000002108F80010ABE6FEF776F958F80900D1
:10308000046852E7A4210198FFF7F6FCEEE79D687B
:10309000002DBCD1B8E7A84758F80900046844E7F8
:1030A00025680178AA6820469047A06E00283FF462
:1030B0002BAF0468216803B0BDE8F04F084700BF9C
:1030C0001D0700001B8000400431FF1F10B403687F
:1030D00041681A7890F809C00C78037A14EA0C0F4A
:1030E00002EA03021DD0847A04F003010AB141F020
:1030F000040141F008039A1003F1FF3C8272BCF115
:103100000D0F0BD8DFE80CF021071B070A15212152
:10311000150A071B0721C268531EC3605DF8044BE4
:103120007047817A01F00303002AE4D043F00403DE
:10313000E1E7C3689C1EC4605DF8044B7047C1683A
:103140005DF8044B0231C1607047C4680134C4604B
:103150005DF8044B704700BF08B5034BD3F8EC0093
:10316000FFF7B4FF08BD00BF7CDC012008B5034BAE
:10317000D3F8E800FFF7AAFF08BD00BF7CDC012000
:1031800008B5034BD3F8E400FFF7A0FF08BD00BF6C
:103190007CDC012008B5034BD3F8E000FFF796FF75
:1031A00008BD00BF7CDC012008B5034BD3F8DC0070
:1031B000FFF78CFF08BD00BF7CDC012008B5034B86
:1031C000D3F8D800FFF782FF08BD00BF7CDC0120E8
:1031D00008B5034BD3F8D400FFF778FF08BD00BF54
:1031E0007CDC012008B5034BD3F8D000FFF76EFF5D
:1031F00008BD00BF7CDC012008B5034BD3F8CC0030
:10320000FFF764FF08BD00BF7CDC012008B5034B5D
:10321000D3F8C800FFF75AFF08BD00BF7CDC0120CF
:1032200008B5034BD3F8C400FFF750FF08BD00BF3B
:103230007CDC012008B5034BD3F8C000FFF746FF44
:1032400008BD00BF7CDC012008B5034BD3F8BC00EF
:10325000FFF73CFF08BD00BF7CDC012008B5034B35
:10326000D3F8B800FFF732FF08BD00BF7CDC0120B7
:1032700008B5034BD3F8B400FFF728FF08BD00BF23
:103280007CDC012008B5034BD3F8B000FFF71EFF2C
:1032900008BD00BF7CDC012008B5034BD3F8AC00AF
:1032A000FFF714FF08BD00BF7CDC012008B5034B0D
:1032B000D3F8A800FFF70AFF08BD00BF7CDC01209F
:1032C00008B5034BD3F8A400FFF700FF08BD00BF0B
:1032D0007CDC012008B5034BD3F8A000FFF7F6FE15
:1032E00008BD00BF7CDC012008B5034BD3F89C006F
:1032F000FFF7ECFE08BD00BF7CDC012008B5034BE6
:10330000D3F89800FFF7E2FE08BD00BF7CDC012087
:1033100008B5034BD3F89400FFF7D8FE08BD00BFF3
:103320007CDC012008B5034BD3F89000FFF7CEFEFC
:1033300008BD00BF7CDC012008B5034BD3F88C002E
:10334000FFF7C4FE08BD00BF7CDC012008B5034BBD
:10335000D3F88800FFF7BAFE08BD00BF7CDC01206F
:1033600008B5034BD3F88400FFF7B0FE08BD00BFDB
:103370007CDC012008B5034BD3F88000FFF7A6FEE4
:1033800008BD00BF7CDC012008B5024BD86FFFF7F9
:103390009DFE08BD7CDC012008B5024B986FFFF74D
:1033A00095FE08BD7CDC012008B5024B586FFFF785
:1033B0008DFE08BD7CDC012008B5024B186FFFF7BD
:1033C00085FE08BD7CDC012008B5024BD86EFFF7F6
:1033D0007DFE08BD7CDC012008B5024B986EFFF72E
:1033E00075FE08BD7CDC012008B5024B586EFFF766
:1033F0006DFE08BD7CDC012008B5024B186EFFF79E
:1034000065FE08BD7CDC012008B5024BD86DFFF7D6
:103410005DFE08BD7CDC012008B5024B986DFFF70E
:1034200055FE08BD7CDC012008B5024B586DFFF746
:103430004DFE08BD7CDC012008B5024B186DFFF77E
:1034400045FE08BD7CDC012008B5024BD86CFFF7B7
:103450003DFE08BD7CDC012008B5024B986CFFF7EF
:1034600035FE08BD7CDC012008B5024B586CFFF727
:103470002DFE08BD7CDC012008B5024B186CFFF75F
:1034800025FE08BD7CDC012008B5024BD86BFFF798
:103490001DFE08BD7CDC012008B5024B986BFFF7D0
:1034A00015FE08BD7CDC012008B5024B586BFFF708
:1034B0000DFE08BD7CDC012008B5024B186BFFF740
:1034C00005FE08BD7CDC012008B5024BD86AFFF779
:1034D000FDFD08BD7CDC012008B5024B986AFFF7B2
:1034E000F5FD08BD7CDC012008B5024B586AFFF7EA
:1034F000EDFD08BD7CDC012008B5024B186AFFF722
:10350000E5FD08BD7CDC012008B5024BD869FFF75A
:10351000DDFD08BD7CDC012008B5024B9869FFF792
:10352000D5FD08BD7CDC012008B5024B5869FFF7CA
:10353000CDFD08BD7CDC012008B5024B1869FFF702
:10354000C5FD08BD7CDC012008B5024BD868FFF73B
:10355000BDFD08BD7CDC012008B5024B9868FFF773
:10356000B5FD08BD7CDC012008B5024B5868FFF7AB
:10357000ADFD08BD7CDC012001380B463A2800F285
:103580005C82DFE810F053024C0245023E02370233
:103590003002290222021B02AE01A701A0019901FB
:1035A00092018B0184017D0176016F016801610147
:1035B0005A0153014C0145013E01370130012901F7
:1035C00022011B0113010B010301FB00F300EB00BF
:1035D000E300DB00D300CB00C300BB00B300AB00B3
:1035E000A3009B0093008B0083007B0073006B00A3
:1035F00063005B0053004B0043003B00BC4ABD49E5
:10360000C2F8EC303B2004220BF00EBFB848BA4998
:10361000C0F8E83004223A200BF006BFB44AB7499C
:10362000C2F8E430392004220BF0FEBEB048B449A1
:10363000C0F8E030042238200BF0F6BEAC4AB149A5
:10364000C2F8DC30372004220BF0EEBEA848AE49A9
:10365000C0F8D830042236200BF0E6BEA44AAB49AD
:10366000C2F8D430352004220BF0DEBEA048A849B1
:10367000C0F8D030042234200BF0D6BE9C4AA549B5
:10368000C2F8CC30332004220BF0CEBE9848A249B9
:10369000C0F8C830042232200BF0C6BE944A9F49BD
:1036A000C2F8C430312004220BF0BEBE90489C49C1
:1036B000C0F8C030042230200BF0B6BE8C4A9949C5
:1036C000C2F8BC302F2004220BF0AEBE88489649C9
:1036D000C0F8B83004222E200BF0A6BE844A9349CD
:1036E000C2F8B4302D2004220BF09EBE80489049D1
:1036F000C0F8B03004222C200BF096BE7C4A8D49D5
:10370000C2F8AC302B2004220BF08EBE78488A49D8
:10371000C0F8A83004222A200BF086BE744A8749DC
:10372000C2F8A430292004220BF07EBE70488449E0
:10373000C0F8A030042228200BF076BE6C4A8149E4
:10374000C2F89C30272004220BF06EBE68487E49E8
:10375000C0F89830042226200BF066BE644A7B49EC
:10376000C2F89430252004220BF05EBE60487849F0
:10377000C0F89030042224200BF056BE5C4A7549F4
:10378000C2F88C30232004220BF04EBE58487249F8
:10379000C0F88830042222200BF046BE544A6F49FC
:1037A000C2F88430212004220BF03EBE50486C4900
:1037B000C0F88030042220200BF036BE4C4A694904
:1037C000D3671F2004220BF02FBE49486649836748
:1037D00004221E200BF028BE454A644953671D2071
:1037E00004220BF021BE42486149036704221C20D9
:1037F0000BF01ABE3E4A5F49D3661B2004220BF031
:1038000013BE3B485C49836604221A200BF00CBEB1
:10381000374A5A495366192004220BF005BE344832
:1038200057490366042218200BF0FEBD304A554963
:10383000D365172004220BF0F7BD2D48524983654C
:10384000042216200BF0F0BD294A5049536515207B
:1038500004220BF0E9BD26484D49036504221420DB
:103860000BF0E2BD224A4B49D364132004220BF033
:10387000DBBD1F4848498364042212200BF0D4BDED
:103880001B4A46495364112004220BF0CDBD184851
:1038900043490364042210200BF0C6BD144A414979
:1038A000D3630F2004220BF0BFBD11483E49836350
:1038B00004220E200BF0B8BD0D4A3C4953630D2085
:1038C00004220BF0B1BD0A483949036304220C20DD
:1038D0000BF0AABD064A3749D3620B2004220BF035
:1038E000A3BD03483449836204220A200BF09CBD27
:1038F0007CDC0120593100006D3100008131000075
:1039000095310000A9310000BD310000D131000027
:10391000E5310000F93100000D32000021320000D5
:1039200035320000493200005D3200007132000083
:103930008532000099320000AD320000C132000033
:10394000D5320000E9320000FD32000011330000E2
:1039500025330000393300004D330000613300008F
:10396000753300008933000099330000A93300004B
:10397000B9330000C9330000D9330000E933000037
:10398000F933000009340000193400002934000024
:103990003934000049340000593400006934000013
:1039A000793400008934000099340000A934000003
:1039B000B9340000C9340000D93400001F4A20493E
:1039C0005362092004220BF02FBD1C481D490362DD
:1039D000042208200BF028BD184A1B49D361072098
:1039E00004220BF021BD15481849836104220620EA
:1039F0000BF01ABD114A16495361052004220BF041
:103A000013BD0E4813490361042210460BF00CBD90
:103A10000A4A1149D360032004220BF005BD074870
:103A20000E498360042202200BF0FEBC034A0C49BD
:103A30005360012004220BF0F7BC70477CDC0120AE
:103A4000E9340000F93400000935000019350000A0
:103A5000293500003935000049350000593500008E
:103A60006935000070B5234B036104460D461646C8
:103A700000216FF00042C260836181724561C661BE
:103A80000221E8B20CF0BEF9207F02210CF0BAF955
:103A9000194850F83510012201F500732360227295
:103AA00050F83600627200F50071616002200CF07F
:103AB00009FA226894F808C0137813EA0C0F03D0AF
:103AC000A07A40F00101A172626894F809E01378CD
:103AD00013EA0E0F03D0A07A40F00201A17228462B
:103AE0002146FFF749FD30462146FFF745FD2046B8
:103AF00070BD00BF706E010014130400F0B486B0F6
:103B000072B6C26862B6C04C066A23680593059F08
:103B1000456ABE1B92080E2E426200F30A81C56AF6
:103B20000D6372B6C26B62B627680497049F066D78
:103B3000436DBE1B95080E2E456500F3CE80C56D06
:103B40004D6372B6C26E62B627680397039FD0F8C2
:103B50008060D0F88430BE1B95080E2EC0F88450CB
:103B600000F38780D0F88C508D6372B6D0F89C201B
:103B700062B627680297029FD0F8B060D0F8B430E0
:103B8000BE1B95080E2EC0F8B4503EDCD0F8BC50D9
:103B9000CD6372B6D0F8CC7062B624680194019AF5
:103BA000D0F8E060D0F8E450BB08971B0E2FC0F8A7
:103BB000E43040F31C81D0F8E8405B1B18BFC0F82C
:103BC000E0209A0292FBF7F6002C40F0DC8004EB38
:103BD0004404A21948BF0332951085EAE5768B4F5D
:103BE000A6EBE57CACF1020687FB0642A2EBE6778A
:103BF0000137D0F8EC40C0F8E85007FB0343C0F8A9
:103C0000EC300B6406B0F0BC7047ED1A18BFC0F87A
:103C1000B070D0F8B870AA0292FBF6F6002F40F010
:103C2000BC8007EB4707BA1948BF0332961086EAF3
:103C3000E673A3EBE67CACF10207012FC0F8B86095
:103C400040F3B580BA10A2F10B06171F26EAE673FF
:103C5000002FA8BFDB1901321A44012A00F0A78007
:103C6000561E7200D0F8BC3002FB0535C0F8BC50BF
:103C70008EE7ED1A18BFC0F88070D0F88870AA02DD
:103C800092FBF6F6002F40F0A68007EB4707BA1923
:103C900048BF0332961086EAE673A3EBE67CACF1EC
:103CA0000207012FC0F8886040F39F80BA10A2F18C
:103CB0000B06171F26EAE673002FA8BFDB19013297
:103CC0001A44012A00F09180561E7200D0F88C3000
:103CD00002FB0535C0F88C5046E7ED1A18BF0765A2
:103CE000876DAA0292FBF6F6002F6BD107EB470710
:103CF000BA1948BF0332961086EAE673A3EBE67C56
:103D0000ACF10207012F866563DDBA10161FA2F120
:103D10000B0726EAE673002FA8BFDB1901321A440D
:103D2000012A56D0561E7200C36D02FB0535C565CB
:103D300006E7836A551B18BF0762AF0297FBF6F2CE
:103D4000BBBB03EB43039F1848BF0337BE1086EA93
:103D5000E67CACEBE672931E012B866230DD9F1091
:103D6000A7F10B063A1F26EAE67C002AA8BF944476
:103D700001376744012F23D07B1E5F00C66A07FB13
:103D80000565C562CCE6002E3FF421AF35DD002C81
:103D90003FF71DAF012700252BE7002E3FF441AF71
:103DA00036DD002F3FF73DAF0023C0F8B8300122C9
:103DB00058E7002AC5D023DD002BC2DC002686622E
:103DC0000127DBE7002E91D025DD002F8EDC0023BC
:103DD00083650122A8E7002E3FF457AF1EDD002FB8
:103DE0003FF753AF0023C0F8883001226EE7D0F8C8
:103DF000EC300B6406B0F0BC7047002CCADCE6E681
:103E0000002BDBDC9DE700BFB4DE0120ABAAAA2AB1
:103E1000002FC9DC05E7002FD9DC67E7002FE1DCC4
:103E200033E700BF10B50446D4ED007A007A2DEDDB
:103E3000028BB0EE408AB8EEE70A20EE080A0BF0DB
:103E4000DBFE6168207A012303FA01F202EBD271F2
:103E500019410BF0C7FC84ED038ABDEC028B10BD49
:103E60002DE9F04F854B854ADD6A196854689BB08F
:103E7000002D1191064640F38181032D57DC304619
:103E80000FF05EF83278002A5AD000284FF0000E6A
:103E9000ACBF07466FF00047F44606F1FF3801203B
:103EA00018F8013F33B99FB918F8013F4FF0FF37B9
:103EB000002BF8D00A2B04D01F2BF1D90EF1060EDF
:103EC000EEE7F445B8BFF44601304FF0000EE7E7E7
:103ED0006A4FB96A083100FB01F06849F44505FBF7
:103EE00000F7C8686346B8BF734605FB03F30128B3
:103EF00016932CD0022800F04481604B19690129E7
:103F000030D0022908BFE41B5C4BDFF870B1D3F856
:103F100018E0196A119B01EB0E0843459C4603DA31
:103F200016998C44E64522DB1BB0BDE8F08F534860
:103F30000325C56230460FF003F83278002AA4D179
:103F40004E491692C86801284FEAC507D2D1169982
:103F5000119B01EBD179A3EB6901484B11911969D0
:103F60000129CED107EBD77AA4EB6A04CCE7DBF8C2
:103F70001CE0DBF8243073449C42D5DA2744BE456C
:103F8000D2DA002AD0D00996CDF864B00A2A099F67
:103F900000F0DB853E461346002102E00A2B00F0CC
:103FA000A0831F2B16F8013F88BF0131002BF5D1EC
:103FB00001EB410E4FEA4E01179605FB01FE2F4E15
:103FC000B76A083705FB07F90128A9EBC50600F019
:103FD0009283022800F0B185119806902749087D48
:103FE000002840F0D38009EB04032644022D0E93F1
:103FF000109600F08A83032D40F0FF80002A00F025
:10400000AE810A2A00F0AB811C4E109D1B4C316A18
:10401000776AD6F81890D6F81CB0237A0293203A23
:10402000EE01D0B2AB1C09EB010A01350BEB070125
:104030006B2806F1020703910A970C930B9500F287
:1040400026830F4E56F820703E78069C0A990D4B39
:10405000059701EB04080022601CA11CDDF830E08C
:10406000DDF82CC0109F04920790984408910846F0
:10407000224607994446002335E000BF10CEFF1FBB
:104080005CFF01000831FF1F814500F37381824509
:1040900040F37081894540F34782BB4505DC039DB1
:1040A000BD42C4BF9DF808502570E34506DC039D62
:1040B000654503DD9DF8085084F88050F34506DC23
:1040C000039D754503DD9DF8085084F800510133C8
:1040D000062B02F1030204F1030401F1030100F1D4
:1040E000030000F0678146FA03F5ED07EFD591452F
:1040F000CADC824500F37381814540F3968189458E
:1041000000F37281924540F30582BB4500F389823A
:10411000039DBD4240F385829DF8085004F8025C7F
:104120008A4506DD9DF8085004F8015C924540F38D
:10413000E381E34500F3E081039D654540F3DC81C5
:104140009DF8085084F87E508A4540F3AE829DF871
:10415000085084F87F50924540F32481F345B6DC43
:10416000039D7545B3DD9DF8085084F8FE508A45DF
:10417000ADDD9DF8085084F8FF50A8E70125D56211
:104180007DE6119B16995B1A1193B6E6199A517D3B
:104190009069D2F81CA0136A576A0091069909EB3E
:1041A00004028946F14400EB030E0E920EF1FF3833
:1041B00009F1FF3242450AEB070B0E9FA8BF4246AA
:1041C0008842B8BF08460BF1FF3307F1FF3CA24518
:1041D0005146B8BF21466345A8BF6346FDF71CFEA4
:1041E0003019099E1090022D327800F08E82032D36
:1041F0003FF404AF002A00F0B2800A2A00F0AF803A
:10420000B94DB94FD5F81CB0387A6B6A109FA969BF
:104210002E6A069D07905B44F80105350E44059310
:1042200006900837A2F1200A5FFA8AF36B2B96BF3B
:10423000AE4AAF4C52F82340069AAE4B0395501944
:10424000013C05F1FF3E109ACDF810E01844A5F1AD
:10425000050AA5F10409A5F10308A5F1020C0294D1
:10426000029D15F8013F0295DC070FD551450DDC85
:1042700056450BDD934509DC059C944206DD039D04
:10428000441B9DF81C5004F80A50A6469D070FD504
:1042900049450DDC4E450BDD934509DC059C9442F8
:1042A00006DD039D441B9DF81C5004F80950A646EA
:1042B0005C070FD541450DDC46450BDD934509DC18
:1042C000059C944206DD039D441B9DF81C5004F898
:1042D0000850A6461D070FD58C450DDBB4450BDAFB
:1042E000934509DC059C944206DD039D441B9DF823
:1042F0001C5004F80C50A646DC0611D5049DA942BA
:104300002C460DDCAE420BDD934509DC059C944246
:1043100006DD039C041BA6469DF81C400EF80540D4
:104320009B060CD5039B994209DC9E4207DD934511
:1043300005DC059D9542C4BF9DF81C5005700132F7
:10434000974200F180008BD10998039D10F8012F4E
:10435000099022B10A2A05F106057FF463AF179E82
:104360000E9C3278002A3FF4DFAD5F490996CD6A92
:10437000C8680BE689453FF7AAAE8A457FF7A7AE26
:10438000BB4506DC039DBD4203DD9DF8085004F8E3
:10439000015CE34506DC039D654503DD9DF808509F
:1043A00084F87F50F3453FF792AE039D75453FF784
:1043B000E0AE8CE6049E0336182E049608F5C0780D
:1043C0000EF1030E07F103070CF1030C00F04D8111
:1043D000059A089812F8016F0592069A49E68145F8
:1043E00051DD4945BFF68EAE92457FF770AEBB45B5
:1043F00006DC039DBD4203DD9DF8085004F8025C15
:10440000E34506DC039D654503DD9DF8085084F80F
:104410007E50F3453FF75BAE039D75457FF757AE82
:104420009DF8085084F8FE5051E68945DCDC924541
:1044300040F34281BB4500F34A81039DBD4240F3F6
:1044400046819DF8085004F8025C8A4506DD9DF817
:10445000085004F8015C924540F31C81E34500F3E9
:104460001981039D654540F315819DF8085084F836
:104470007E508A4540F32E819DF8085084F87F5085
:1044800092458FDD6AE68A457ADC924540F3D98011
:10449000BB450CDC039DBD4209DD9DF8085004F8C6
:1044A000025C9DF808502570924540F3D080E345AA
:1044B0000DDC039D65450ADD9DF8085084F87E50AB
:1044C0009DF8085084F8805092457FF7F7ADF3458A
:1044D0003FF7FDAD039D75457FF7F9AD9DF8085099
:1044E00084F8FE50EFE500BF10CEFF1F5CFF010017
:1044F000F0B301000831FF1F8A4507DDE3453FF7B0
:104500002AAE039D65457FF726AE20E692457FF7EC
:10451000DEAD23E68A45F9DDBB453FF707AE039DD7
:10452000BD427FF703AEFDE58A457EDDBB450BDC72
:10453000039DBD4208DD9DF8085004F8015C9DF81C
:10454000085025708A4575DDE3450DDC039D654502
:104550000ADD9DF8085084F87F509DF8085084F8D3
:1045600080508A457FF7AAADF3453FF7B0AD039D74
:1045700075457FF7ACAD9DF8085084F8FF50A2E573
:10458000924542DDBB4540DC039DBD423DDD9DF8CB
:10459000085004F8025C89453EDD039DBD4202DD02
:1045A0009DF80850257092451FDDE3451DDC039DF5
:1045B00065451ADD9DF8085084F87E5089451BDD5D
:1045C000039D654503DD9DF8085084F880509245B1
:1045D00017DDF34515DC039D754512DD9DF8085088
:1045E00084F8FE508945C6DD6AE5894537DCE34538
:1045F000EDDC039D6545EADD9DF8085084F87F50A9
:10460000E1E789453FF75AADAEE789452ADCBB456E
:10461000C9DC039DBD42C6DD9DF8085004F8015C6D
:10462000BEE78A453FF778AF83E5BB4502DC039DD3
:10463000BD4284DCE3453FF741AD039D65458CDC1D
:104640003CE5BB4503DC039DBD423FF72AAFE34594
:104650003FF734AD039D65453FF732AF2EE5E345A7
:10466000B5DCADE7BB459EDC97E70999069B11F8E1
:10467000012F099112330693002A3FF470AE0A2AE3
:104680003FF46DAE203AD0B26B287FF6DAAC9B4F88
:104690000026DAE48A457FF739AFE3453FF7F0AE0D
:1046A000039D65457FF7ECAEE6E692453FF756ADD4
:1046B0008A453FF777AE0AE58A457FF727AFBB45C6
:1046C0003FF7C9AE039DBD427FF7C5AEBFE68A4541
:1046D000F5DCC3E692453FF741AD8A457FF7F7AC7D
:1046E00060E601EB41077B00179605FB03FE3746AA
:1046F0000137179763E41698119BCEEB000A0AEB7B
:10470000DA7B03EB6B07069768E4002A3FF427AED9
:104710000A2A3FF424AE7A4F069B796AFE693D6A05
:10472000BC69774898465F1C06EB010A0B3341468B
:10473000093104EB050B0F934546434690F808906A
:104740000C910A35591D4046083003970D95DF1D21
:104750009D1D0691203A109904900B97181DDF1C9F
:104760000A95C8469D1C9946D3B201316B2B08901F
:1047700007970595189100F24281624850F823701E
:104780003978109A189B029700208CE0CD0711D53C
:10479000039DA542C0F29F81A14580F2E3815D4562
:1047A00008DAB34206DB534504DA574F07EBC31C64
:1047B0000CF805808D0713D5079D059FAC4200F3CB
:1047C0007581BC4240F3C881079DAB4508DD9E4220
:1047D00006DC9A4504DD4C4F07EBC31C0CF8058042
:1047E0004F0713D5069D089FAC4200F30B81BC42D6
:1047F00040F3BB81069DAB4508DD9E4206DC9A4531
:1048000004DD414F07EBC31C0CF805800D0713D5E1
:104810000B9D0A9FA542C0F20A81BC4240F3A981C8
:104820000B9D5D4508DA9E4206DC9A4504DD364F55
:1048300007EBC31C0CF80580CF0613D50C9D049F15
:10484000AC4200F30981BC4240F397810C9DAB451B
:1048500008DD9E4206DC9A4504DD2B4F07EBC31CA6
:104860000CF805808D0613D50F990D9DA142C0F25D
:104870000881AC4240F36D810F9F5F4508DA9E428C
:1048800006DC9A4504DD204901EBC31505F80780D5
:104890000130082802F1020203F102037DD0029FD9
:1048A00017F8011F029796423FF770AF924513DC4D
:1048B000CF077FF57FAF039DA542C0F22A81A145B6
:1048C00080F24D815D45BFF675AF9E423FF772AFF6
:1048D0009A457FF76FAF68E70B4DDDF80CC0CDF858
:1048E000509005EBC217084D129705EBC3151395B1
:1048F000CE460027029D159222E000BFF0B30100D2
:1049000010CEFF1F5CFF01000831FF1FDE4502DAF9
:10491000129A02F80E8064451BDDDE4509DA9E42DC
:1049200004DC9A45C4BF139A02F80E80644540F334
:10493000EC800137062F0CF1020C0EF1020E21D093
:1049400041FA07F919F0010FF3D0A645DEDA644504
:10495000EFDCE34540F3D380129AA64502F80C80C1
:1049600080F2D0809E42E4DC9A45C8BF139A07F1DA
:104970000107C8BF02F80C80062F0CF1020C0EF1E3
:10498000020EDDD1159ADDF850900295013008280D
:1049900002F1020203F1020381D1099810F8012FFC
:1049A000099009F10C09002A3FF4D9AC039B0F9937
:1049B0000D9D0C9F04980C3303930B9B0C310C350D
:1049C0000C370C300C330F910D950A99069D0C97FE
:1049D0000490089F07980B93059B0C310C350C37FE
:1049E0000C300C330A2A0A91069508970790059314
:1049F0003FF4B5AC203AD3B26B2B7FF6BEAE614F1D
:104A00000021BEE6BC423FF701AFBB457FF7FEAEDB
:104A10009E4207DC9A4505DD5B4D089F05EBC31CF4
:104A20000CF80780069DAC423FF7F0AEE2E6BC42D0
:104A30003FF702AFBB457FF7FFAE9E4207DC9A45CA
:104A400005DD514D0A9F05EBC31C0CF807800B9D3B
:104A5000A542FFF6F1AEE3E6BC423FF703AFBB452C
:104A60007FF700AF9E4207DC9A4505DD464D049F67
:104A700005EBC31C0CF807800C9DAC423FF7F2AE6F
:104A8000E4E6AC423FF704AFAB457FF701AF9E428F
:104A900007DC9A4505DD3C4F0D9907EBC31C0CF86C
:104AA00001800F9DA542FFF6F3AEE5E6BC423FF75D
:104AB00097AEBB457FF794AE9E4207DC9A4505DD75
:104AC000314D059F05EBC31C0CF80780079DAC42D8
:104AD0003FF786AE78E6A145FFF66CAED945BFF646
:104AE00069AE9E4206DC9A4504DD274F07EBC31CE6
:104AF0000CF80980039DA542FFF65CAE4FE6A64583
:104B0000FFF617AFDE45FFF60AAFE3453FF72AAFE2
:104B10000FE7A145FFF64EAED945BFF64BAE9E421C
:104B200006DC9A4504DD184D05EBC31707F809802C
:104B3000039DA542FFF63EAEC4E6169B1199CEEB4F
:104B400003070F440697FFF749BA17974FF0000E77
:104B5000CEE5AB459BDC8FE6BB45ADDC34E6D94505
:104B6000DDDBAFE6D945BCDB19E6BB453FF750AF0F
:104B700040E6BB453FF761AF52E6BB453FF772AF3A
:104B800064E600BFF0B301000831FF1F0FB410B599
:104B900082B004AB074C53F8042B0193402120460C
:104BA0000EF076FA2046FFF75BF902B0BDE8104040
:104BB00004B07047C430FF1F2DE9F04F8BB001F5F2
:104BC0004C700591059B0290D3F8AC0FA74ADFF813
:104BD000BC82A74DA74E039289460024A6490491A2
:104BE000431C4FF02607019400F03D81019A90424A
:104BF00014BF7724FF2411469C4899F8243050F8BC
:104C000031200399C8F800204968C8F80410022030
:104C1000C8F80C000199984888F808400122C8F8A3
:104C20002C2099F825B050F831A03BB99348944B0B
:104C3000BBF1000F08BF1846FFF712F95246DDF826
:104C400008C007F1230A02F1300B5CF8047F07F576
:104C50000040C0EB00114F0086FB070EBE44FB175F
:104C6000C3EBEE300230C0EB0A03991E5F1E581CE6
:104C700005EBC11E991C05EBC71705EBC01005EB32
:104C8000C31305EBC1110EF80240BC549C5484546C
:104C90008C5401329345D8D17A4A019F0FCA0DF145
:104CA000180A8AE80F0099F827005AF82770042894
:104CB00000F2C382DFE810F04D02DC016701F6006C
:104CC0000500714BEA190021186818B102F51B5C48
:104CD0008CF82F40586818B102F51B5E8EF83040F2
:104CE000986818B102F51B5A8AF83140D86818B193
:104CF00002F51B5B8BF83240186918B102F51B5C9A
:104D00008CF83340586918B102F51B5E8EF83440B8
:104D1000986918B102F51B5A8AF83540D86918B15C
:104D200002F51B5B8BF83640186A18B102F51B5C64
:104D30008CF83740586A18B102F51B5E8EF838407F
:104D4000986A18B102F51B5A8AF83940D86A18B126
:104D500002F51B5B8BF83A40186B18B102F51B5C2F
:104D60008CF83B40586B18B102F51B5E8EF83C4046
:104D7000986B18B102F51B5A8AF83D40D86B18B1F0
:104D800002F51B5B8BF83E40186C18B102F51B5CFA
:104D90008CF83F400131072903F1440302F18002FE
:104DA00092D1019B059A88F8084003EB8301022405
:104DB000C8F8007002EB810E0127C8F80C40C8F853
:104DC0002C70BEF82400314CB0F5807F0BD0D9F8A0
:104DD00028202F492F4B30485927002AC8BF194691
:104DE0006760FFF7D3FE6322D9F82C102B48C8F870
:104DF0000420284C2A4FFFF7C9FED9F83020244957
:104E00002548002AC8BF21466E23C8F80430FFF7A2
:104E1000BDFE019AD9F834102048013207EB810A0F
:104E200014460192029ADAED007A049F02F572723A
:104E3000BDEEE70A0292039A7823083210EE101AA8
:104E4000083704970392C8F80430FFF79FFE042C3C
:104E500009F1140900F0EE81059B7F68D3F8AC0FCF
:104E6000431C7FF4C3AEAA240199C5E6DC6E0100A1
:104E70000831FF1F01800080FC6E010090BC010022
:104E80008CBC0100386F01001472010010CEFF1FAE
:104E9000C4BC010094BC0100C8BC0100D0BC01002E
:104EA0005CBF0100704BEA190021186818B102F5C7
:104EB0001B5E8EF82F40586818B102F51B5A8AF80D
:104EC0003040986818B102F51B5B8BF83140D86808
:104ED00018B102F51B5C8CF83240186918B102F564
:104EE0001B5E8EF83340586918B102F51B5A8AF8D8
:104EF0003440986918B102F51B5B8BF83540D869CE
:104F000018B102F51B5C8CF83640186A18B102F52E
:104F10001B5E8EF83740586A18B102F51B5A8AF8A2
:104F20003840986A18B102F51B5B8BF83940D86A93
:104F300018B102F51B5C8CF83A40186B18B102F5F9
:104F40001B5E8EF83B40586B18B102F51B5A8AF86D
:104F50003C40986B18B102F51B5B8BF83D40D86B59
:104F600018B102F51B5C8CF83E40186C18B102F5C4
:104F70001B5E8EF83F400131072903F1440302F123
:104F8000800292D10DE7394BEA190021186818B157
:104F900002F51B5A8AF82F40586818B102F51B5BBE
:104FA0008BF83040986818B102F51B5C8CF83140E2
:104FB000D86818B102F51B5E8EF83240186918B136
:104FC00002F51B5A8AF83340586918B102F51B5B89
:104FD0008BF83440986918B102F51B5C8CF83540A9
:104FE000D86918B102F51B5E8EF83640186A18B100
:104FF00002F51B5A8AF83740586A18B102F51B5B54
:105000008BF83840986A18B102F51B5C8CF839406F
:10501000D86A18B102F51B5E8EF83A40186B18B1C9
:1050200002F51B5A8AF83B40586B18B102F51B5B1E
:105030008BF83C40986B18B102F51B5C8CF83D4036
:10504000D86B18B102F51B5E8EF83E40186C18B193
:1050500002F51B5A8AF83F400131072903F1440346
:1050600002F1800292D19CE664BA01007401020050
:10507000754BEA190021186818B102F51B5B8BF813
:105080002F40586818B102F51B5C8CF830409868C6
:1050900018B102F51B5E8EF83140D86818B102F5E0
:1050A0001B5A8AF83240186918B102F51B5B8BF85D
:1050B0003340586918B102F51B5C8CF8344098698C
:1050C00018B102F51B5E8EF83540D86918B102F5AB
:1050D0001B5A8AF83640186A18B102F51B5B8BF828
:1050E0003740586A18B102F51B5C8CF83840986A52
:1050F00018B102F51B5E8EF83940D86A18B102F576
:105100001B5A8AF83A40186B18B102F51B5B8BF8F2
:105110003B40586B18B102F51B5C8CF83C40986B17
:1051200018B102F51B5E8EF83D40D86B18B102F540
:105130001B5A8AF83E40186C18B102F51B5B8BF8BD
:105140003F400131072903F1440302F1800292D16B
:1051500027E63E4BEA190021186818B102F51B5CDE
:105160008CF82F40586818B102F51B5E8EF830405D
:10517000986818B102F51B5A8AF83140D86818B1FE
:1051800002F51B5B8BF83240186918B102F51B5C05
:105190008CF83340586918B102F51B5E8EF8344024
:1051A000986918B102F51B5A8AF83540D86918B1C8
:1051B00002F51B5B8BF83640186A18B102F51B5CD0
:1051C0008CF83740586A18B102F51B5E8EF83840EB
:1051D000986A18B102F51B5A8AF83940D86A18B192
:1051E00002F51B5B8BF83A40186B18B102F51B5C9B
:1051F0008CF83B40586B18B102F51B5E8EF83C40B2
:10520000986B18B102F51B5A8AF83D40D86B18B15B
:1052100002F51B5B8BF83E40186C18B102F51B5C65
:105220008CF83F400131072903F1440302F1800269
:1052300092D1B6E50BB0BDE8F08FA722044905482E
:10524000FCF71AFBADE500BF48B70100387001005C
:105250000C01020098BC01002DE9F04F8DB001F562
:105260004C700023079188469B4A9C499C4E9D4D5B
:10527000059026270691049203937724B9469C460D
:105280009548049950F83C204868706098F824309C
:1052900092483260022101223472F160F26298F881
:1052A00025B050F83C703BB98F48904BBBF1000FD4
:1052B00008BF1846FEF7D4FDDFF850B2DDF814C081
:1052C0003A4609F1230907F1300A5CF8041F01F599
:1052D0000040C0EB001779008BFB010E8E44CB170A
:1052E000C3EBEE300230C0EB0903991E5F1E581C61
:1052F00005EBC11E991C05EBC71705EBC01005EBAC
:10530000C31305EBC1110EF80240BC549C548454E5
:105310008C5401329245D8D1754A039F0FCA0DF1C2
:10532000200B8BE80F0098F827005BF82770042803
:1053300000F21B83DFE810F04302D2015D01EC00B4
:1053400005006C4BEA190021186818B102F51B5AC8
:105350008AF82F40586818B102F51B5C8CF8304071
:10536000986818B102F51B5E8EF83140D86818B104
:1053700002F51B5B8BF83240186918B102F51B5916
:1053800089F83340586918B102F51B5A8AF834403D
:10539000986918B102F51B5C8CF83540D86918B1D2
:1053A00002F51B5E8EF83640186A18B102F51B5BD9
:1053B0008BF83740586A18B102F51B5989F8384004
:1053C000986A18B102F51B5A8AF83940D86A18B1A0
:1053D00002F51B5C8CF83A40186B18B102F51B5EA5
:1053E0008EF83B40586B18B102F51B5B8BF83C40C4
:1053F000986B18B102F51B5989F83D40D86B18B16C
:1054000002F51B5A8AF83E40186C18B102F51B5C75
:105410008CF83F400131072903F1440302F1800277
:1054200092D1039B079A376003EB830102EB810A59
:10543000022001273472F060F762BAF824C0BCF58C
:10544000807F0CD02C4BD8F828202C49244F2C4896
:10545000002AC8BF194659237B60FFF797FB6322D8
:10546000D8F82C1027487260FFF790FBD8F830204E
:10547000214B22492248002AC8BF19466E2777606F
:10548000FFF784FBD8F834101F4A039B1D48144FC4
:1054900002EB810B069ADBED007A08320692049A41
:1054A0000832BDEEE70A0492059A0133039302F530
:1054B0007279782310EE101ACDF814907360FFF70C
:1054C00065FB0398042808F1140800F0E9810699A7
:1054D0008446D1F80490D3E6DC6E0100FC6E010036
:1054E00010CEFF1F0831FF1F90BC01008CBC0100D3
:1054F000386F01001472010094BC0100C4BC0100AB
:10550000C8BC0100D0BC01005CBF0100018000806C
:10551000704BEA190021186818B102F51B5E8EF86D
:105520002F40586818B102F51B5B8BF83040986823
:1055300018B102F51B5989F83140D86818B102F545
:105540001B5A8AF83240186918B102F51B5C8CF8B6
:105550003340586918B102F51B5E8EF834409869E3
:1055600018B102F51B5B8BF83540D86918B102F50C
:105570001B5989F83640186A18B102F51B5A8AF887
:105580003740586A18B102F51B5C8CF83840986AAD
:1055900018B102F51B5E8EF83940D86A18B102F5D1
:1055A0001B5B8BF83A40186B18B102F51B5989F850
:1055B0003B40586B18B102F51B5A8AF83C40986B77
:1055C00018B102F51B5C8CF83D40D86B18B102F5A0
:1055D0001B5E8EF83E40186C18B102F51B5B8BF811
:1055E0003F400131072903F1440302F1800292D1C7
:1055F00017E7394BEA190021186818B102F51B5951
:1056000089F82F40586818B102F51B5A8AF83040C3
:10561000986818B102F51B5C8CF83140D86818B155
:1056200002F51B5E8EF83240186918B102F51B5B5B
:105630008BF83340586918B102F51B5989F834408A
:10564000986918B102F51B5A8AF83540D86918B123
:1056500002F51B5C8CF83640186A18B102F51B5E27
:105660008EF83740586A18B102F51B5B8BF838404A
:10567000986A18B102F51B5989F83940D86A18B1EF
:1056800002F51B5A8AF83A40186B18B102F51B5CF8
:105690008CF83B40586B18B102F51B5E8EF83C400D
:1056A000986B18B102F51B5B8BF83D40D86B18B1B5
:1056B00002F51B5989F83E40186C18B102F51B5AC7
:1056C0008AF83F400131072903F1440302F18002C7
:1056D00092D1A6E664BA010074010200A64BEA1951
:1056E0000021186818B102F51B5C8CF82F4058682F
:1056F00018B102F51B5E8EF83040986818B102F5BB
:105700001B5B8BF83140D86818B102F51B5989F83A
:105710003240186918B102F51B5A8AF833405869AB
:1057200018B102F51B5C8CF83440986918B102F589
:105730001B5E8EF83540D86918B102F51B5B8BF8FB
:105740003640186A18B102F51B5989F83740586A73
:1057500018B102F51B5A8AF83840986A18B102F558
:105760001B5C8CF83940D86A18B102F51B5E8EF8C4
:105770003A40186B18B102F51B5B8BF83B40586B35
:1057800018B102F51B5989F83C40986B18B102F525
:105790001B5A8AF83D40D86B18B102F51B5C8CF897
:1057A0003E40186C18B102F51B5E8EF83F40013187
:1057B000072903F1440302F1800292D131E66F4BD5
:1057C000EA190021186818B102F51B5B8BF82F400D
:1057D000586818B102F51B5989F83040986818B11B
:1057E00002F51B5A8AF83140D86818B102F51B5CE3
:1057F0008CF83240186918B102F51B5E8EF8334000
:10580000586918B102F51B5B8BF83440986918B1E0
:1058100002F51B5989F83540D86918B102F51B5AB1
:105820008AF83640186A18B102F51B5C8CF83740CC
:10583000586A18B102F51B5E8EF83840986A18B1A4
:1058400002F51B5B8BF83940D86A18B102F51B5979
:1058500089F83A40186B18B102F51B5A8AF83B4098
:10586000586B18B102F51B5C8CF83C40986B18B172
:1058700002F51B5E8EF83D40D86B18B102F51B5B3C
:105880008BF83E40186C18B102F51B5989F83F405F
:105890000131072903F1440302F1800292D1C0E5EE
:1058A000FF24002500951F2353220E21FD602E208A
:1058B0003C72FCF7B1FA2D22104620230D210094F2
:1058C000FCF7AAFA214628222D480DF093FA2D4B19
:1058D000A24603F5206783F8D4A683F854A783F87B
:1058E000D4A783F854A883F8D4A883F854A983F8DC
:1058F000D4A983F854AA83F8D4AA83F854AB03F547
:10590000A0639F424FF0FF04E5D1282221461E48A4
:105910001E4F0DF06FFA07991D48D1F89C2FD1F852
:10592000985F50F8222050F825101A480223F3629D
:1059300010252E2386E82800FFF728F91648079B34
:1059400002680892089D1549D3F8A00FC5EB05120F
:10595000A1FB02310123C1F34015F36220B3002DF6
:1059600000F08780274600241FE0A7220C490D483D
:10597000FBF782FF55E500BF48B701003870010012
:10598000B537FF1F0831FF1F3541FF1F10CEFF1F26
:105990008C22FF1FD4BC0100B4DE01201F85EB5117
:1059A0000C01020098BC010007463123492229213D
:1059B00037200097FCF730FA362210463223282190
:1059C0000094FCF729FA282319464A22362000942D
:1059D000FCF722FA4A221046322328210094FCF7D1
:1059E0001BFA322319464A2236200094FCF714FA97
:1059F00037222A233648347286E80C00FEF730FA44
:105A00000798D0F8A42F002A5FD0002D0BBF0025E7
:105A1000FF25FF2400240095432349223B21372002
:105A2000FCF7FAF936221046009444233A21FCF799
:105A3000F3F93A23194600944A223620FCF7ECF990
:105A40004A221046009444233A21FCF7E5F9442306
:105A5000194600944A223620FCF7DEF93A223C230C
:105A60001C48347286E80C00FEF7FAF90DB0BDE868
:105A7000F08F00953123492229213720FCF7CCF9FA
:105A800036221046009432232821FCF7C5F928233A
:105A9000194600944A223620FCF7BEF94A221046E5
:105AA000009432232821FCF7B7F9322319460094D9
:105AB0004A223620FCF7B0F937222A2304483C72E8
:105AC00087E80C00FEF7CCF9A5E71546FF24A2E70E
:105AD000DCBC0100E0BC01002DE9F043A44EA54C64
:105AE0000D460FCE91B008AF0FC796E80F00802685
:105AF00087E80F000023E36023614FF0010832467E
:105B0000FF219D48A36223756375A361E36123723E
:105B100095F8B07FC4F82C80C4F8008026626662D5
:105B20000DF068F93246FF2194480DF063F93246D2
:105B3000FF2193480DF05EF93246FF2191480DF0A8
:105B400059F93246FF2190480DF054F93246FF21B1
:105B50008E480DF04FF93246FF218D480DF04AF97D
:105B60003246FF218B480DF045F93246FF218A4825
:105B70000DF040F989498A48C4F80480FFF706F817
:105B8000FF20207295ED010A6846FBF747FD0B21C7
:105B90006160F7B1834A84486946FEF7F7FF6846BB
:105BA00095ED050AFBF73AFD14224745626040F087
:105BB000AB807E4A7E486946FEF7E8FF684695ED71
:105BC000060AFBF72BFD1D21764A6160794869467C
:105BD0001AE0764A74486946FEF7D8FF95ED050A43
:105BE0006846FBF71BFD14266E4A714866606946DD
:105BF000FEF7CCFF684695ED060AFBF70FFD1D2367
:105C0000684A6C4863606946FEF7C0FFE868262270
:105C1000626000284CD06849032F4AD1634A674824
:105C2000544EFEF7B3FFE9692F236360002940F06B
:105C3000088163495B4A6348FEF7A8FF286A382257
:105C40006260002852D1052F5D4952D05E48554A06
:105C5000FEF79CFF2E6841206060002E00F0CF8090
:105C6000062F5A4900F0CF8059484E4AFEF78EFF62
:105C7000A8686F260528666061D9072F554963D04B
:105C8000484A5548FEF782FF2D69484B454A0DF1B9
:105C9000400808EB85097820606059F8201C4F48BF
:105CA000082F08BF1A46FEF771FF11B0BDE8F08358
:105CB0004B493C4A4148424EDFF81081FEF766FFEF
:105CC000E9692F2300290CBF31464146042F636048
:105CD000B0D1364A3B48DFF89C90FEF757FF296A5F
:105CE0003823636000297FD13146AFE7052F37495C
:105CF000ACD12E4A34481F4EFEF748FF2968412395
:105D0000636091B92E49AFE7264A29486946FEF7F4
:105D10003DFF684695ED060AFBF780FC1D26022F25
:105D2000666040F09D80214A50E71E4A2848274976
:105D3000FEF72CFFA8686F22052872606DD82949EC
:105D4000072F51F820109BD1184A2348FEF71EFF59
:105D50002F69144A21480DF1400C0CEB8706782579
:105D600056F8201C6560FEF711FF11B0BDE8F08306
:105D7000486F010010CEFF1F0831FF1F8831FF1F41
:105D80000832FF1F8832FF1F0833FF1F8833FF1FB1
:105D90000834FF1F8834FF1F0835FF1F08BD0100AE
:105DA00010BD0100C4BC01001CBD010004BD010008
:105DB0002CBD01003CBD0100ECBC01004CBD01004C
:105DC000F8BC010060BD010074BD0100F4BC01001D
:105DD00088BD0100FCBC01009CBD0100B0BD0100FC
:105DE000E4BC010090030200244A25484146FEF726
:105DF000CDFE29684122C9F8042000292ED1062FA2
:105E000020497FF431AF2048204A214EFEF7BEFEE4
:105E1000A8686F230528636091D9184A1D491E4858
:105E2000FEF7B4FE2C69154A1C4810AD05EB840C36
:105E300078275CF8201C7760FEF7A8FE11B0BDE85B
:105E4000F0830E4A16481749FEF7A0FE286A38224A
:105E5000726000283FF4F7AE1249F7E6414603E7C7
:105E60001148064A6946FEF791FEEB6826206060FD
:105E7000002B7FF4D0AE0D49CEE600BFC4BC0100BC
:105E800074BD0100F8BC010088BD010004BD010023
:105E900010CEFF1FFCBC01009CBD0100B0BD010085
:105EA00060BD0100F4BC01003CBD0100E4BC010088
:105EB0002DE9F043C3B001AC804625460DF582794B
:105EC0002B462A1B03F8012BEF1C2E1D681DA91D54
:105ED000EA1D03F1010EC4EB0E0EC4EB030C3F1BD5
:105EE000361B001B091B121B85F801C083F801E05B
:105EF000083505F8057C05F8046C05F8030C05F871
:105F0000021C05F8012C4D45DAD10DF105077B1B6C
:105F1000FF20DE4384F800010CF0C8FF06F00309FF
:105F20002E462D1B16F8013D90FBF5F101FB150CDB
:105F3000BE4214F80C20327004F80C3071D0B9F164
:105F4000000F2FD0B9F1010F1CD0B9F1020F0BD007
:105F50000CF0ACFF351B90FBF5F101FB150016F8BA
:105F6000013D225C327023540CF0A0FF351B90FBE6
:105F7000F5F101FB150916F8010D14F8093033701D
:105F800004F809000CF092FF351B16F8012D90FB68
:105F9000F5FC0CFB1509BE4214F80910317004F829
:105FA00009203ED00CF082FF331B90FBF3F505FB7C
:105FB000130016F8011C14F800C006F801CC215497
:105FC0000CF074FF721E131B90FBF3F505FB130915
:105FD00016F8020C14F8091006F8021C04F809005F
:105FE0000CF064FFB21E151B90FBF5FC0CFB1509B1
:105FF00016F8033C14F8090006F8030C04F80930FD
:106000000CF054FFF11E0D1B16F8043D90FBF5F249
:1060100002FB150CBE4214F80C00307004F80C3072
:10602000C0D121464FF48072404609F0D7F821468E
:1060300008F580704FF4807209F0D0F843B0BDE8E5
:10604000F08300BF2DE9F041D0F850322DED048BE4
:1060500093F8445084B004461E460DB121F00F0160
:1060600007EE901ADFEDA86AB8EEE77ABEEE000AF6
:10607000A7EE260AB7EE008A70EE000AF4EEC80A10
:10608000F1EE10FA00F1FF8093F8431093ED021A3D
:1060900071B3D3ED061A9FED9D6A9FED9D5AD3ED26
:1060A000044ADFED9C5AB1EE042A61EE022A68EE42
:1060B000213A21EE063AF4EEC52A23EEA44AF1EE87
:1060C00010FAB4EE653A58BFF0EE452AF1EE10FA38
:1060D000B5EEC04A48BFB0EE653AF1EE10FACBBF5C
:1060E00072EEC12A31EE433AA4EE221AA4EE031A4C
:1060F00093F8420083ED031A002863D0F7EE007A8C
:1061000093ED059AD3ED049AB0EE677AA9EE087A7A
:10611000B6EE000A67EE000AF4EEE70AF1EE10FAB6
:1061200000F1DC80F0EE670AB7EE006A76EE698A6D
:10613000E9EEA08AC3ED088A002D49D193F8450005
:1061400086F84150E8B193ED072AD3ED032A9FED7D
:10615000723ADFED723A93ED044A9FED717AF0EEF8
:10616000009A68EE027AA2EEA93A67EEA36AA4EE5C
:10617000263AB4EEC73AF1EE10FA6AD482ED007A0C
:10618000012093F84620C2B104F27C4C9CED000A39
:10619000B5EEC00AF1EE10FA7FD46249D4F87074FB
:1061A0000B680393039DD4F87464EA1B0136C82A74
:1061B000C4F874642CD88CED008A04B0BDEC048B58
:1061C000BDE8F081F7EE008AC3ED088A002DB5D056
:1061D000DFF8608193ED049AD8F80070F90778EE43
:1061E000088A72D5504FF0EE001ABFEE005AA9EEA1
:1061F000215AF4EEC58AF1EE10FA34D5D7ED005AE3
:10620000B4EEE55AF1EE10FA2DD8C7ED008A95E705
:10621000D4F86C740968029106EB860807EB8703D3
:1062200009EE103A01EE908AF8EEC98AB8EEE15A0A
:10623000002204F58F65029EC5ED008A04F5906783
:10624000C4F86C2487ED005AC4F87064C4F8742450
:10625000B1E7B7EE007AB4EEC73AF1EE10FAC8BF74
:10626000B0EE437A8AE7F4EEC58AF1EE10FA06DD65
:10627000D7ED004AB4EEE45AF1EE10FAC5DAC7EDF4
:10628000008A00255AE7BFEE008AF4EEC80AF1EE54
:1062900010FAC8BFB0EE608AF6E6B5EEC08AF1EE3D
:1062A00010FA7FF77AAF70EE480A9FED201AB0EE31
:1062B000E06AB4EEC16AF1EE10FA7FF76EAFD4F87F
:1062C0006C640136C4F86C6467E74046019209F0DB
:1062D00065F8019A60B9D4F8503283E7F5EEC00A48
:1062E0009FED131AF1EE10FAD8BFF0EE410A1BE74A
:1062F0000D4F01924046C7ED008A09F055F8D4F8D9
:106300005032019A6FE700BF01088039CDCC4C3E76
:1063100000005C4500005C4100007A440000FA4542
:1063200000409C46B4DE0120C030FF1FCDCC4C3D68
:1063300000000000BC30FF1F2DE9F04182B002AB2D
:106340004FF4936604460D4606FB0100002143F816
:10635000041D00F57F560C36114630461A46FFF7ED
:1063600071FE012875D04FEA850808EB050204EBA1
:10637000820C671945F6ED409CF87B2017F800E089
:10638000964549D008EB050C04EB8C0E9EF878304E
:106390008BBB3949DFED397A032A4A6D14BF9FED73
:1063A000380A9FED380A04F56453002A03F13803D4
:1063B00018BFB0EE670A03EB0510FDF733FD08EBDD
:1063C000050004EB800C9CF87B0004284DD045F6BA
:1063D000ED464544B85504EB850445F6F54594F87B
:1063E0007A207A5545F6F14894F8783007F8083065
:1063F00002B0BDE8F08108EB050604EB860604F563
:10640000645396F87A20383303EB0510E2B9FBF7B2
:1064100069F896F87B00DAE745F6F5439CF87A10C0
:10642000F85C8842AED145F6F1419CF87830785C52
:106430009842ADD145F6EC4C616D14F80CE08E45F8
:10644000D6D0002BD7D1A4E7FBF76CF896F87B00E9
:10645000BDE704F56457383707EB05109DED010AD9
:10646000FDF7E0FC02B0BDE8F08106F28C4E064973
:10647000CEF80010ABE700BF1071FF1F00007A4597
:1064800000409C4600A00C463333733F2DE9F04F8B
:106490002DED088B604DDFED618A2B68604E9FED1E
:1064A000618A91B004460E930E98C4F80402C4EDBC
:1064B000808A8B460CF0F0FC2046FFF7F9FC286838
:1064C0000C90DDF830E02F680B97574BC4F80C3276
:1064D00004F5027004F58B6A04F25447002300228D
:1064E000C4F81462C4F850024FF07E564F48504929
:1064F000C4F818224FF086484FF00109C4F8402232
:10650000C4F8443284F8483284F8493284F84B3273
:1065100084F84C3284F84D3204F58F6CC4F83C8218
:1065200084F84A92C4F81C62C4F82062C4F8246259
:10653000C4F83462C4F83002C4F83802C4F808124F
:1065400004F27C483A6004F59169CAF8002004F22C
:106550008C46C4F868E404F2944A04F5906EC4F8DA
:106560005C34C4F8603484F86434C4F86C340B9937
:10657000C4F87014C4F874342046CCF80020C8F86D
:106580000020CEF8002084F88434C9F8002032605E
:1065900084F89034CAF8002008F0D6FB204608F0B2
:1065A000B3FB204608F0E6FB642008F0DDFD07EEB3
:1065B000900A2A680D92B8EE670A0D9860EE080AF4
:1065C000A0EEA88A10B92D680F950F98C4F80402A0
:1065D0000CF062FC2046FFF76BFCB5EEC08AF1EED2
:1065E00010FA04F51573D2BFD4ED802A84ED808AA9
:1065F000F0EE482A0393DFED0F9A9FED0FAA9A461B
:106600000026B1EE089AFAEE0EBAF2EE048AB5EE62
:1066100000BAF7EE00AA1DE0B4DE01200AD7A33CC1
:1066200000005C410AD7233C40D00020000080BF1E
:1066300010DC002000000000FFFF7F7F6666E63F61
:106640006666663F00FEFF4600F07F45000080461C
:10665000D4ED802A01EE106AF8EEC11A013621EE5F
:10666000A22A12EE100A0BF0BFFE8046894649ECC2
:10667000108B0BF0C5FC53EC102B10EE100A1946D2
:10668000CDE900230BF08CFFDDE90023C5B24946BC
:1066900040460BF049FD0BF0CBFF02EE900A605D27
:1066A000254400F0030195F801C003EE101A0CF028
:1066B0000308F8EEC33A08EE108AB0EE6B7AF0EEFB
:1066C0006A5AE3EE8B5A0207A2EE897AB8EEC80A3C
:1066D000F0EE6A0AE0EE0B0AB0EE686AF0EE654A88
:1066E00072EEEA7A62EEA26AA2EE876A4CBF65EEAB
:1066F000E24A62EEA44A5FEA0C734CBF60EEE77AAE
:1067000067EEA07A26EEA24A77EEE41A24EE065A45
:10671000E5EE214AF4EECA4AF1EE10FAF4EE694AC7
:10672000D8BFB0EE64AAF1EE10FAC8BFF0EE649ADA
:10673000802EEAEC014A8BD1039A5FED40BA92EDCC
:10674000009A5FED418A39EE4ABA79EECA9A6BEE49
:106750002BAA13468AEEA97ABE1A351FC5F381000B
:1067600077EE686AE3EC016A9F425ED048B3012885
:1067700019D002280BD093ED006A36EE4A3A63EE48
:106780002B3A83EEA94A74EE685AE3EC015AD3ED32
:10679000004A34EECA5A25EE2B8A88EE290A70EE9A
:1067A000687AE3EC017AD3ED000A30EECA1A61EEA2
:1067B0002B1A81EEA92A72EE682AE3EC012A9F4285
:1067C00033D093ED009A39EE4ABA9E466BEE2BAA6F
:1067D00010338AEEA97A77EE686AEEEC016A13ED5F
:1067E000036A36EE4A3A63EE2B3A83EEA94A74EE18
:1067F000685A43ED035ADEED014A34EECA5A25EEDB
:106800002B8A88EE290A70EE687ACEED017A53ED74
:10681000010A30EECA1A61EE2B1A81EEA92A72EE35
:10682000682A43ED012A9F42CBD103995FED7BBAE1
:106830000B46B3EC01AA6AEE2B8A7A1AFDEEE89AAF
:106840000020CDED009A161FBDF90050C4F85C047D
:106850009F42C4F86004C6F38201DA46CBF80050C8
:1068600000F0C980002962D0012952D0022944D009
:10687000032936D0042928D005291AD006290CD09E
:10688000B3EC019A29EE2BBADA46FDEECBAACDED98
:1068900000AABDF900204AF8042FB3EC017A67EE94
:1068A0002B6ABDEEE66A8DED006ABDF900604AF81C
:1068B000046FB3EC013A63EE2B3ABDEEE34A8DED83
:1068C000004ABDF900504AF8045FF3EC015A65EE46
:1068D000AB4ABDEEE45A8DED005ABDF900004AF80E
:1068E000040FB3EC018A28EE2B0AFDEEC07ACDED41
:1068F000007ABDF900104AF8041FF3EC010A20EEFB
:10690000AB1AFDEEC11ACDED001ABDF900204AF810
:10691000042FB3EC012A62EE2B2A9F42BDEEE2AABD
:106920008DED00AABDF900604AF8046F63D0994666
:10693000F9EC018AD3ED019A93ED03BAD3ED04AAE1
:1069400093ED056AD3ED066A93ED077A99ED019A06
:1069500028EEAB3A29EE2B4A69EEAB4A2BEE2B5AC6
:106960006AEEAB5A26EE2B8A26EEAB0A67EE2B7A3E
:10697000FDEEC33AFDEEC40ABDEEE41AFDEEC51A03
:10698000BDEEE52AFDEEC82ABDEEC0AAFDEEE78AFF
:10699000CDED003ACDED040A8DED031ACDED051ACB
:1069A0008DED062ACDED072A8DED08AACDED098AD9
:1069B0002033BDF91090BDF90080BDF90CC0BDF9C0
:1069C00014E0BDF91820BDF91C50BDF92000BDF937
:1069D0002410CAF80C909F42CAF80480CAF808C074
:1069E000CAF810E0CAF81420CAF81850CAF81C00F7
:1069F0004AF8201F9BD104F58A67D7ED00BA5FEDF6
:106A0000EE9A5FEDEEFA9FED1AFADFED1AEA9FEDCE
:106A10001AEADFED1ADA9FED1ADAB7EE009A3BEECA
:106A200089BAF6EE00AA2BEE296A204666EE2A6A9B
:106A30000122BCEEE67A00268DED007ABDF800401A
:106A4000CBF8806303EE104AB8EE434A0023CBF83C
:106A500084338BEDEF4A8BF8C0638BF898238BF867
:106A600099238BF8B92311B0BDEC088BBDE8F08FEA
:106A70007D21153EC728004433333346000034429D
:106A80000000403A2DE9F04F4B8C2DED068B00EEC7
:106A9000103A0F460546ADF2344D00F59870B8EE49
:106AA000400A1446FBF762F9B88C95ED587A95EDDB
:106AB000595AD5ED577AD5ED566A85ED6C0A06EE32
:106AC000100AF8EE460A77EEE65A30EEC71AA5EE3F
:106AD000017AB4EEE57AF1EE10FA85ED587A41F1DB
:106AE000758077EE267AC5ED577A95ED542AD5ED67
:106AF0005A2A95ED553A76EE823AF0EE424A37EE52
:106B0000E34AE4EE224AF4EEC34AF1EE10FAB0EEA4
:106B100064AA41F16A81B4EE642AF1EE10FA58BF1A
:106B2000B0EE42AA04F6E471DFEDF39A0A689FED35
:106B3000F39ADFEDF38A9FEDF38A85ED6BAAC5F832
:106B4000B421B84605F1B00BAA462E464FF0040911
:106B5000B8F810C00AEE90CA5846B8EE6A0AFBF7B9
:106B600005F9B8F818308AED6E0A06EE103A96ED7F
:106B7000080AD6ED096A96ED0A7AF8EE460AB7EEEB
:106B8000001A30EEC05A70EEE67AA5EE290AE7EE5A
:106B9000896A86ED080A70EE665AC6ED096AF0EE5B
:106BA000E51AF4EE471AF1EE10FAD8BFF0EE471AE4
:106BB00021EEA83AB4EEC13AF1EE10FA40F3F687AE
:106BC000DFEDD14ADFEDD13AB0EE413AB6EE004A00
:106BD00096ED0FAAD6ED0DAA96ED0B7A96ED0C0A5E
:106BE00086ED0A3A34EE8A6A70EEEA6A76EE230A95
:106BF000F0EE6A7AC6EE201AB7EE001AE1EEA67A37
:106C000037EE402A31EE615AF4EEC27A65EE065A4A
:106C1000F1EE10FAC6ED0E1AC6ED0F5AC6ED0D7A5A
:106C200007D577EE802A32EEC73A37EE037A86ED43
:106C30000B7A70EE074AF4EEE47AF1EE10FA07DD13
:106C400077EEC03A33EEC7AA37EE0A7A86ED0B7AB2
:106C5000F3EE0AAADFEDAE0A9FEDAE1A86ED0A4A00
:106C600037EE6A0ADFEDB16A20EE204A84EE016A4F
:106C700076EE261AF4EEE01AF1EE10FA40F17F8576
:106C8000F4EEE61AF1EE10FAD8BFF0EE661AB9F19A
:106C90000109C6ED101A08F10208EAEC011A0BF11D
:106CA000200B06F124067FF453AF04F6D47EDEED0C
:106CB000009A388C9FED9C9A08EE900A39EEA98ACA
:106CC000BFEE002AA8EE092A04F57D61B8EE685AE5
:106CD000D1ED005A65EE097AF7EE002A22EE273A46
:106CE000A5EE893AB4EEE23AF1EE10FA01F18180B4
:106CF000DFED894A94ED0CAAD5ED00AA9FED890A33
:106D0000666B864AC5ED7A4AB8EECA7AFDEEEA0AA3
:106D100027EE001AF8EEE06A40F65C7321EE264A90
:106D200003FB06F3BDEEC46A82FB0310C118DE1735
:106D300016EE10CAC6EBE12AD44440F65B7204F5A5
:106D4000856804F5FE6B04F6B83904F5786E944551
:106D5000C8ED004ACBED004AC9ED004ACEED004A2D
:106D600000F344876E482CEAEC7100EB810633682F
:106D7000C4F8FC33D5ED011AD4ED118ADFED699A20
:106D8000A06C664ABDEEE19AB8EEE88AB8EEC92A70
:106D900028EE295A40F65C7365EE025A03FB00F3B5
:106DA000FDEEE57A82FB0316F118D81717EE90CAAC
:106DB000C0EBE12AD44440F65B78C44500F3138766
:106DC000574A2CEAEC7B02EB8B09D9F80060E16DA5
:106DD000D4ED162A9FED533A504804F2C47EF8EEE3
:106DE000E23ACEF80060D5ED024ABDEEE4AA63EEC9
:106DF00083AAB8EECA0A40F65C732AEE807A03FBD7
:106E000001F3FDEEC70A80FB0316F118DA1710EE46
:106E100090CAC2EBE12AD44440F65B70844500F38B
:106E2000EB863F492CEAEC7801EB880BDBF800603D
:106E3000206F94ED1B1ADFED3B6A384A04F68C395B
:106E4000B8EEC16AC9F8006095ED034AFDEEC41AB8
:106E500066EE269AB8EEE19A40F65C7369EE898A8E
:106E600003FB00F3BDEEE88A82FB0316F118D81786
:106E700018EE10AAC0EBE12EF24440F65B7CE2452E
:106E800000F3B786264E2AEAEA7806EB880BDBF891
:106E9000002094ED0B5AB4F824909FED222AF8EECE
:106EA000C55A04F65473B9F5807F65EE822A1A60DC
:106EB00001F02B80398AD4ED0A3A9FED1B3A07EE98
:106EC000901AB8EEE3AAF8EE674A2AEE020A64EED8
:106ED00083AAF0EE620AEAEE800AB7EE007AF4EED8
:106EE000C70AF1EE10FA01F10580F0EE470A04F549
:106EF0008060C0ED000A1BE06666663F9A99993E85
:106F00000AD7A33B9A99D93FAE47813FD0CC4C3E9C
:106F100000F07F4500007E45295C0F3E810008801F
:106F2000F0730100B57E253C0108803900000000A7
:106F300094ED104A268F5FED056A97F82CA084F82F
:106F400035A4B8EEC46AB6F5807F66EE261A00F066
:106F500086877A8A94ED0F8A1FED0D9A09EE902AA2
:106F6000B8EEC82AF8EE698A62EE262A28EE895A17
:106F7000F0EE617AE5EE227AF7EE005AF4EEE57A69
:106F8000F1EE10FA00F16087F0EE657A04F5F96C25
:106F9000CCED007AD4ED153AB4F84CB05FED1F4A51
:106FA00097F82D3084F8FD37B8EEE3AABBF5807F63
:106FB0006AEE24AA00F04287B98A94ED141A1FEDF4
:106FC000267A00EE101AF8EEC16AF8EE400A26EEB4
:106FD000A46A20EE874AF0EE6A9AE4EE069AF7EE8B
:106FE000001AF4EEE19AF1EE10FA00F11C87F0EECF
:106FF000619A04F53969C9ED009A94ED1A8AB4F8DA
:1070000060605FED388A97F82EE084F8C5EBB8EE43
:10701000C82AB6F5807F62EE287A1AD0FA8A94EDF3
:10702000193A5FED3F2A05EE102AF8EEC34AF8EE52
:10703000455A24EEA8AA65EEA23AF7EE00AAE3EEBE
:107040008A7AF4EEEA7AF1EE10FA00F1DD86F0EEDB
:107050006A7A04F6587ACAED007A95ED6B7A5FED9C
:107060004E0A97F82F7084F88D7F04F6D87C27EEAF
:10707000201ADCED006AA6EEA01AF7EE007AB4EE54
:10708000E71AF1EE10FA00F162875FED589A0826D0
:107090000723B1EE0C7A3421EA4F9FEDEB5ADFF86B
:1070A000BCB3EA489FEDEAAA01FB03F201FB06F13B
:1070B000BB187E18BA587958D3ED024A96ED021AD9
:1070C000D3ED015A93ED036A96ED013AD6ED031A1A
:1070D00002EE901A02EE102AF8EEE43AF8EEC20A36
:1070E000B8EEC14AF8EEE26AF8EEE5AAB8EEC30AD5
:1070F000B8EEC69A93ED043AF8EEE18A76EEE02A0D
:1071000074EE635AD6ED046A93ED054AD6ED051A7E
:1071100030EE6A8A38EEC92AB8EEC30AF8EEE64ABB
:10712000B8EEC46AF8EEE18AE2EEA90A04F6F47158
:1071300034EEC01A78EEC62AA1EE290AA2EEA96A98
:10714000E5EEA93A96ED063AD3ED065A93ED071A05
:10715000D6ED071AA2EE299AF8EEC36AB8EEE52A30
:10716000E8EE29AAF8EEE18AB0EE408AB0EE460ACF
:10717000B8EEC16A76EEC24A78EEC62AA9EEA42A13
:10718000A9EEA26AFDEEE00AB0EE424ABDEEC63AB2
:10719000BDEEC02AFDEEEAAABDEEC40AFDEEE33A5A
:1071A000BDEEC99ABDEEC88AF8EEE06AF8EEEA5A7A
:1071B000B8EEC91AF8EEC81ACBED01AACBED000A59
:1071C000F8EEE3AA66EE850ACBED023AF8EEC36A62
:1071D000F8EEC23A8BED039AB8EEC09A65EE854A96
:1071E0002AEE854A21EE056A61EE858A63EE852ADC
:1071F00069EE055A8BED048A26EE858AC0ED014AB8
:10720000C0ED000A80ED024A80ED036AC0ED048AF9
:107210008BED052AC0ED052A8BED060AC0ED065A56
:107220008BED073AD1ED00AA80ED078A93ED082A8D
:1072300093ED093AD3ED0A1AD3ED0C2AD3ED0B4A9C
:1072400096ED080A96ED0A1AD6ED090AD6ED0B5A04
:10725000D6ED0C6AE769B8EEC06AF8EEC38AB8EEFC
:10726000E09AF8EEE13AB8EEC18AB8EEE53AB8EE47
:10727000E21AB8EEC24AF8EEE44AF8EEE62A36EE32
:10728000442A39EE680A38EE636A73EE641A72EEC5
:10729000C10AE9EE863AE9EEA14AA2EE294AE9EEF0
:1072A000808AA0EEA91A77EE6AAAFDEEE89ABDEEF2
:1072B000C44AFDEEE38ABDEEE49AFDEEC13AF0EE7B
:1072C000EA6AF4EECA6AF8EEC45AB8EEE98AB8EE91
:1072D000E8AAF8EEC94AB8EEE30A25EE856A28EE78
:1072E000052A2AEE053A64EE851A20EE055AF1EEDB
:1072F00010FA8BED084A80ED086ACBED099A80ED13
:10730000092ACBED0A8A80ED0A3A8BED0B9AC0ED83
:107310000B1ACBED0C3A80ED0C5ACCBF01230023A5
:10732000002F40F0308294F82420002A40F0F883A7
:1073300094F82500012805D094F827A0BAF104029A
:1073400018BF012204F2144CCCED007A94F80D849D
:1073500094F8380084F80E2443EA080684F80D6493
:10736000002840F0548494F83970012F00F07D8596
:1073700094F83B60B6F1040A18BF4FF0010A04F21A
:10738000DC7CCCED007A94F8D52794F84C7084F826
:10739000D6A743EA020884F8D587002F40F02F844F
:1073A00094F84D00012800F0A28594F84F60371F33
:1073B00018BF012704F6A43ECEED007A94F89D0B89
:1073C00094F8602084F89E7B43EA000684F89D6B65
:1073D000002A00F0E583276A002F00F01E8294F84F
:1073E0006300061F18BF012604F66C7ACAED007A06
:1073F00094F8652F84F8666F134384F8653F9FED1A
:10740000158A81ED007A002304F51C71DFED128AE4
:107410000B95019402930D4695F89C71002F00F096
:107420000081019E96F82400002840F01B840299F8
:10743000D5F88401F22202FB01F20BAB0DF5866157
:10744000AA460DE09C22FF1F0001003844DC012009
:1074500017B7D138ABAAAA4000FEFF4610DC0120C6
:10746000451C00F07F0705F07F0ED51904EB85055C
:1074700000F1020C071DC61C6D6F5D600CF07F09EA
:10748000964407F07F0C471D41F8045C06F07F0826
:10749000C51D04EB8E0607F07F0E871D07F07F07E2
:1074A00005F07F0591449044944496441744154454
:1074B00004EB890904EB880804EB8C0C04EB8E0EBA
:1074C00004EB870704EB8505766FD9F87490D8F83C
:1074D0007480DCF874C0DEF874E07F6F6D6F9E60BE
:1074E00041F8086CC3F80C9041F80C9CC3F810806C
:1074F00041F8108CC3F814C041F814CCC3F818E05C
:1075000041F818ECDF6141F81C7C43F8205F8BAE3A
:10751000B34200F1080041F8205DA1D15546C149B0
:107520002F46012600204FF000080BF061F8B0F55F
:10753000807F28BF4FF48070404540F2188400F1EE
:1075400080420CAB511E03EB880A0DF1300909EBA8
:10755000810CAAF1040101F1040ECAEB0C02F445FE
:10756000C2F382024B683ED01AB3012A1CD0022A11
:1075700017D0032A12D0042A0DD0052A08D0062AD3
:1075800018BF5EF8042F5EF8041F18BF9B180B4449
:107590005EF8042F13445EF8041F0B445EF8042FBA
:1075A00013445EF8041F0B445EF8042FF4451344A3
:1075B00019D0DEF80420DEF808101344DEF80C20A1
:1075C0001944DEF810301144DEF814201944DEF8B6
:1075D000183011440B44DEF81C205EF8201F1344C1
:1075E000F4450B44E5D10136312EC8EB000293FB84
:1075F000F2F147F8041F11D009EE106AF8EEC93A0B
:10760000804663EE88AA1AEE900A0AF0EDFE41EC7D
:10761000100B0AF0F5FC51EC100B86E7002085F802
:107620009C01029E019F01361437042E029605F537
:10763000727501977FF4F0AE04F592570B9D9FEDA4
:107640007AAADFED7A9A9FED7A9ADFED7A8A10377F
:1076500004F54C76B5EE008A96F8DD3053B196F815
:10766000DE20002A40F0EA80C022A6F1BC01301DD5
:107670000BF05CFB06F57276B742EDD194F82770FB
:1076800095F8DC01B8420BD0042800F09483042F55
:1076900000F088834FF0010C84F80DC485F8DC718C
:1076A00094F83B1095F8DD218A420AD0042A00F0B4
:1076B0008F83042900F08483012384F8D53785F86B
:1076C000DD1194F84F1095F8DE218A420AD0042A81
:1076D00000F00784042900F0FB83012384F89D3B1C
:1076E00085F8DE1194F8631095F8DF2191420DD0F2
:1076F000042A04BF95F8E32184F86120042900F0EE
:107700006C83012084F8650F85F8DF1195F8E4118A
:1077100094F824A0514505D04FF0010884F80C845A
:1077200084F80D8495F8E5B194F83890CB4505D0F0
:107730004FF0010C84F8D4C784F8D5C795F8E6213A
:1077400094F84C309A4204D0012684F89C6B84F85B
:107750009D6B94F8607095F8E701874204D0012191
:1077600084F8641F84F8651FD5F8B05104F57F6470
:1077700025600DF2344DBDEC068BBDE8F08FF0EEC8
:10778000601AFFF784BA226A002A40F0F28294F865
:107790002400012800F06D8394F82760042E00F087
:1077A000688304F21449C9ED007A94F80D0494F842
:1077B000386018434FF0010E012E84F80D0484F850
:1077C0000EE400F0668394F83B00042800F0278262
:1077D00004F2DC7CCCED007A94F8D56701221E43DC
:1077E00084F8D56784F8D62794F84C20012A00F055
:1077F000618394F84F60042E00F05C8304F6A43E8D
:10780000CEED007A94F89D2B4FF0010A1A4384F8CC
:107810009D2B84F89EAB94F86020012A7FF4DFADA5
:107820000026E1E500001440000000C700FEFF460E
:1078300000000034000100380AD7233CA6F1C00A3A
:10784000B1464FF000486FF0004E4FF0000C04EED0
:1078500010CAF8EEC44A0CF1010124EE880A05EEC4
:10786000901ABDEEC02AB8EEE56A12EE100A26EEB6
:10787000083A01300CF102035BF82020BDEEC35A38
:1078800006EE903A01EE902A12EE101A15EE102A2A
:10789000B8EEE61A5BF82100DAF80430511C61EE0C
:1078A000083A07EE900ABDEEE34A5BF821005BF868
:1078B0002210B8EEC27AF8EEE70A04EE900AF8EE6B
:1078C000E12A14EE100A70EE47AA05EE901A421C47
:1078D00032EEE00A5BF822105BF82020EAEE800A24
:1078E0000CF1030CF8EEE51AB8EEC52AF8EEE46ADE
:1078F00005EE101A07EE902A33EE423A36EEE11A00
:10790000F8EEC4AAF8EEE74ABDEEE07AE3EE011A1B
:10791000B8EEC50A17EE101A73EEEA3A70EE645A22
:107920001944BDEEE14AE3EEA54AC9F80410DAF8BD
:10793000083014EE102A8E451A44BDEEE46AA8BF42
:107940008E46C9F808208845B8BF88465AF80C0FFB
:1079500016EE101A96450144A8BF96469045B8BF4A
:1079600090468E45A8BF8E468845B8BF8846BCF174
:10797000300F49F80C1F7FF46AAF02EE10EA06EEF2
:10798000908AF8EEC21AB8EEE63AD6ED397A3AEEB7
:10799000611A39EEC35AF0EE612AE7EE812ACEEB86
:1079A000080A06F1C009A7EE853A3146FDEEE20A63
:1079B000FDEEC3AA10EE902A1AEE903A07EE10AA36
:1079C000981AB8EEC70A04EE900A70EE095AF8EE5B
:1079D000E43AB8EEE04A83EEA56A4B68CEEB0308C2
:1079E000081D02EE108AB8EEC23AF0EE446AE6EEE6
:1079F000036AFDEEE67A17EE90CA0CF30F024A60B6
:107A00004368CEEB030A05EE10AAF8EEC52AB0EEE5
:107A1000447AA6EE227AFDEEC7AA1AEE908A08F3FF
:107A20000F024260C868CEEB000300EE103AF8EE99
:107A3000C04AF0EE443AE6EE243ABDEEE32A12EEF6
:107A4000102A02F30F000B69C860CEEB030C03EEA3
:107A500010CAB8EEC31AF0EE446AE6EE016ABDEE53
:107A6000E65A15EE102A02F30F004B690861CEEBBF
:107A7000030A02EE90AAB8EEE27AF0EE440AE6EECD
:107A8000070ABDEEE00A10EE102A02F30F008B6920
:107A90004861CEEB030804EE908AF8EEE43AF0EE8B
:107AA000445AE6EE235ABDEEE53A13EE10CA0CF343
:107AB0000F02C8698A61CEEB000301EE103AF8EEBE
:107AC000C17AF0EE446AE6EE276AFDEEE62A12EE8F
:107AD00090AA0AF30F02CA6151F8200FCEEB0003FF
:107AE00007EE103AF8EEC70AF0EE44AAE6EE20AA36
:107AF000FDEEEA4A14EE908A08F30F0289450A6007
:107B00007FF46BAF61EEA81A24EE284A0021C6ED7F
:107B10003A1A86ED3C4A86ED386A86F8DD10A9E50A
:107B2000266A002E7FF408AC012A7FF405AC04F22B
:107B3000144ECEED007A94F80D7494F8380084F861
:107B40000E641F4384F80D7400283FF40CAC012828
:107B50007FF40EAC04F2DC79C9ED007A94F8D50715
:107B600094F84C7018434FF0000E84F8D50784F851
:107B7000D6E7002F3FF414AC012F7FF416AC04F6C7
:107B8000A439C9ED007A94F89D7B94F860201F43D6
:107B9000002084F89D7B84F89E0B002A7FF43DAE84
:107BA00094F86120012A7FF41AAC39E65FEDDE4AD1
:107BB000B7EE082AF6EE002AF0EE483AE3EE034A62
:107BC000E3EE423A23EE224AFFF702B877EEA61A16
:107BD000B4EEE17AF1EE10FAC4BF77EE667AC5ED45
:107BE000577AFEF782BFEE4EFFF7F1B8EC4BFFF786
:107BF000BFB8EB4AFFF74DB9E94EFFF719B9266A4E
:107C0000002E7FF4D2AB012F7FF4CFABB7E7226A0F
:107C1000002A7FF4ADAB01287FF4AAAB9AE70027D6
:107C200004F2DC7CCCED007A94F8D50784F8D677A2
:107C3000184384F8D507002A3FF4D6AD94F84F00D6
:107C4000042800F0768104F6A438C8ED007A94F890
:107C50009D2B4FF001091A4384F89D2B84F89E9BBD
:107C6000FFF7BDBB019ACF4992F826C0CE4B0DF16C
:107C70002C08BCF1000F08BF19460DF586698CAAC7
:107C80008E46BEEC011AD1ED012AD1ED039ADEED4C
:107C9000010A91ED049AD1ED053AD1ED06AA91EDD4
:107CA00007AA21EE284A22EEA80A60EEA84A69EE49
:107CB000A85A29EE286A63EEA86A2AEEA82AFDEEE1
:107CC000C41ABDEEC07A2AEE283ABDEEE45AFDEEA3
:107CD000E57ABDEEC61ACDED031A8DED047AFDEE00
:107CE000E62AFDEEC20ABDF90C60BDF910008DED6B
:107CF000055ACDED067A8DED071AFDEEC39AC8F848
:107D00000460BDF9147049F8046CBDF91830C8F866
:107D10000800CDED082A49F8080CCDED090ABDF997
:107D20001C00C8F80C70BDF9246049F80C7CCDED3E
:107D30000A9AC8F81030BDF9207049F8103CC8F80C
:107D4000140049F8140CBDF92830C8F8187049F827
:107D5000187CC8F81C6049F81C6C48F8203F49F8AA
:107D6000203D914501F120018AD1FFF7D8BB0023C6
:107D700039E494F82770042F00F0CD8004F2144EFB
:107D8000CEED007A94F80D744FF0010A1F4384F889
:107D90000D7484F80EA494F83B60042E3FF43FAFBA
:107DA00001273DE794F825B085F8E0B14FF00009D0
:107DB00084F825906EE495F8E03184F8253066E487
:107DC00094F8397085F8E171002084F8390073E483
:107DD00095F8E16184F839606BE494F8616085F8A6
:107DE000E361002784F861708BE4B0EE43AAFEF7EC
:107DF00099BEB5EEC03AF1EE10FA10DDDFED6B3A48
:107E000063EE234AFEF776BFF5EEC07A9FED680A6F
:107E1000F1EE10FAD8BFF0EE407AFFF71AB9DFEDB5
:107E2000644AFEF767BFF5EEC09A9FED619AF1EEE6
:107E300010FAD8BFF0EE499AFFF7DBB804F53960C5
:107E4000C0ED00AAFFF7D9B8F5EEC07A9FED583A19
:107E5000F1EE10FAD8BFF0EE437AFFF797B804F5C9
:107E6000F968C8ED001AFFF795B84FF0000AFFF760
:107E700086BA04F21448C8ED007A94F80D7494F8A8
:107E8000386084F80E241F43012E84F80D747FF4AB
:107E90009AAC04F2DC7ACAED007A94F8D5271A433A
:107EA00084F8D52794F84C200027012A84F8D67747
:107EB0007FF49FAC04F6A438C8ED007A94F89D7B5B
:107EC0004FF000091F4384F89D7B84F89E9BA2E439
:107ED00094F84D7085F8E271002084F84D00FFF7AA
:107EE000FCBB95F8E26184F84D60FFF7F3BB002717
:107EF000FFF760BAF5EEC00A9FED2D1AF1EE10FA09
:107F0000D8BFF0EE410AFEF7F2BF04F5806ECEED69
:107F1000002AFFF70DB804F21448C8ED007A94F86F
:107F20000D044FF00009184384F80D0484F80E94F2
:107F300031E704F6A43CCCED007A94F89D6B002761
:107F40001E4384F89D6B84F89E7BFFF748BA9FED33
:107F5000194AB4EEC41AF1EE10FA2FDDB1EE0C6A34
:107F600021EE067AB4EEE77AF1EE10FA0CDCFDEEC3
:107F7000C71AB8EEE19A11EE903A77EE497A5E1C94
:107F8000F0EE679AFFF787B8FDEEC78A18EE903AD1
:107F9000B8EEE88A5E1C77EE489AFFF77CB800BF1F
:107FA00000005C45980D0400980B0400295C0F3E0E
:107FB0000000000000000034000060355FED027A30
:107FC0000126B0EE677A0023DAE700BF0B8D00EEE2
:107FD000103A70B5B8EE400A0446006E0E461546DB
:107FE000F9F7C4FED4ED1C7A84ED1E0A70EE676AC0
:107FF000F5EEC06AF1EE10FA00F1258140F33D8103
:1080000094ED1A7A94ED1B5ADFEDB04A94ED196A9B
:1080100077EE670A77EE455AF4EEE40AF1EE10FACD
:1080200025EEA61AD8BFF0EE640AC1EE201A31EE92
:10803000852AB4EEC72AF1EE10FA08D5B4EEC62AA6
:10804000F1EE10FAD4BFB0EE467AB0EE427A728DFD
:1080500084ED1C0A02EE902A05F57D6084ED1B7A02
:10806000B8EE620A80ED007AE06FF9F77FFE94EDDA
:10807000233A84ED250A70EE433AF5EEC03AF1EE6C
:1080800010FA00F1D38040F3FF8094ED211A94EDB3
:10809000224ADFED8E6A94ED205A71EE437A71EE3A
:1080A000444AF4EEE67AF1EE10FA24EEA36AD8BF61
:1080B000F0EE667AC6EE270A70EE845AB4EEE51A40
:1080C000F1EE10FA08DDB4EEE55AF1EE10FA54BF05
:1080D000B0EE451AB0EE651A95F8E81FF68C84EDFF
:1080E000230A05F6D47C84ED221A00EE106A8CED8A
:1080F000001A002952D0D4F8B400B8EE400AF9F7BB
:1081000035FED4ED311A84ED330A30EE612AB5EE36
:10811000C02AF1EE10FA00F1A38040F3BC8094ED88
:108120002F7AD4ED302A9FED693AD4ED2E3A37EE0E
:10813000614A77EE626AB4EEC34AF1EE10FA26EEB7
:10814000825AD8BFB0EE434AC5EE047A77EEA24A0F
:10815000B4EEE47AF1EE10FA08DDF4EEE43AF1EE72
:1081600010FA54BFB0EE637AB0EE647A05F6EC7E96
:1081700084ED307A84ED310A05F6E4738EED007AF1
:10818000D4F8CC201A6005F6DC7EA66FCEF800602D
:1081900005F57E65D4F894402C6070BDD4F8980045
:1081A000B8EE400AF9F7E2FDD4ED2A0A84ED2C0A74
:1081B00030EE601AB5EEC01AF1EE10FA72D47EDD20
:1081C000D4ED286AD4ED291A9FED402A94ED276A50
:1081D00076EEE02A76EEE15AF4EEC22AF1EE10FADB
:1081E00025EE813AD8BFF0EE422AC3EE223A33EEB2
:1081F000A14AF4EEC46AF1EE10FA08DDB4EEC46AE6
:10820000F1EE10FA54BFF0EE466AF0EE446A05F65D
:10821000D870C4ED296A84ED2A0A05F6E47CC0ED25
:10822000006AD4F8B010CCF80010ACE794ED205AF6
:1082300094ED224ADFED256A94ED211A73EE457A1A
:1082400074EE454A2DE794ED196A94ED1B5ADFED63
:108250001F4A94ED1A7A77EEC60A75EE465ADBE6A7
:10826000D4ED2E3AD4ED302A9FED183A94ED2F7AC2
:1082700031EEE34A72EEE36A5DE794ED196A94ED3C
:108280001A7A94ED1B2AD4E694ED205A94ED211A23
:10829000D4ED225A12E7D4ED2E3A94ED2F7AD4ED94
:1082A000304A55E794ED276AD4ED291A9FED072A45
:1082B000D4ED286A70EEC62A71EEC65A8CE794EDAA
:1082C000276AD4ED286A94ED294A92E7BD378635AE
:1082D0004FF47A72704B02FB01F19942F0B400F254
:1082E000AF806E4CA14200F2AF806D4DA94200F20A
:1082F000AD806C4EB14200F2AE806B4FB94200F2DD
:10830000AE806A4B994200F2B080694CA14200F203
:10831000AE80684DA94200F28A804AF6A836B14282
:1083200088BF4FF4807200F28380634F4FF40046A1
:108330004FF48072B94280F08B8053005F4FB7FBDF
:10834000F3FC614580F089801344B7FBF3F5A94243
:1083500080F087801344B7FBF3F4A14280F0838060
:108360001344B7FBF3FC614580F083801344B7FBF3
:10837000F3F5A9427FD21344B7FBF3F4A1427CD2B8
:108380001344B7FBF3FC614579D21344B7FBF3F513
:10839000A94276D21344B7FBF3F7B94273D2134420
:1083A000464CB4FBF3FC61456FD21344B4FBF3F5C8
:1083B000A9426CD21344B4FBF3F7B9423ED2134442
:1083C000B4FBF3FC614564D21344B4FBF3F5A9425A
:1083D00029D21344B4FBF3F2914228BF102223D2D6
:1083E000F024374D3549374A4FF47A7707FB03F3CA
:1083F000B1FBF3F34360286820F008072F60296879
:1084000021F47F2C2CF47F6343F46020304320431D
:10841000286016683307FCD5294C256845F008020A
:108420002260F0BC70470F22511E0C01D9E7802258
:108430005308224CB4FBF2F71E027BE70D22F3E750
:108440001E4F0026012275E70222F1E70422EFE722
:1084500013460024C5E70822EAE70222E4E71022D7
:10846000E6E70322E0E70422DEE72022E0E74022FD
:10847000DEE70522D8E70622D6E70722D4E708225E
:10848000D2E70922D0E70A22CEE70B22CCE70C2262
:10849000CAE70E22C8E700BF4FA9AB00A7D455001A
:1084A00053EA2A002975150094BA0A00495D0500AF
:1084B000A4AE02005157010095BA0A000095BA0A0D
:1084C0002C100B4024100B402DE9F0410746884644
:1084D00007F0D4FC194C1A4E054604E007F0CEFC18
:1084E000431BB34226D82368DB07F7D4154A164846
:1084F000C2F80080076007F0C1FC144C104F06461C
:1085000004E007F0BBFC851BBD4213D82568104B67
:108510000E492B40002BF4D00E480A6802600A6016
:1085200006680B4C3440A4F10104B4FA84F77809CE
:10853000BDE8F0810020BDE8F08100BF24100B40B1
:1085400040420F0008100B400C100B4030100B4045
:1085500001000F00A0DE01202DE9F04F85B03F4F54
:1085600001900291039207F089FCDFF82CA13C4EA8
:10857000BB468146DAF800803A4D07F07FFC04469E
:1085800004E007F07BFC011BA94225D83368D9071A
:10859000F7D4354A3548C2F80080506007F06EFCC9
:1085A000304C054604E007F069FC401BA04213D89C
:1085B00039682F4B0B40002BF5D02E4CDBF8000018
:1085C0002060CBF800002268294B1340012B03D117
:1085D000294D2968CA050FD407F050FC214BC9EB7F
:1085E00000049C42C6D9019840F23312292105B0FB
:1085F000BDE8F04F06F0F4BC204D214F2B701A4817
:10860000039B2049029E002222603B601E4A1F4BB2
:1086100006600A601E481F49B863196007F02EFC07
:10862000104E074604E007F029FCC21BB2420BD8EB
:108630002B78002BF7D12468154D2540022D03D14E
:10864000012005B0BDE8F08F019840F23D122321D2
:1086500005B0BDE8F04F06F0C3BC00BF30100B40C2
:1086600024100B4040420F0008100B4000001A0D70
:1086700001000F00A0DE012010100B40A4DE01203D
:1086800000100B4004100B40400001000C100B4088
:1086900002007F1111003A06A8DE01202DE9F04FFB
:1086A00093B0804607F0EAFB784C794E054605E02A
:1086B00007F0E4FB421BB24200F2DC80236813F0B7
:1086C0000100F5D17349744A0860106007F0D6FBC9
:1086D000724C6F4D064605E007F0D0FB871BAF429A
:1086E00000F2C88020686E4B6C4F0340002BF3D023
:1086F000DFF8C0913968C9F800103960D9F8002056
:10870000674E1640012E40F0B580604EBB464FF0DC
:108710000A0A07F0B3FB5E4D044604E007F0AEFB27
:10872000021BAA4225D83068C007F7D459495A4DD0
:108730005C4B574C4FF4D5720A602B6007F09EFBE0
:10874000054604E007F09AFB401BA04211D83868A8
:10875000534A0240002AF5D0DBF80030C9F8003057
:10876000CBF80030D9F800104D4D0D40012D00F030
:108770005281BAF1010ACCD198F811104A4B002964
:1087800008BF4FF44013019307F078FB434F3F4C71
:10879000DFF800B10090BA4607F070FB3C4E05468A
:1087A00004E007F06BFB411BB14258D8206810F081
:1087B0000101F6D1384B3D4ACBF800101A6007F0A2
:1087C0005DFB334D064604E007F058FB801BA842D2
:1087D00045D83868324901400029F5D0DAF8002040
:1087E000C9F80020CAF80020D9F800602C4B3340AB
:1087F000012B34D107F042FB254E054604E007F07B
:108800003DFB431BB3422AD82068C107F7D4224B53
:10881000019A2749CBF80020196007F02FFB1C4D67
:10882000064604E007F02AFB821BAA4217D83868E4
:108830001B4901400029F5D0DAF80020C9F80020D2
:10884000CAF80020D9F80030154E1E40012E06D17E
:1088500007F014FB00990E4D401AA8422CD940464F
:1088600040F29112432106F0BBFB0446204613B0B0
:10887000BDE8F08F40464FF4BF72202106F0B0FBF8
:108880000446204613B0BDE8F08F00BF24100B4013
:1088900040420F0008100B400C100B4030100B40F2
:1088A00001000F0000001A080000304000001A37D5
:1088B00000000229A0DE0120A04B1A68002ABFF6A2
:1088C0006BAF9F4D196829601868420048BF9D48EA
:1088D0004FF0000148BF06709B48FFF7F5FD0028E8
:1088E00000F0B38000219948FFF7EEFD002800F06A
:1088F000A480924D964C2E689648370C3B0419463E
:108900002360FFF7E1FD002800F0A780DFF878A2E0
:10891000DFF878922B68904FDAF80010D9F8002031
:10892000386888F82C100E0A4FEA114C4FEA116E85
:1089300088F82B60110C160A4FEA102B88F82400D7
:1089400088F82820000C88F8303088F82AC0120EE9
:108950004FEA132C88F8276088F826100026190C97
:108960001B0E88F8220088F82E1088F829E088F875
:10897000252088F823B088F82FC088F82D3088F893
:10898000316021687548FFF79FFD002875D0296880
:10899000DAF80020D9F80030386888F821600D0C2A
:1089A0000F0A160A88F81E50150C88F8140088F86B
:1089B000201088F81C20090E88F8183088F81F70DD
:1089C000120E1F0A88F81B6088F81A501E0C050A40
:1089D0001B0E000C88F81D1088F8120088F819206A
:1089E00088F8177088F8166088F8153088F81350E2
:1089F00021685B48FFF768FDB8B321685948FFF765
:108A000063FD002841D1404640F2AB12402106F000
:108A1000E7FA044635E7494F3C68B4F5D57F04D101
:108A2000514E88F811500196AEE640464FF4C2729E
:108A3000252106F0D5FA044623E740464FF4CE72CE
:108A4000222106F0CDFA04461BE7404640F2991277
:108A5000212106F0C5FA044613E7404640F2A11270
:108A6000262106F0BDFA04460BE7404640F2A71265
:108A7000242106F0B5FA044603E740464FF4D272CB
:108A8000272106F0ADFA0446FBE602213748FFF73E
:108A90001BFD04460028B6D0354F36493A6822F00F
:108AA00006063E603B684FF0101543F00200386048
:108AB00002AA0D6040466FF07F41FFF74DFD18B1EF
:108AC0009DF81570BB0729D446F2A811DFF8C0B095
:108AD000DFF8C0A0DFF8C090274F284E284D0023B4
:108AE000CBF800304046CAF80030C9F800303B608F
:108AF00033602B60FFF7ECFB40F243404FF488619A
:108B00004FF0010CCBF80000CAF80000C9F80010C3
:108B100038603060286088F810C0B2E602AA1949AF
:108B20004046FFF719FD0028CED09DF8181001F03F
:108B30000F02012AC8D14CF25031C7E710100B4088
:108B400098DE012094DE01200000090200001A03D3
:108B5000A8DE0120000009091C100B400000090AD2
:108B600000001B0700001A370000304000001A0602
:108B700028100B4044100B400CD0044010D004408F
:108B800014D00440F1FFFF8014100B4018100B406C
:108B900000D0044004D0044008D004402DE9F04F38
:108BA00085B08DE80E003C4FDFF82C91DFF800A176
:108BB0003A4E0390BB46D9F80080394D07F05EF974
:108BC000044604E007F05AF9031BAB42F3D83368BC
:108BD000D907F7D4334A3448C2F80080506007F010
:108BE0004DF92F4C054604E007F048F9411BA1421E
:108BF000E1D839682D4B0B40002BF5D0DBF8000095
:108C0000CAF80000CBF80000DAF80020274D284908
:108C10001540012DCFD1274C2368DA05CBD5264F3F
:108C200026483D70264D00222E780A600199016089
:108C300036BB009C6202029B1A4D224E2A601C0425
:108C40002148224A2249234D44F4007333600560D1
:108C5000116007F013F9124C064604E007F00EF914
:108C6000851BA5420ED838780028F7D1DAF80070B5
:108C7000184A3A40022A05D1012005B0BDE8F08F1C
:108C8000009AD8E703984FF40272332105B0BDE88B
:108C9000F04F06F0A5B900BF30100B4024100B4078
:108CA00040420F0008100B4000001A0D01000F0099
:108CB000A0DE012010100B40A4DE012000100B40AC
:108CC00094DE012004100B4038100B400C100B40B8
:108CD00027003A1902007F11A8DE01202DE9F04F8C
:108CE000ADF6140D01238C00019011461C4402A81E
:108CF0005C2200948DF80C383D4FDFF83891DFF896
:108D000008A13C4E06F06AFABB46D9F800803A4DFD
:108D100007F0B4F8044604E007F0B0F8001BA842DE
:108D2000F3D83068C107F7D4344A3549C2F8008017
:108D3000516007F0A3F8304C054604E007F09EF8B8
:108D4000431BA342E1D838682E4B0340002BF5D0DB
:108D5000DBF80010CAF80010CBF80010DAF8002099
:108D6000284D29481540012DCFD1284C2368DA051C
:108D7000CBD5274F274A3D70274D00212E78016023
:108D800002A8106026BB009C63021C48234D2449A6
:108D9000244A0360244E254B254C2E600C60136042
:108DA00007F06CF8144E054604E007F067F8421B24
:108DB000B2420FD838780028F7D1DAF800701C4991
:108DC0003940022906D100200DF6140DBDE8F08FC0
:108DD000009BDAE701984FF40272332106F000F9A4
:108DE0000028F0D105200DF6140DBDE8F08F00BF6E
:108DF00030100B4024100B4040420F0008100B4075
:108E000000001A0D01000F00A0DE012010100B4021
:108E1000A4DE012000100B4094DE012004100B4062
:108E200038100B400C100B400002040027003A19C8
:108E300002007F11A8DE01202DE9F04F0123ADF6DD
:108E40001C0D424FDFF84491DFF818A1404E03900B
:108E500089001944019102928DF81438BB46D9F863
:108E600000803C4D07F00AF8044604E007F006F8DD
:108E7000031BAB42F3D83068C107F7D4364A3749F1
:108E8000C2F80080516006F0F9FF324C054604E05C
:108E900006F0F4FF401BA042E1D83868304B034095
:108EA000002BF5D0DBF80010CAF80010CBF800104A
:108EB000DAF800202A4D2B481540012DCFD12A4C3D
:108EC0002368DA05CBD5294F294A3D70294D002169
:108ED0002E78016004A8106046BB019C63021E4A04
:108EE00025492648264D274E274C13600D601663F2
:108EF000046006F0C3FF174E054604E006F0BEFF0F
:108F0000411BB14214D83B78002BF7D1DAF800703E
:108F10001C4A3A40022A0BD104A902985C2206F0AE
:108F20005DF900200DF61C0DBDE8F08F019BD6E722
:108F300003984FF4F472312106F052F80028EBD177
:108F400005200DF61C0DBDE8F08F00BF30100B4062
:108F500024100B4040420F0008100B4000001A0D77
:108F600001000F00A0DE012010100B40A4DE012044
:108F700000100B4094DE012004100B400C100B403D
:108F80000002040002007F1137003A12A8DE01201F
:108F90000EB42DE9F04F82B00BAB064653F8042B0C
:108FA00071480093402106F5BD570AF071F810375B
:108FB00042F2940242F2950142F296033068B854AC
:108FC0000125002406F560567C54DFF8B481FD5479
:108FD0002C36664D02E0012006F074FF326892F8EC
:108FE00064100029F7D14FF48042604809F002FF75
:108FF0005F4800F17B0E00F510698346DA460AF8F7
:10900000804B8BF880408AF880408BF800448BF8C6
:1090100080418BF800428BF880428BF800438BF83C
:1090200080430BF5906BCB45E8D101308645E2D10A
:109030000023FF2203F5D85C03F5DC5003F5E05173
:109040000CF1020E0230023105F80E2003F5E45B4C
:109050002A5403F5E85A6A5403F5EC5903F5F05C19
:1090600003F5F45E03F5F85003F5FC510BF1020B28
:109070000AF1020A09F102090CF1020C0EF1020ECA
:109080000230023103F5A063B3F5206F05F80B2021
:1090900005F80A2005F8092005F80C2005F80E202F
:1090A0002A546A54C6D17D22FF21324809F0A2FE1B
:1090B0000023FF2203F5DB5C03F5DF5003F5E351EA
:1090C0000CF11E0E1E301E3105F80E2003F5E75B75
:1090D0002A5403F5EB5A6A5403F5EF5903F5F35C90
:1090E00003F5F75E03F5FB5003F5FF510BF11E0B83
:1090F0000AF11E0A09F11E090CF11E0C0EF11E0EDA
:109100001E301E3103F5A063B3F5206F05F80B2068
:1091100005F80A2005F8092005F80C2005F80E20AE
:109120002A546A54C6D17D22FF21134809F062FEF9
:10913000124A10680190019BC3F3080001224021EC
:10914000B0F5807FC8F80010C8F80410C8F80C20EB
:10915000C8F81020C8F82C2002D90348FAF780FE7E
:109160003846F9F727FE36E77C30FF1F0831FF1F2E
:109170008B4CFF1F0A4CFF1F8A55FF1FB4DE0120D6
:1091800010CEFF1F2DE9804800F5BD5808F11008EA
:1091900042F29404056808F8045042F2950742F23E
:1091A00096034FF00109002400F5605608F80740C7
:1091B00083B008F80390684D684F894692462C3674
:1091C00002E0012006F07EFE306890F8641000296D
:1091D000F7D14FF48042604809F00CFE604800F17E
:1091E0007B0E00F5106183465A4602F8804B8BF8DF
:1091F000804082F880408BF800448BF880418BF8E7
:1092000000428BF880428BF800438BF880430BF5CB
:10921000906B8B45E8D101308645E2D10023FF22D7
:1092200003F5D85101F1020B03F5DC5C03F5E05EB8
:1092300003F5E45003F5E8510CF1020C0EF1020EB7
:109240000230023105F80B2005F80C2003F5EC5B29
:1092500005F80E2003F5F05C2A5403F5F45E6A5419
:1092600003F5F85003F5FC510BF1020B0CF1020C65
:109270000EF1020E0230023103F5A063B3F5206F48
:1092800005F80B2005F80C2005F80E202A546A5426
:10929000C6D17D22FF21334809F0ACFD0023FF2217
:1092A00003F5DB5B03F5DF5C03F5E35E03F5E750F5
:1092B00003F5EB510BF11E0B0CF11E0C0EF11E0E03
:1092C0001E301E3105F80B2005F80C2003F5EF5B6E
:1092D00005F80E2003F5F35C2A5403F5F75E6A5493
:1092E00003F5FB5003F5FF510BF11E0B0CF11E0CA7
:1092F0000EF11E0E1E301E3103F5A063B3F5206F74
:1093000005F80B2005F80C2005F80E202A546A54A5
:10931000C6D17D22FF21144809F06CFD134A3C613F
:10932000106801900199C1F3080B012340203821F6
:10933000BBF5807F87E80300FB60FB6202D94846EB
:10934000FAF78EFD4122514609487A60FBF71EFC70
:109350004046F9F72FFD34E70831FF1F10CEFF1FFD
:109360008B4CFF1F0A4CFF1F8A55FF1FB4DE0120E4
:10937000C4BD01009C499D4A0B682DE9F04F43F0A4
:1093800040640C6013689A4FDFF87CE2994E9A4D66
:109390009A4C87B043F40033029002F5D128136051
:1093A00001F57E31002300F5A540CEF8003008F22B
:1093B000FC793B60103107464FF0807220373360F4
:1093C000CB462B6001970B602360C9F80020DBF8C7
:1093D00000608B4CF501FAD401998A4840F2771568
:1093E0004D60236823F008022260276827F47F2657
:1093F00026F47F6545F4612141F0E00323600468B1
:109400002407FCD57E4A7B4C13687F4F784E7A4800
:109410007E497A4D43F00803136040F243433B60BA
:1094200033604FF4886704F5C82627602C36036044
:109430000B60774877492B60774C346060254FF498
:10944000003305700B60176847F0006616601068FF
:109450000001FCD40198FFF721F9002840F09E801C
:109460006E4F3E68741E002C3C60C0F28880029DE6
:10947000284605F5A54BFFF77DFF5A46543258465E
:10948000049260300090009BD3ED017AB7EE007A31
:10949000F4EEC77AF1EE10FA75D4B1EE040AF4EEE8
:1094A000C07AF1EE10FA6EDC00990023D1ED050AC6
:1094B000B7EE001AF4EEC10AF1EE10FA06D4F1EE9E
:1094C000041AF4EEE10AF1EE10FA02DD544E4E6198
:1094D000012391ED062AF7EE002AB4EEE22AF1EE1E
:1094E00010FA06D4B1EE043AB4EEC32AF1EE10FA43
:1094F00002DD4B4C8C610123009DAA68052A02D92C
:109500000520A8600123E968012941D92E690124B9
:10951000072EEC6002D9009A012515610198049A82
:1095200001230021FFF73AFB049F029E0C370FCF67
:10953000344654340FC40FCF0FC43A4B716E3868A1
:10954000206003EBC10E384A9EF805609EF8044087
:1095500043F6440A43F6450543F64607012302F85D
:109560000A405655D35507B0BDE8F08F4FF402724C
:109570003321019805F034FD002840F09E810298C7
:109580002A49FFF705FD0099254F4F6001238DE71C
:109590002F69072FBFD8002BC6D0BFE7029A244FF0
:1095A000DFF8A0B0DFF898A0164E02F5A5415431BF
:1095B000B9460491DBF800801E4D06F05FFC0446BE
:1095C00004E006F05BFC011BA942F3D83368D9071D
:1095D000F7D4194A1948C2F80080506006F04EFCD2
:1095E000144C054635E000BF00D8004030800440F0
:1095F00004D0044008D004400CD0044014D00440EF
:109600002C100B4024100B4000D0044010D004401C
:1096100051E400E008E100E00B007F117C22FF1F15
:1096200000002040500302001071FF1FC8BD010060
:1096300030100B4040420F0008100B4000001A0D84
:10964000A0DE0120A8DE012006F018FC431BA34287
:10965000B0D83968A74B0B40002BF5D0D9F80000E3
:10966000CAF80000C9F80000DAF80020A14DA24CA9
:109670001540012D9ED1A1490B68DA059AD5A04F5E
:10968000A04A3D70A048A14EA14B00252560049C36
:1096900004604FF4813115609E489F4D3160106326
:1096A0001D6006F0EBFB9D4E044605E006F0E6FB70
:1096B000001BB04200F209813A78002AF6D1DAF8AC
:1096C0000010944B0B40022B40F0FF8045F2D42C4D
:1096D000029D934955F80C608E4200F00081029C77
:1096E000904A44F80C1004F5A5460499603600969B
:1096F00042F29E668E60009E0125002405204FF0F8
:109700000809C1F804902B46B06072607261B261C2
:10971000F5603561F46134622146049A0198FFF7DF
:109720003DFA00283FF42BAF0299039501F5A940BB
:1097300045F2DC495C3045F2E04241F809400590D1
:109740004FF0630941F802900D460B46059845F22B
:10975000F44E45F2F04645F2F14845F2F24245F248
:10976000F3418460C0F80C900461AC4645F80E905B
:109770000598AC5505F8084045F20856AC5445F23A
:1097800004586C5445F2055245F2065145F207550E
:10979000C461C0F82090446243F8069045F21B5023
:1097A00003F8084045F21C569C5445F218585C5486
:1097B0005C5545F21951059B45F21A551C63C3F8D7
:1097C00034909C630CF5AA4E4CF806900CF80840B7
:1097D0000CF801400CF805400CF80040059DDFF83E
:1097E0005081514EC5F8489000216C64EC64CEF86D
:1097F0002C10CEF83010CEF83410DBF80090474D26
:1098000006F03CFB044604E006F038FB001BA842CF
:10981000F3D83368DB07F7D43A4A4449C2F80090DA
:10982000516006F02BFB3D4C054604E006F026FB9C
:10983000421BA242E1D8D8F800002E4B0340002B77
:10984000F4D03B493A4A0D68CAF800501560DAF87E
:109850000040284B28492340012BCED127480568DA
:10986000E805CAD500240C603249274A08783B70C5
:10987000059B136038BB039D6C022449214B2E4A83
:109880002E48234D1C600860224C2D49146029602D
:1098900006F0F4FA214D044605E006F0EFFA011B4C
:1098A000A9423FF663AE3A78002AF6D1DAF8000012
:1098B000184B0340022B7FF459AE039D04357D2DD8
:1098C00003959AD1DFE5039CD7E74FF4F472312179
:1098D000019805F085FB00283FF4C2ADF6E6049C34
:1098E000A26842F29E6E72452ED002981549FFF78B
:1098F00049FC00BF01000F00A0DE012010100B404A
:10990000A4DE012008100B4000100B4004100B4097
:109910000C100B4002007F1137003A1240420F003A
:109920004B45454E0000204024100B4000001A0D0E
:1099300030100B4094DE012038100B400002040070
:1099400027003A19D8BD0100049B029958680828DD
:1099500001F5A54000F160003FF494AD0646049C7B
:109960008249009001254FF0000908230520A260DC
:1099700063602246B06071607161B1612B46F56031
:109980003561C6F81C90C6F8209049460198FFF74B
:1099900005F900283FF4F3AD0299039501F5A946B6
:1099A0005C360D46344645F2DC4345F2E04845F26C
:1099B000F44E45F2F04645F2F14045F2F2424FF0E6
:1099C000630C059441F8039041F808C00B46C4F8B5
:1099D0000890C4F80CC0C4F8109045F2F34145F863
:1099E0000EC045F2045805F8069005F8009045F2BF
:1099F000085605F80290059805F8019045F20552C1
:109A0000C0F81C90C0F820C0C0F8249045F2065160
:109A100043F806C045F2075503F8089003F8029092
:109A2000029A03F8019045F21C5603F8059011467E
:109A3000059B45F2185845F2195E45F21A5545F254
:109A40001B50C3F83090C3F834C0C3F8389042F8C4
:109A500006C002F8089001F80E9001F8059001F890
:109A60000090059EDFF81C81C6F848C002F5AA42A6
:109A700035464FF0000E3E4EC5F84490C5F84C9068
:109A8000C2F82CE0C2F830E0C2F834E0DBF8009015
:109A9000384D06F0F3F9044604E006F0EFF9001B38
:109AA000A842F3D83068C107F7D43349334BC1F823
:109AB00000904B6006F0E2F92E4C054604E006F0FB
:109AC000DDF9421BA242E1D8D8F800202C48104012
:109AD0000028F4D02B4B2B4D1968CAF800102960D0
:109AE000DAF800402648284920400128CED1274AEC
:109AF0001368DA05CAD500240C602549254D0A787B
:109B00003870059828602ABB039B5D02224C1A48D6
:109B1000224A2349234B05602160234D234C1560C5
:109B20001C6006F0ABF9134D044604E006F0A6F9FC
:109B3000031BAB4210D83A78002AF7D1DAF80000BC
:109B400019490140022907D1039D04357D2D039554
:109B50009CD198E4039DD9E74FF402723321019818
:109B600005F03EFA0028EFD109E500BF00002040D3
:109B700024100B4040420F0008100B4000001A0D4B
:109B800001000F0030100B40A0DE012010100B4030
:109B900094DE012000100B4004100B4038100B40E5
:109BA000000204000C100B4002007F1127003A193C
:109BB0002DE9F04F2DED048B044697B0002363226E
:109BC000CE49DFF83CA3A16504F1C80701204F2668
:109BD000052502972660E565A166E1662066606658
:109BE0002367636784F8783084F8793084F87A30B2
:109BF00084F87B30C4F88030C4F8883084F88C3026
:109C000084F88D3084F88E3084F88F30C4F8943026
:109C1000C4F89C3084F8A03084F8A13084F8A230D5
:109C200084F8A330C4F8A830E267C4F88420C4F8EC
:109C30009020BB46C4F898204FF00008C4F8A42038
:109C4000C4F8AC20C4F8B03084F8B43084F8B5302F
:109C500084F8B63084F8B730C4F8B820C4F8BC3003
:109C6000C4F8C020C4F8C43004F1780904F6E877D9
:109C70000026CBF88483CBF888A3CBF88C83CBF871
:109C80009083CBF89483CBF8BC83CBF880638BF8BC
:109C900099638BF898638BF8B8638BF8B9638BF88A
:109CA000C06331468022584609F0A4F8314630227C
:109CB0000BF5007009F09EF80BF53070314630223C
:109CC0000BF5727B09F096F85F454FF0000CCFD191
:109CD00004F58055A8461C350395029DC4F8F46F21
:109CE00041F2040041F21C014FF0FF33C9EB050BB8
:109CF000029DC4F8EC3FC4F8F03FC4F8F86F84F854
:109D0000FC6F84F8E86F04F5815EC8F8003004F554
:109D1000825A265409F11403665403996322ABF165
:109D200014009D424E708E70C0F38100CEF804C0C6
:109D3000CEF808C0CEF80CC0CEF810C0CEF814C0D3
:109D4000CEF818C0CAF80CC089F8006089F8016024
:109D500089F8026089F80360C9F80860C9F81060E2
:109D6000C9F80420C9F80C2058D0002801F08187D8
:109D7000012814D0022809D01E705E709E70DE701B
:109D80005A609E60DA601E6109F128031E705E70E1
:109D90009E70DE705A609E60DA601E611433029914
:109DA0001E705E709E70DE705A609E60DA601E618A
:109DB0001433994218BF8E4630D01E705E709E706C
:109DC000DE705A609E60DA601E611E755E759E755B
:109DD000DE759A61DE611A625E6283F8286083F83C
:109DE000296083F82A6083F82B60DA621E635A6365
:109DF0009E6383F83C6003F13C0950339E4589F82B
:109E0000016089F8026089F80360C9F80420C9F884
:109E10000860C9F80C20C9F81060CED1029EBE427D
:109E200000F0C8804FF0000A4FF00009BA1BDFF8BD
:109E3000D0B0C6F88493A2F572733546C6F88C93F9
:109E4000C6F89093C6F89493C6F8BC93C6F888B346
:109E5000C6F880A386F899A386F898A386F8B8A3D5
:109E600086F8B9A386F8C0A3514680223046C3F3D2
:109E7000C00608F0BFFF5146302205F5007008F01B
:109E8000B9FF05F530705146302205F5727508F0BE
:109E9000B1FFAF4200F08E80A6B3C5F880A3C5F82D
:109EA0008493C5F888B3C5F88C93C5F89093C5F82A
:109EB000949385F899A385F898A385F8B8A385F8B5
:109EC000B9A3C5F8BC9385F8C0A3284680225146A3
:109ED00008F090FF029D3022514605F5B96008F068
:109EE00089FFAC46514605F5F26530220CF5D1608C
:109EF00008F080FFAF425DD004E000BF00002040CA
:109F000000005C410026C5F88493C5F888B3C5F805
:109F10008C93C5F89093C5F89493C5F8BC93C5F895
:109F2000806385F8996385F8986385F8B86385F848
:109F3000B96385F8C06331468022284608F05AFF8D
:109F40003146302205F5007008F054FF31463022CA
:109F500005F5307008F04EFF05F57270314680222D
:109F6000C0F88493C0F88063C0F888B3C0F88C93BD
:109F7000C0F89093C0F8949380F8996380F8986340
:109F800080F8B86380F8B963C0F8BC9380F8C06308
:109F900008F030FF3146302205F5B96008F02AFF9D
:109FA00005F5D1603146302205F5F26508F022FF53
:109FB000AF42A7D141F2040041F21C0300224FF04E
:109FC000FF37039DC4F8EC7F41F23C01C4F8F07FF9
:109FD000C4F8F42FC4F8F82F84F8FC2F84F8E82F85
:109FE00004F5835BC8F8007004F58259225441F2ED
:109FF0006408E25441F2500041F278036A70AA709A
:10A0000004F5845C625463279C4EC9F8006041F2F9
:10A010008C01225489F8112089F8122089F8132024
:10A02000C9F81820C9F82020C9F81470C9F81C70A4
:10A0300004F808208BF805208BF806208BF8072001
:10A04000CBF80C20CBF81420CBF80870CBF81070AC
:10A05000E2548BF819208A4B8BF81A208BF81B20BE
:10A06000CBF82020CBF82820CBF81C70CBF824703C
:10A0700004F5855B62544FF000098CF80D208CF8D4
:10A080000E208CF80F20CCF81420CCF81C207D4A30
:10A09000CCF81070CCF8187003F5A07ACBF80090CB
:10A0A000CBF80490CBF80890A4461E689F689C6982
:10A0B0001D6A996A186B02EBC60E02EBC708DEF840
:10A0C00004605F6837601E69D8F80490DF68C9F8DB
:10A0D000007002EBC60B02EBC408DBF804E05C691D
:10A0E000CEF80040D8F80460DF69376002EBC505A0
:10A0F00002EBC1016C685E6A26604F689D6BD96A8D
:10A10000396002EBC0005E6B446802EBC509266053
:10A11000DD6BD9F8047040339A453D60C5D15A4B88
:10A120005A4819685A4E5B4A41F400071F60056897
:10A13000594F25F0020141F2B00A01604FF400309E
:10A140004CF80A20306096684EF6602546F0020111
:10A15000916015601A684FF0804042F400466446F2
:10A160001E60BC463860DCF80030002BFBDB04F5D9
:10A17000855B5F46494E4A4A4A4B4B49DFF84CE102
:10A180004A4DDFF84C91DFF84C8149481837049765
:10A190004FF263073760002717604FF4403C0122FD
:10A1A0001A6041F2B80AC1F8009004F5865BCEF857
:10A1B00000C041F2C403C5F800803E4E049DDFF8A4
:10A1C0001891DFF818E13C49C0F8009044F80AE023
:10A1D000706B6C60CBF80010E750364B354E016861
:10A1E0009B6BD6F830A0354D354E04F5865808F1F6
:10A1F000080904F5865E41F2C80C43EA010B314BB5
:10A2000044F80C30022189F8041089F80C7089F8A0
:10A210000D70C9F81070CEF85C70CEF86070C0F8A0
:10A2200000B0C9F808A08AF80070D9F80800477093
:10A23000D9F808309F70D9F80800FF21C170D9F80B
:10A2400008305F71D9F8080050218171D9F80830C1
:10A25000DF71D9F80800817801F07F038370D9F8A5
:10A2600008001221C1709346BC46BE464FF0FF3134
:10A27000154A0BFA07F80020CCE000BF000080BFB1
:10A2800024B90100141304003C8004400070034012
:10A2900004E100E01071034000F1024004F10240CB
:10A2A00060F0024004F0024008F0024010F002406A
:10A2B00014F0024034120400396300009F8601004C
:10A2C00000879303386E0100921204000CF00240E4
:10A2D00003000007130F0100000F0F0FC06E0100F5
:10A2E000CAF5C333A0338B4202D21946BC46864618
:10A2F000B2F802A008FB0AF3B6FBF3FAAA4500F194
:10A30000010000F29E80CAF5C333A0338B4202D213
:10A310001946BC468646938808FB03F3B6FBF3F365
:10A32000AB4200F1010A40F29880A3F5C333A03B91
:10A330008B4205D2D646BC46002B00F0CC80194695
:10A34000D38808FB03F3B6FBF3F3AB4200F1020A38
:10A3500040F28D80A3F5C333A03B8B4205D2D64695
:10A36000BC46002B00F0B7801946138908FB03F3A5
:10A37000B6FBF3F3AB4200F1030A40F28280A3F58F
:10A38000C333A03B8B4205D2D646BC46002B00F01F
:10A39000A2801946538908FB03F3B6FBF3F3AB42E3
:10A3A00000F1040A76D9A3F5C333A03B8B4205D252
:10A3B000D646BC46002B00F08E801946938908FBD8
:10A3C00003F3B6FBF3F3AB4200F1050A6BD9A3F537
:10A3D000C333A03B8B4204D2D646BC46002B7AD076
:10A3E0001946B2F80EA008FB0AF3B6FBF3F3AB4232
:10A3F00002F10E0200F1060A5ED9A3F5C333A03BB9
:10A400008B4204D2D646BC46002B64D01946073096
:10A4100040285CD0B2F802A008FB0AF3B6FBF3FABE
:10A42000AA4502F102027FF65BAFAAF5C333A03B57
:10A430008B42BFF45DAFBC468646002B4BD019461D
:10A4400056E7AAF5C333A03B8B42BFF464AFBC46CA
:10A450008646002B3FD019465DE7C3F5C333A033D2
:10A460008B42BFF46DAFD6461946BC4668E7C3F5CC
:10A47000C333A0338B42BFF478AFD6461946BC46EF
:10A4800073E7C3F5C333A0338B4283D2D646194654
:10A49000BC467FE7C3F5C333A0338B428ED2D6468A
:10A4A0001946BC468AE7C3F5C333A0338B4298D222
:10A4B000D6461946BC4694E7C3F5C333A0338B4256
:10A4C000A5D207304028D6461946BC46A2D1022F55
:10A4D00001D00137CCE641F2D0050EF03F026159C0
:10A4E000DFF89C83E14F42EA8C10C3B24B70D9F87D
:10A4F0000860727942F020007071D9F8081091F864
:10A5000005A04AF080034B71D9F80860D84BB278A7
:10A5100042F08000B07099F804E00EEB4E0103EBBE
:10A52000C10C04F5895BDCF80C607209900000F145
:10A53000604A0AF5614306F01F0C012606FA0CF288
:10A540001A6041F22811CB4B584641F2301E0BF1F4
:10A55000080B41F2381241F23C1AC3F8089044F853
:10A56000019009F160030021CBF8041044F80E803B
:10A57000436144F80A1004F58A50A750402205931D
:10A5800008F038FC38208BF85A006559A97801F09A
:10A59000BF02AA70DBF8040089F80D6058B10668A4
:10A5A000B54D7368AB420BF1080241F0538340682C
:10A5B0000221F7F7A5FC9BF858008BF8590004F529
:10A5C0008C56B44641F29813043641F2841E41F28F
:10A5D0008C1A41F2941B002109F1BC0244F80E9040
:10A5E00006F11800716044F80A80CCF810209246F9
:10A5F000E150402244F80B7008F0FCFB41F2D0051A
:10A60000392186F85A10605990F802C00CF0BF0347
:10A6100083707068012289F80D2058B10568964949
:10A620006B688B4206F1080241F0198340680221F1
:10A63000F7F766FC04F58F5B41F2E81241F2F41083
:10A6400041F2F01E96F8581086F859100023CBF806
:10A650000430CBF80090194644F80280CBF80CB0D7
:10A66000402223500BF1180044F80E70CDF804B0CE
:10A670003A2708F0BFFB41F2D0008BF85A702158FE
:10A680005D4691F802B00BF0BF038B70686801273C
:10A690002A4689F80D7058B1036877495D688D4284
:10A6A00002F1080241F0E08240680221F7F728FC3D
:10A6B000019DDFF8D0B195F85810079104F591523B
:10A6C00041F23C2E04F5925941F24428002344F80B
:10A6D0000EA0142715624FF4FA71684DC9F81030B6
:10A6E000C9F80870C9F80C10C9F8143089F8183086
:10A6F00089F81930504644F80850C9F81CA04FF0AA
:10A70000020A89F820A096F95950069504F5985147
:10A71000079D0431089145F00F01069D079104F54E
:10A72000935A65F0030102F12405CAF8105006910E
:10A730004FF4FA7504F59951CAF80C50043141F2FE
:10A74000642509914D49CAF8087004F59459CAF86E
:10A7500014308AF818308AF8193061514FF0030527
:10A76000CAF81C008AF8205002F1440AC9F810A067
:10A7700041F2842A4FF4FA75C9F8087004F5955827
:10A78000C9F80C50C9F8143089F8183089F8193014
:10A790004FF0040544F80A1041F2A42AC9F81C003D
:10A7A00089F8205002F164094FF4FA75C8F808706E
:10A7B000C8F80C50C8F8143088F8183088F81930E8
:10A7C000C8F8109004F5965C44F80A104FF005059F
:10A7D00041F2C42AC8F81C0088F8205002F184080D
:10A7E0004FF4FA75CCF81080CCF80870CCF80C5007
:10A7F000CCF814308CF818308CF8193004F5975ECA
:10A8000044F80A104FF0060841F2E42ACCF81C0084
:10A810008CF820804FF4FA7502F1A40CCEF810C029
:10A82000CEF80870CEF80C50CEF814308EF81830F0
:10A830008EF8193044F80A10CEF81C004FF00700CB
:10A840008EF8200008989DF8185086F8595002F1AB
:10A85000C40E0546C0F80CE04FF4FA7A41F2043E0B
:10A8600047600199C5F808A00EE000BF550D000033
:10A870003412040084DE0120ED230000946E0100F8
:10A88000886E0100B4DE0120C14D0361037543757C
:10A8900044F80E5081610377099802F1E40E0546F1
:10A8A00041F22431C0F80CE04760B948C5F808A06F
:10A8B0002B612B756B7504F59A5960504FF0010AA6
:10A8C0000198A86185F81CA04FF4FA7141F2443553
:10A8D00004F59B56C9F80C1002F5827EAC49C9F804
:10A8E00010E0C9F80870C9F8143089F8183089F8F0
:10A8F000193041F2643E6151C9F81C0001464FF421
:10A90000FA754FF0020089F82000F56002F59270A8
:10A910009F4DB760736133767376306144F80E50A3
:10A92000F1614FF0030186F82010019E9DF81C5044
:10A9300086F8595002F5A270C2F86401DBF80000F5
:10A940000B90DDF82CE0DBF80010059D0C9104F570
:10A950009C5C41F288370C99E551CCF80C60DBF82F
:10A9600000600D960D9ADBF800700E9741F2903959
:10A9700004F59D57DDF838C00592DBF800000F9014
:10A9800004F59C5244F809504FF0020982F81490E3
:10A99000C2F81CE0F96004F59F51069141F2B0390C
:10A9A0004FF00701397104F59E5605993D6041F25B
:10A9B000D03E44F809500F98F96187F814804FF0A1
:10A9C00004024FF00507C6F80CC03560377144F833
:10A9D0000E50F0613275DBF800601096DDF840C073
:10A9E000DBF800001190119FDBF80020069912920D
:10A9F000129EDBF800000D6081F804A00597069612
:10AA000041F2F03E1390139FDBF800201492C1F83E
:10AA10000CC0079744F80E500F46149D08954FF050
:10AA200003053D7504F5A056059DFD614FF0040733
:10AA3000377104F5A150019FDBF800B0069DCDF8F9
:10AA400054B0314641F21049024641F2304C0F6099
:10AA5000BB46F560089944F80970079DF5614FF011
:10AA60000507377541F2D00E80F804804FF00707D4
:10AA7000C2F800B0C16044F80CB0077554F80E80FD
:10AA8000159DC56198F806004249434FDFF81C91B7
:10AA9000424A04F5A255AC4640F0040603C988F8C2
:10AAA00006604CF8047B8CE803003D483D4F03C82A
:10AAB00005F10C0E8EE80300D9F80060C5F8843269
:10AAC00046F00061C5F8883285F814A0AA61C9F87B
:10AAD000001093687D6023F00C009060966846F04B
:10AAE00004019160536A43F004075762506A20F0F2
:10AAF00003065662516A41EA0A035362D76847F077
:10AB00000800D060966846F003019160936843F0B6
:10AB100020079760D06840F00406D660116A11F0F3
:10AB2000400104F1140B04D0136A23F0400751468E
:10AB300017621A4A506A40F0C0065662536A174FAD
:10AB40001E06FBD47B6A3B6919B1396A41F04002A9
:10AB50003A62124B1448D3F84CA09F6C5A6C196C93
:10AB6000DE6BDFF84C805744174439449F6B314407
:10AB70000F447A0842F40042DA62DF6E996E5E6E2C
:10AB800039440E44196EDF6D31440F4412E000BFAA
:10AB9000946E0100686F0100286E010000B00B4048
:10ABA000706F01007CDD0120A06E01003080044048
:10ABB0000D130000996D394411444F0847F40041CA
:10ABC000196341F2D46300274FF0100CC5F88CB222
:10ABD0002860C5F8907204F5B65944F803C041F2F4
:10ABE000E463984904F5B7564FF0110E13204FF067
:10ABF000120BC9F818E0C9F81C00C9F820B00436D7
:10AC0000E15041F2EC63C6F804C004F5B752E150DC
:10AC100041F2F4631746C2F810E01C37E15041F2EC
:10AC2000FC6943464345906144F80910C7F804B0F5
:10AC30004FF001010BD1307905F0E4F8B7420BD0A9
:10AC400056F8082F136843454FF00101F3D0012156
:10AC500030469847B742F3D1D5F88C62DFF808B296
:10AC6000C5F8CC62B31C301D06F10E07C5F8D4320E
:10AC7000C5F81433C5F8DC0206F11003C5F81C034F
:10AC8000C5F8047306F11200032706F1060806F161
:10AC9000080106F10A0206F10C0EC5F82C33C5F8BE
:10ACA0003403C5F8E072C5F8207304230520092792
:10ACB000C5F8E482C5F8248306F1140CC5F8EC123B
:10ACC000C5F8F42200210122C5F8FCE24FF0020A87
:10ACD000C5F8E832C5F8F002C5F82873082006F177
:10ACE00016074FF006094FF007080A234FF00B0E26
:10ACF000C5F80C63C5F83CC3C5F8C412C5F8C81242
:10AD0000C5F80813C5F8D8A2C5F818A3C5F8F89275
:10AD1000C5F80083C5F83033C5F83803C5F8D0222C
:10AD2000C5F81023C5F840E3DBF80030C5F84473DC
:10AD300006F11A071836C5F84C73C5F854630D2789
:10AD40000C26C5F84863C5F8507304F5BC5EDFF8FF
:10AD50001CC1DFF81CA143F4806332260027CEE932
:10AD60000667CBF80030DCF80030374E374F0BF574
:10AD7000012543F0007347F6FF79CCF8003005F564
:10AD80007E6BCAF80010C6F80090314E314DF6695E
:10AD90002823CBF800303B602D4F286030683D6A97
:10ADA0002B4BCEF8241004F55E5B5F46284343F23C
:10ADB000B0753837D3F818C0224BCEF8281004F5F8
:10ADC0005F5A43F2B878CEF82C106351224DCBF87D
:10ADD000341044F808503973797339613A71CAF8FC
:10ADE0004C10CAF850103060C7F808C08CF800103A
:10ADF000B8681A4E4170BB68194D9970BB680192D2
:10AE0000FF20D870BB685971BB6850209871BB682F
:10AE1000D971B86890F802E00EF07F038370B868CB
:10AE20008E4604F5BD591221C170F046F44609F171
:10AE3000100B4FF0FF31104600FA0EF9094A0020BE
:10AE4000BCE000BF706E010008A00C4014A00C40D4
:10AE50003412040000A00C40386E010000879303F8
:10AE60003F771B00921204002C80044004800440B1
:10AE700004A00C40CAF5DB1A0AF5BA53994202D96C
:10AE800019468446F046B2F802A009FB0AF3B6FB65
:10AE9000F3FAAA4500F1010000F2A880CAF5DB1A16
:10AEA0000AF5BA53994202D919468446F046938866
:10AEB00009FB03F3B6FBF3F3AB4200F1010A40F2E6
:10AEC000A280A3F5DB13A3F5BA53994205D9D44662
:10AED000F046002B00F0DF801946D38809FB03F30E
:10AEE000B6FBF3F3AB4200F1020A40F29780A3F500
:10AEF000DB13A3F5BA53994205D9D446F046002B8B
:10AF000000F0C9801946138909FB03F3B6FBF3F37C
:10AF1000AB4200F1030A40F28C80A3F5DB13A3F5EA
:10AF2000BA53994205D9D446F046002B00F0B380BD
:10AF30001946538909FB03F3B6FBF3F3AB4200F167
:10AF4000040A40F28180A3F5DB13A3F5BA539942BA
:10AF500005D9D446F046002B00F09D801946938910
:10AF600009FB03F3B6FBF3F3AB4200F1050A75D915
:10AF7000A3F5DB13A3F5BA53994205D9D446F0469D
:10AF8000002B00F088801946B2F80EA009FB0AF3E6
:10AF9000B6FBF3F3AB4202F10E0200F1060A67D9E9
:10AFA000A3F5DB13A3F5BA53994204D9D446F0466E
:10AFB000002B70D019460730402865D0B2F802A0A7
:10AFC00009FB0AF3B6FBF3FAAA4502F102027FF687
:10AFD00051AFAAF5DB13A3F5BA5399427FF653AFED
:10AFE000F0468446002B56D019464CE7AAF5DB13F1
:10AFF000A3F5BA5399427FF65AAFF0468446002B28
:10B0000049D0194653E7C3F5DB1303F5BA53994208
:10B010007FF663AFD4461946F0465EE7C3F5DB130F
:10B0200003F5BA5399427FF66EAFD4461946F046FF
:10B0300069E7C3F5DB1303F5BA5399427FF679AF9D
:10B04000D4461946F04674E7C3F5DB1303F5BA534B
:10B05000994284D9D4461946F04680E7C3F5DB13FC
:10B0600003F5BA5399428FD9D4461946F0468BE777
:10B07000C3F5DB1303F5BA5399429CD90730402836
:10B08000D4461946F04699D1BEF1020F03D00EF115
:10B09000010E0198D0E604F55F5A0CF03F02DAF891
:10B0A0000050E449DFF8B0939FEDE38A42EA881349
:10B0B000DEB26E70B868427942F020034371BD6819
:10B0C0006E7946F080006871BA68DC4E92F802C072
:10B0D0004CF08003937097F8048008EB480506EB6A
:10B0E000C50E0126DEF80C004209930003F1604C06
:10B0F0000CF5614843F2B87ED14A00F01F0506FA0C
:10B1000005F00025C8F800005760082044F80E102C
:10B110003D6687F86450BD6604F080F92946804694
:10B1200003F084FFB968C7F860808B78C548DFF802
:10B130002CE303F0FE028A70396EC04A0B7903706B
:10B1400097F804C0386E0CEB4C0802EBC801037989
:10B15000086903F1804C0CF5043100F03F0848F019
:10B1600080020D700A70386E3B79B449027903EBA6
:10B17000430C01EBCC08531102F1100CD8F8141059
:10B180004EF82C109B0003F1604E0EF5614802F062
:10B190001F02016806FA02F3C8F80030888B82B2F9
:10B1A00042F0080CA1F81CC08B8B1FFA83FE4EF0F6
:10B1B00002028A8343F62C00A14A04F560580BF57D
:10B1C000015357603C3327500BF500514FF03C0CB6
:10B1D0004FF40057C8F8301088F838C0C8F834B0B9
:10B1E00088F84060C8F83C7018460193F7F718FCDF
:10B1F0000198F7F799FC42F2970C42F2960388F80F
:10B200004050DAF800100BF80C600BF803508A7904
:10B2100004F56157083704F5615B42F007000BF154
:10B22000380804F5625A8871022231463846F8F728
:10B2300019FC0AF1280A3D627D62BD62C7F82C90B4
:10B24000404604F5635706220521F8F70BFC183732
:10B2500004F5645BC8F82050C8F82450C8F828509A
:10B26000C8F82C90504608220721F8F7FBFBD84677
:10B27000CAF820500BF1080BCAF82450CAF828501D
:10B28000CAF82C9038460B221F21F8F7EBFB3D62E1
:10B290007D62BD62C7F82C901C2258461B21F8F72E
:10B2A000E1FBCBF82C9043F6381904274FF0320A13
:10B2B0000A21CBF82050CBF82450CBF82850384640
:10B2C00044F809A0C8F84010C8F83C7088ED118A0D
:10B2D000019104F081FC43F6381C44F6206954F8CF
:10B2E0000C3098F8400009FB03F200EE102AB8EE8B
:10B2F000C00A04F081FCD8F83C00019B06FA00FB70
:10B300000BEBDB7104F56558184643F6481B3141D9
:10B3100004F068FA032144F80BA03846C8F810106E
:10B32000C8F80C7088ED058A04F056FC54F80B2020
:10B3300098F8100009FB02FC00EE90CAB8EEE00A93
:10B3400004F05AFCD8F80C0006FA00F808EBD871A3
:10B350003141032004F046FA04F5655B43F65813C7
:10B360004FF01D0844F803A03846CBF81C70CBF80A
:10B3700020808BED098A04F02FFC43F658119BF8CE
:10B380002000625809FB02FC01EE10CAB8EEC10AA7
:10B3900004F032FCDBF81C0006FA00F303EBD37177
:10B3A0003141404604F01EFA04F5655B43F668112E
:10B3B0004FF0230844F801A03846CBF82C7043F630
:10B3C00068178BED0D8ACBF8308004F005FCE2594C
:10B3D0009BF8300009FB02FA01EE90AAB8EEE10AF0
:10B3E00004F00AFCDBF82C0006FA00F909EBD9712D
:10B3F0003141404604F0F6F9134B144A04F5655701
:10B4000093E80300383743F6781C07F1040E44F83C
:10B410000C208EE803000E490E4B03C907F10C0BFC
:10B420008BE803001A683D75C7F88452C7F8885244
:10B4300016E000BF546E010000000000341204004A
:10B4400084DE01201A800040686F0100286E010030
:10B45000706F01003C800440010000800002FF1F6B
:10B46000DE4DDF48B86142F000612F6019608368EB
:10B4700023F00C058560826842F004018160436A14
:10B4800043F004054562426A22F003014162436AC7
:10B490004362C56845F00802C260816841F0030359
:10B4A0008360856845F020028260C16841F0040332
:10B4B000C360056A15F040021EBF026A22F0400216
:10B4C0000262C748416A41F0C00308BF16464362A2
:10B4D000456AC34A2B06FBD4536A13691EB1166A28
:10B4E00046F040001062BE4DDFF80093D5F84C8066
:10B4F000A96C6B6C2E6CE86BAA6BDFF8F4E2DFF8DA
:10B50000F4A29FEDB89A41441944314401441144D6
:10B510004B0843F40046EE62D5F86CC0AA6E6B6E21
:10B52000286EE96D62441A441044AA6D084400EB89
:10B53000020899E80F00464443F6781C760807F5A0
:10B54000237846F400462E63002644F80CE004F508
:10B55000705588E80F0043F6304C43F634420498A7
:10B56000C7F89C024FF0000BC7F8A0620C2340F212
:10B57000DC589D4FC5F824A0C5F81CB0C5F820B014
:10B580001846AE62EE62012144F80C80A750AB630E
:10B5900004F038FC04F57153F7EE009A04F5725C80
:10B5A0001946F6EE008A43F6A44785F84060043356
:10B5B000C3F800B0C3F80CB0C3F810B0C3F814B0AF
:10B5C000C3ED019AC3ED079A83ED029AC3ED068A93
:10B5D000C1F824B0C1F830B0C1F834B0C1F838B007
:10B5E000C1ED0A9A81ED0B9AC1ED0F8AC1ED109A57
:10B5F000CCF804B0CCF810B0CCF814B0CCF818B03B
:10B60000CCED029A8CED039ACCED078ACCED089A2A
:10B61000E351012704F5735ACCF828B0CCF830B0C8
:10B62000CCF834B08CF83870CCED0B9A43F6F84176
:10B6300043F6DC4C04F5745804F5755503F120020B
:10B640004033CAF80020CAF804B0CAF80CB0CAF8EF
:10B6500010B08AF81470CAED029A44F80C30CAF897
:10B6600020B0CAF828B0CAF82CB0CAED099A8AF8F6
:10B67000306063504FF0FF33CAF83CB0CAF844B0B2
:10B68000CAF848B0CAED109A8AF84C6008F1780000
:10B69000C5F81CB0C5F820B0C5F824B03146C8F8CC
:10B6A0006830C8F87030202288F86C6088F86D60C7
:10B6B00088F8746007F09EFB08F19800314620225C
:10B6C00007F098FB09F1100A08F1B8003146202272
:10B6D00007F090FB9AE80F0004F5775E0EF1300C4E
:10B6E00088F8DC7088F8D86088F8D96088F8DA6063
:10B6F00088F8DB608CE80F00902209F1200104F546
:10B70000785003F06BFD04F57A5504F57B5004F591
:10B710007C5304F57D59C5F810B0C5F81CB0C5F8C8
:10B7200020B0C5F824B0C5F830B0C5F83CB0C5F8B5
:10B7300040B0C5F844B0C5ED059A85ED069AC5ED53
:10B740000A8AC5ED0B9AC5ED0D9A85ED0E9AC5EDE9
:10B75000128AC5ED139A0299C0F810B0C0F81CB057
:10B76000C0F820B0C0F824B0C0F830B0C0F83CB089
:10B77000C0F840B0C0F844B0C0ED059A80ED069A1C
:10B78000C0ED0A8AC0ED0B9AC0ED0D9A80ED0E9ABD
:10B79000C0ED128AC0ED139A04F57F50C3F810B0C3
:10B7A000C3F81CB0C3F820B0C3F824B0C3F830B05D
:10B7B000C3F83CB0C3F840B0C3ED059A83ED069AD8
:10B7C000C3ED0A8AC3ED0B9A83ED0E9AC3ED0D9A71
:10B7D000C3ED118AC3ED129A0EE000BF7CDD01209B
:10B7E00000B003400AD7233C706E0100786F01005F
:10B7F000B06E0100000096430C30C9F80CB0C9F8D7
:10B8000014B0C9F818B0C9F81CB0C9F824B0C9F808
:10B8100028B0C9F82CB0C9F834B0C9F838B0C9F8A4
:10B820003CB0C9F844B0C9F848B0C9ED049AC9EDB4
:10B83000089AC9ED0C9AC9ED109AFAF727FE04F59B
:10B84000884004F592616430FAF720FE04F59140D7
:10B8500004F658017C30FAF719FE04F59B4004F514
:10B8600042611430FAF712FE04F5A44B45F22C2184
:10B87000AE4A66540BF1300E45F23020D2F804C0C7
:10B88000AA4BAA4926548EF80160DCF8002008680B
:10B890009D68A74BCEF8043004F5A441894645F2D3
:10B8A000382338312A43A34DE5500E710E734E7381
:10B8B0000E61C9F88C60C9F89060CCF800208860EF
:10B8C000067088689C4A46708D689C4BAE7088688C
:10B8D0004FF0FF35C570886846718D685020A8719B
:10B8E0008D68EE71D1F8088098F802A004F5A44C98
:10B8F0000AF07F0B654688F802B02C3588680295FF
:10B900004FF0120980F803900298019704300EF16D
:10B9100008074FF0FF350597B046B14604900198EF
:10B92000874F00FA06FA4FF0000C9CE0CBF5C330CD
:10B93000A030854202D90546B146E046B7F802B0CC
:10B940000AFB0BF0B2FBF0FB9B450CF1010C00F283
:10B95000A180CBF5C330A030854202D90546B1465F
:10B96000E046B8880AFB00F0B2FBF0F098420CF118
:10B97000010B40F29B80A0F5C330A038854205D969
:10B98000D846B146002800F0DD800546F8880AFB5D
:10B9900000F0B2FBF0F098420CF1020B40F2908004
:10B9A000A0F5C330A038854205D9D846B146002855
:10B9B00000F0C880054638890AFB00F0B2FBF0F0C1
:10B9C00098420CF1030B40F28580A0F5C330A038FB
:10B9D000854205D9D846B146002800F0B380054617
:10B9E00078890AFB00F0B2FBF0F098420CF1040BEE
:10B9F00079D9A0F5C330A038854205D9D846B146DB
:10BA0000002800F09F800546B8890AFB00F0B2FBD1
:10BA1000F0F098420CF1050B6ED9A0F5C330A038B8
:10BA2000854205D9D846B146002800F08B800546EE
:10BA3000B7F80EB00AFB0BF0B2FBF0F0984207F13A
:10BA40000E070CF1060B60D9A0F5C330A038854273
:10BA500004D9D846B146002874D005460CF1070C2D
:10BA6000BCF1400F5ED0B7F802B00AFB0BF0B2FB9E
:10BA7000F0FB9B4507F102077FF658AFABF5C330EB
:10BA8000A03885427FF65AAFB146E046002859D02B
:10BA9000054653E7ABF5C330A03885427FF661AF6A
:10BAA000B146E04600284DD005465AE7C0F5C33000
:10BAB000A03085427FF66AAFD8460546B14665E7B5
:10BAC000C0F5C330A03085427FF675AFD846054635
:10BAD000B14670E7C0F5C330A030854280D9D84662
:10BAE0000546B1467CE7C0F5C330A03085428BD90E
:10BAF000D8460546B14687E7C0F5C330A030854239
:10BB000096D9D8460546B14692E7C0F5C330A03075
:10BB10008542A3D90CF1070CBCF1400FD84605466D
:10BB2000B146A0D1022E0DD00136F8E63412040041
:10BB3000A9110000386E0100008793039F86010061
:10BB40009212040045F2402B08F03F0754F80B50C6
:10BB500047EA8910C2B26A708E6896F805A04AF06A
:10BB6000200373718F68787940F080057D718A6851
:10BB70004148967846F08003937091F8048008EB72
:10BB8000480700EBC7090122D9F80C506E09B30031
:10BB900003F1604C05F01F070CF5614A374B059E19
:10BBA00002FA07F00025CAF800001E608EF86850FF
:10BBB0008F68BD7000BF8E68314B3248DFF8C8E037
:10BBC000DFF8C8A08027B7708F684D733D7054F8B8
:10BBD0000B80029E98F802901E6049F0400C88F895
:10BBE00002C0049B54F80BB00360022048739BF81A
:10BBF000067004F5A54045F24828034647F00709BA
:10BC00008BF80690203344F808E004F5A941B046CB
:10BC100045F2A02B5C3145F6E44C45F6E84E039E18
:10BC2000C8F870604FF0FF3744F80B501D72DD60AC
:10BC30001D745D7480F85822204681F80428CAF8E3
:10BC4000003044F80C7044F80E7017B0BDEC048B53
:10BC5000BDE8F08F114602229847FEF7ACBC1146B2
:10BC600002229847FEF7E6BC11460222A847FEF7DB
:10BC70001FBDAE46FEF7A1B83412040084DE0120D9
:10BC80000871FF1F78DC0120191A00009CDE0120DA
:10BC90002DE9F04FDE4B2DED068B0FCB97B012AD9B
:10BCA00085E80F00042003F097FF55F8044B9FED43
:10BCB000D90AE6B2304603F09FFF3046082103F070
:10BCC00091FD16A88542F0D101210D2004F09AF8CB
:10BCD000D14FD24ED24AD34DD349D448D44B00246D
:10BCE0003C703470402714705026702207700E701C
:10BCF00028461A70FDF73EFB41F2D06041F2087110
:10BD00002C5015F80180C74FE30003F5B7500430FD
:10BD100048FA04F62A5806F00101936828440134D1
:10BD20009847042CEFD141F25444C24E385DC249C9
:10BD3000821C41F2584956F8222057F809404D27F5
:10BD400007FB001A530998009AF843B0266800F1DF
:10BD5000604C02F01F0E0CF5614701220BF01F0032
:10BD600002FA0EF346F040061F2826603B600AD018
:10BD70005FEA0B624ABFE768102727F01007E76009
:10BD800040F04007276043F68C1443F618482B5DBB
:10BD900055F80800A94E9A1CA23056F8227056F8A1
:10BDA000204043F690194FF04D0A0AFB031155F855
:10BDB000090011F804B006687B099A0002F1604C92
:10BDC0000CF5614E07F01F0701240BF01F0104FA68
:10BDD00007F346F040061F290660CEF800300AD06F
:10BDE0005FEA0B624ABFC268102222F0100241F0E3
:10BDF0004007C26007600A2004F064F8A88D904CE8
:10BE0000B5F82E809FED8F8AB5F82A90DFED8E8AE7
:10BE10008E4EC4ED098A06EE900AB8EE660A2346F5
:10BE200010EE10CA07EE108A43F810CFA046119307
:10BE300048F80CCF10EE103AA446A2464CF8703FDA
:10BE400010EE103ACDF824C0D446F8EE470A4CF86C
:10BE50006C3F18EE103ACDF828C0D44607EE909A01
:10BE60004CF8143F18EE103ACDF800C0D446A14665
:10BE70004CF8203F10EE903ACDF804C0D446B8EE0E
:10BE8000671A4CF82C3F10EE903ACDF808C04AF8EB
:10BE9000303FCC4618EE103A4CF8343F18EE103ACA
:10BEA000CDF80CC0CC46A3464CF8403F11EE103AFA
:10BEB000CDF810C0CC46ABEC018A4CF84C3F11EEEB
:10BEC000103ACBED008AA34649F8503FCDF814C094
:10BED00018EE103ADC46C4ED118A4CF8543F18EEC7
:10BEE000103ACDF818C0DC4659494CF8643F18EEBA
:10BEF000903ACDF81CC0DC46564A4CF8683F18EE24
:10BF0000103ACDF820C0DC46DFF854E14CF8803F11
:10BF100018EE903ACDF82CC0DC4684ED311A4CF87E
:10BF2000843F84ED301A10EE903ACDF830C0A66010
:10BF3000A662A664A161A163A165E261E263E26514
:10BF4000C4F8D462C4F8E412C4F8E82284ED2E8A5E
:10BF5000C4ED2F8A84EDB38AC4EDB48A84EDB68A29
:10BF600084EDB78A84EDB88A84EDBB8AC4EDBC8ABF
:10BF700084EDBE8A84EDBF8A84ED938AC4ED948AF1
:10BF8000C4F85462C4F804E3DE4633484EF8883FF0
:10BF9000C4F8F4025846CDF838E040F88C3FA64685
:10BFA00011EE103A4EF8A83FCDF83CE0DE462B4F9C
:10BFB0004EF8A43FC4F800730D90274618EE100AFF
:10BFC00018EE903ACDF840E047F8A03FC4F864126C
:10BFD000EB8B4BF89C0FC4F86822A88BC4F87462F2
:10BFE000C4F88412C4F88822C4F8946284ED968A56
:10BFF00084ED978A84ED988A84ED9B8AC4ED9C8AAF
:10C0000084ED9E8A84ED9F8A84EDA08A2AE000BF99
:10C010002870010000BADB4818E400E019E400E0F1
:10C020004AE400E01071FF1F1CE400E051E400E06E
:10C0300027E400E05485FF1F981104008CAAFF1F1D
:10C0400054ADFF1F0000000000F07F45BAE8144225
:10C050000AD7233C87D4843F0000C8416666663F08
:10C060000B95813F84EDA38AC4EDA48A84EDA68A52
:10C0700084EDA78AC4F8A412C4F8B462C4F8C41248
:10C080002E8C698CC4F8A82201EE900A02EE103AB8
:10C0900003EE906A04EE101AF8EE612AB8EE423A06
:10C0A000F8EE634AB8EE445AC4ED702AC4ED6F2A24
:10C0B00084ED793A84ED783AC4F8C82284EDA88AF0
:10C0C000944A84EDAB8AC4EDAC8A84EDAE8A84EDEB
:10C0D000AF8A84EDB08A84EDC28AC4EDC38A84ED50
:10C0E000C58A84EDC48A1E2184EDC68AC4EDC78A40
:10C0F00084EDC98A84EDC88A84EDCA8AC4EDCB8AEE
:10C1000084EDCD8A84EDCC8A84EDCE8AC4EDCF8ACD
:10C1100084EDD18A804884EDD08AC4ED824AC4ED92
:10C12000814A84ED8B5A84ED8A5AFCF785FE794961
:10C13000DFED7AAA9FED7A9ADFED7A9A9FED7AAADF
:10C14000A1F6FC70A0F1540602F020FEAA8D119811
:10C150000299D0F800C00598DFF8E8E1D9F800307E
:10C16000036005EE902ADAF800200A60009AD4F8FD
:10C1700078A0D4F89490D4F8B01082ED008A2046CC
:10C18000069A039CC8F800C0AEF10C0341F21E08E9
:10C19000CEF800A0CEF80490CEF80810B8EE650AEC
:10C1A0004FF0000184ED008A82ED008A05F8081046
:10C1B000D3F800A0DFF8908100F61404A0F54379CD
:10C1C000F5F7D4FDB5F82EC0089A0998C2ED008A9B
:10C1D00006EE10CA0A9A0799544B80ED000AC2F87D
:10C1E00000A0019881ED008AB8EE460AD3F800A0BD
:10C1F000F5F7BCFD6A8D0D9D0C9985ED000A06EEE4
:10C20000902A0B9D0E9A4A4B0498C2F800A085ED27
:10C21000008AB8EE660AC1ED008AD3F800A0F5F7EF
:10C22000A5FDC7ED008A0F98109F80ED000AC7F8A2
:10C2300000A0A8F104058BED008A374697F87B3003
:10C2400015F8011F994240D097F87820A2BB032B24
:10C25000716D54D0002914BFB0EE490AB0EE690ADE
:10C260004846F7F7DFFD97F87B20042A44D02A7070
:10C2700097F87A00287297F878302B71454507F1C6
:10C28000140704F5936409F11009D7D141F2B00500
:10C29000284F725928499668284846F001034FF004
:10C2A00080754FF0805493603D6038600C6017B02B
:10C2B000BDEC068BBDE8F08F97F87A304846B3B9ED
:10C2C000F5F710F997F87B20D1E7287A97F87AB03C
:10C2D0005845B9D195F804A097F878209245B5D182
:10C2E0001749706D91F800C08445AFD1C6E7F5F7E6
:10C2F00019F997F87B20BAE784ED00AAB7E700297F
:10C3000014BFB0EE490AB0EE6A0A4846F7F78AFD54
:10C31000A9E700BF6081FF1FB0C3FF1F00A00C464C
:10C3200000007A4500409C463333733F3881FF1F3D
:10C330003C81FF1F00F0024000E100E0000100909E
:10C34000FCCDFF1F4081FF1F00CEFF1F70B543F6DD
:10C350003003214C214AE05801680D6804F561560C
:10C3600001219542317034D1007903F04BFD43F641
:10C37000300501216059026893689847322003F024
:10C38000A1FD605901688A6800219047322003F0BE
:10C3900099FD605905680121AB689847322003F088
:10C3A00091FD0F48F6F7C0FB606E0E4901EBC00C23
:10C3B00043F6440543F6450143F646029CF8043033
:10C3C00063559CF8050060540125A5540024347081
:10C3D00070BDA847CBE700BF1071FF1F0D13000011
:10C3E0003CA9FF1F500302002DE9F04FDFF8B09386
:10C3F0002DED0A8BD9ED007A41F23C03A3B004463F
:10C40000F5EE407A011DC65C0391543004F27C4283
:10C41000F1EE10FA0590049215D192ED000AB5EEF6
:10C42000400AF1EE10FA0ED0DFF8788304F571526D
:10C43000043200921046211D059A04F58157FBF73E
:10C44000C5FD10370FE0002E00F0B081DFF85483F7
:10C4500098F80070002FE9D004F5715004F5815769
:10C46000043000901037049D41F23C21D5F800A023
:10C470006558C9F800A0286888F80060066895F833
:10C480005A10736801229847294604F5915951F8CA
:10C49000580B026809F11C0AD5680122A847DAF88E
:10C4A0000460306896F85A10036801225D68A84756
:10C4B0003146012251F8580B0668F3689847DAF8BC
:10C4C0004851B5480690002D3BD00494DFF8D8B20F
:10C4D00081460AF168064FF00008044611E06968D9
:10C4E000101A88420BD3002B40F0DE81AB689842D3
:10C4F0004FF0010234BF002001202A756875ED68F5
:10C50000F5B1B54200F0D78129680A685A4540F074
:10C51000C881AB69297F93F8583022682869129244
:10C520000B4103F00103129A0028D8D1002BE6D169
:10C53000D9F80010119111982861ED68002DE0D113
:10C54000049C9AF8DC0004F5925604F5975E96F880
:10C5500018C09EF818900EF1040B04F5935104F5E1
:10C56000945204F5955304F59655043691F81880C5
:10C57000767D92F818E093F818B084F804C004317E
:10C5800095F818C0497D84F80580043204330435D9
:10C590005B7D527D6D7D84F806E084F809909AF801
:10C5A0001CE19AF8FC909AF83CA1E673039EA072F5
:10C5B00004F5615084F808C0A37484F80CE084F892
:10C5C0000B90A573217462743146083084F807B06B
:10C5D00084F80DA0F7F792FA04F580593146059AD0
:10C5E0000098FBF7F3FC04F14D060021D9F8005048
:10C5F00084F848100422304606F0FCFB301BA0F102
:10C60000490204F14803002104F14900079306F0B0
:10C61000F1FB681C01F0068205EB850204EB820A3F
:10C620000AF1780CBCE80F000DF1740EAEE80F00B3
:10C630002544BDF87400DCF80060CEF800604FF0CF
:10C64000010885F84D80002801F0E28141F23C03A9
:10C6500014F803A0A0F580700022B0FA80F67309E8
:10C6600084F8482085F84930BAF1000F00F02A8795
:10C67000256E4FF0010A002D40F024874FF0030C87
:10C6800004F580501C30427884F851C041F21C0EF1
:10C69000002A00F00E8714F80E60002E01F02F82A1
:10C6A0008378002B0CBF0123022384F8523094F8C6
:10C6B000E88F08F1FF3004F57455012805F11805DD
:10C6C00049D929460F22039806F0FEFA626B696B7E
:10C6D000A36B2E6B95ED115AD7ED006A95ED126A9A
:10C6E00097ED017AD5ED135A97ED022A961B5A1A47
:10C6F000AB6BE16B1643C91A0E43236CE96B2A6CD2
:10C7000076EEC52A5B1A37EE463A616CB7EE004A00
:10C71000F0EEE23A72EE654A3343F4EEC43A8E1A12
:10C72000F0EEC39AF1EE10FA43EA0603F4EEC49A6F
:10C73000B0EEE4AAC8BF43F00103F1EE10FAB4EE84
:10C74000C4AAC8BF43F00103F1EE10FAC8BF43F01A
:10C750000103034307D006980268109241F20C0BC4
:10C76000109B44F80B30069904F5815B0E680F9618
:10C770000F98DBF80020831AB3F5FA7FC1F03C81F3
:10C7800006490891B8F1030F01F2D081DFE818F0F3
:10C79000D0046A0132019500B4DE01200431FF1F8C
:10C7A0007430FF1F7830FF1F010F0000DFF8208674
:10C7B00098F80050002D3FF44FAE04F571573946FC
:10C7C000043104F5725C0B697A6BDCF814E0CB6021
:10C7D0004FF0000AC1F814A0C7F838A03A63A78D3B
:10C7E000CCF818A000EE907A04F581571037CCF8F9
:10C7F00010E00D460091DCF83C10396004F5735CE4
:10C8000004F57353DCF818207A60586BB86004F5AF
:10C81000815EB8EE600A28469EED018ADFF8B4B565
:10C82000F5F7A4FAE18D04F5725C01EE101A8CEDB7
:10C830000D0A04F581538CED0C8ACCF828A0CCF8B5
:10C840002CB005F12000B8EE410AD3ED028AF5F7CD
:10C850008DFA628D009504F5735001EE902A04F56F
:10C860008151C0ED038A80ED040AC0F804A0C0F82D
:10C8700008B0B8EE610A05F1400091ED039AF5F7B2
:10C8800075FA04F5735585ED0B0AC5F820A0C5F8B7
:10C8900024B0009885ED0A9A059A211DFBF796FBB6
:10C8A000E1E5284690472AE6C5F8108085F814800F
:10C8B00085F8158023E600BF26E60F222946039857
:10C8C00006F002FA2B6B6A6B616B04921E4695EDC3
:10C8D00011BAD7ED00AA0A93891BAB6B049EA26B19
:10C8E000D7ED01BA099395ED12CAE36BD7ED02CAF1
:10C8F000D5ED137AD5F83CA0D5F84090921B7AEE8E
:10C90000CBAA099E3BEECCBA9E1BF7EE000A114360
:10C91000B0EEEA0A7CEEE7BAB4EEE00A3143B0EEDC
:10C92000CB1A266C626CF1EE10FAF0EEEB1AB4EE54
:10C93000E01ACCBF01230023CAEB0606F1EE10FA81
:10C94000F4EEE01AC8BF43F001033143F1EE10FAF0
:10C95000C9EB0208C8BF43F0010341EA080843EAF3
:10C96000080C5CEA000300F0B48026798EB9607987
:10C9700078B9A3796BB9E17959B9227A4AB9607A61
:10C9800038B9A37A2BB9E17A19B9227B0AB9607B4D
:10C9900018B14FF0010E85F855E005F13008B8E800
:10C9A0000F0004F1340CACE80F000346D8F8000087
:10C9B000A16BE26BCCF800000A98C0EB030E049B5D
:10C9C000206C0490C91A94F8E93F84F8E83F099B69
:10C9D000606CD21A049B4EEA01011143CAEB0303B7
:10C9E0000B43C9EB0008002043EA080885F85C0007
:10C9F000E36D70E043F66D56A15DD9B994F807C0B8
:10CA0000BCF1000F05D143F61B52A35C002B41F093
:10CA10007B86207A70B943F61C56A15D51B141F274
:10CA2000040E41F2040314F80E200132082AD8BF84
:10CA3000D0B2E054D5F84080636CB3EB080601F047
:10CA4000678141F20401635C082B01F2C886DFE8CC
:10CA500013F0BD109D1062103D10F910DD100F1184
:10CA60000810BD0FE179002901F0DC8066791EB95C
:10CA70006878002841F0C38294F8FC2F002A41F026
:10CA80009B872A6BA36B696B606BE66B97ED006A03
:10CA9000D5ED115A97ED012AD5ED122A97ED027ABC
:10CAA00095ED138A801A5A1AAB6B40EA0201F61A06
:10CAB000E86B626C0E43216C0B1A286C46EA03018A
:10CAC000121A76EE65AA32EE62BA77EE48BA42EAF8
:10CAD0000108E36D2679042B28D8B64A52F82320A2
:10CAE00022B3069BB44918680E9041F20C0C0E9BC1
:10CAF00054F80C001B1A9A4218D294F8E8EF0EF181
:10CB0000FF32022A12D908680D9041F2080C41F256
:10CB1000190184F8E9EF01200D9B44F80C304FF027
:10CB2000030E605484F8E8EF85F85C000F22294674
:10CB3000039806F0C9F8F7EE009AF0EEEA4AF4EE30
:10CB4000E94AB0EECBAAF1EE10FAB4EEE9AACCBFF6
:10CB500001220022F1EE10FACCBF01210021F0EEFB
:10CB6000EBAAF4EEE9AA1143F1EE10FA41EA080843
:10CB7000C8BF48F0010858EA000305D108980368C7
:10CB80005A1C0F2B02600ADD97E8070005F14408E4
:10CB900088E8070008994FF0000EC1F800E0AEB930
:10CBA00066799EB9A07988B9E3797BB9227A6AB9A6
:10CBB000617A59B9A67A4EB9E07A38B9237B2BB994
:10CBC000627B1AB943F66D510026665497E8070058
:10CBD00005F1440C8CE807002846039D44222946B1
:10CBE00002F0FCFA04F577502946059A2030F9F74F
:10CBF00049FF04F59C5008300799F5F7FFFB43F611
:10CC00002C00235893F86450BDB941F2190814F868
:10CC10000810002900F07787626E6848032ACCBFAD
:10CC2000FF2100214FF4804206F0E4F804F5BD50E6
:10CC30001030F6F7BFF804F8085045F6E44B04F559
:10CC4000825154F80B601031002E089113DB894695
:10CC5000084641F21E05059902F056F9002304F535
:10CC6000A54031464A4663552030FCF737F84FF06F
:10CC7000FF3044F80B0045F6E84A54F80A10002942
:10CC80007CDB089E04F5A54032462030FCF7D4F842
:10CC90003146059802F07AF804F57258009ED8F8EB
:10CCA00014E0316904F5715C434641F21E09DCF879
:10CCB00034204FF0000B3C33002504F80950F1609C
:10CCC000C6F814B0CCF83020CCF838B004F5735264
:10CCD000C8F810E0C8F818B01868B4F82CC038606C
:10CCE000183204F57359116879600BEE10CAD9F83F
:10CCF0003450BD6004F5815E3046B8EE4B0ADEF874
:10CD00000470DFF8D080F5F731F8E28D04F5725346
:10CD10000BEE902A04F5815C83ED0D0A1F63C3F8C6
:10CD200028B0C3F82C8006F12000B8EE6B0ADCF8BE
:10CD30000850F5F71BF8618D04F573590CEE101AC5
:10CD400006F1400004F5815689ED040AC9F80C503B
:10CD5000C9F804B0C9F80880B8EE4C0AF568F5F7D0
:10CD600005F804F573534FF0FF3283ED0B0AC3F857
:10CD700020B0C3F824809D6244F80A2045F6EC47B1
:10CD8000616DE65D8E4200F0CD8004F5884A04F5C1
:10CD90006456DFF844B09FED0A9ADFED0ACADFED72
:10CDA0000A8A0AF158083836A24604F15009074F9A
:10CDB000642559E060010200B4DE01200831FF1F44
:10CDC00000A00C4600007A4500409C461071FF1FF1
:10CDD0007830FF1F00F07F453333733F9AF87B00B4
:10CDE000796D032800F02A83002914BFB0EE6C0A85
:10CDF000B0EE680A3046F7F715F89AF87B30042B46
:10CE000000F019839AF87820013D002A3DD19AF864
:10CE10007B00032800F01C837A6D002A14BFB0EE5B
:10CE20006C0AB0EE680A3046F6F7FCFF9AF87B1001
:10CE3000042900F0F2829AF8780090B39AF87A30D8
:10CE40003046002B00F0E682F4F76CFB9AF878206D
:10CE5000002A3FD09AF87A103046002900F0D1829B
:10CE6000F4F760FB033D4CD09AF87830002BB5D036
:10CE70009AF87A203046002A40F0C682F4F732FB56
:10CE80009AF87820013D002AC1D09AF87A103046ED
:10CE9000002900F0BC82F4F745FB9AF878000028DE
:10CEA000CCD19AF87B20032A00F0DD82786D00282F
:10CEB00014BFB0EE6C0AB0EE680A3046F6F7B2FF67
:10CEC0009AF87B30042BC1D19AF87820C8F800B0CA
:10CED000002ABFD19AF87B00032800F0A1827A6D66
:10CEE000002A14BFB0EE6C0AB0EE680A3046F6F7BE
:10CEF00099FF9AF87B100429B4D1033DC8F800B01B
:10CF0000B2D10AF1140ACA4508F5936806F1100671
:10CF10007FF44DAF606D45F6EC4E031C18BF012346
:10CF200004F80E3004F5884204F584465432203665
:10CF3000A24600270396A3460497D046914607943D
:10CF4000079C98F8785094ED168AD4ED1A8A94EDDF
:10CF50001B9A0AF57F560C36002D40F08F829BF805
:10CF60008034002B40F0BE820AF583450AF58446E2
:10CF70000AF5884E039C634A6A650120AC653061FE
:10CF8000DEF83430604F614D9FED614ADFED614A5C
:10CF90009FED617A9FED610ADFED610A614ADFED85
:10CFA0005D5A9FED612ADFED612A07FB03F31D4403
:10CFB000C5F30E4107EE901AB8EEE71ACEF83450DA
:10CFC00061EE041A0BF27C4CA1EEA47A0AF58440BF
:10CFD00004469CED005A99ED006A77EE056AA6EECC
:10CFE000806AB4EEE06AF1EE10FAA8BF36EE606A2D
:10CFF000BDEEC6CA89ED006A1CEE106A02EB860E11
:10D000009EED003AF1EE43BAABEEA52AEBEEA52A6F
:10D0100080ED022AC4ED032A0BF26C430AF5834526
:10D020001F6898F87B30EF670BF274410AF5844C67
:10D030000E68CCF804600BF264420AF58340D2F823
:10D0400000E0C0F878E00AF584449BF86274277524
:10D050000BF58A650AF583462968F1650BF2544C95
:10D060000AF58340DCF80040039D4466A3F101000B
:10D070000AF5844E05F59361B3FA83F6B0FA80F5AC
:10D08000049F039174096909A3F10306A3F1020542
:10D09000A3F104038EF816408EF81710B6FA86F442
:10D0A00001377246B5FA85F1B3FA83F30AF5834C7A
:10D0B00060094E095C09042F8EF818008EF819607B
:10D0C0000497947609F593690BF5727B08F11408BF
:10D0D0008CED1A8A0AF5936ACCED1B8A8CED1C9AAA
:10D0E0007FF42EAF05990898079F01F07FFE18B1D5
:10D0F00041F21E0001253D5423B0BDEC0A8BBDE872
:10D10000F08F00BF40CEFF1FFD430300C39E2600EB
:10D1100080008037CDCCCC3D8FC2753D6F128341EE
:10D120000000804610DC00200000FE4233334B41FB
:10D13000A67A2EB9A87918B12A6D002A01F0378491
:10D1400094F80BC0BCF1000F07D1EB792BB1286D1F
:10D15000012804BF4FF0FF30286594F80C80B8F127
:10D16000000F07D12A7A2AB1296D022904BF4FF096
:10D17000FF312965637B1A463BB9687A28B1296D6E
:10D18000032904BF4FF0FF31296595F8C40000283A
:10D1900040F0DB8594F806E0236ECDF810E0714690
:10D1A0000993002900F0C087637A002B40F0C08704
:10D1B0006979002941F0048443F66D53E35C94F8E7
:10D1C00078E0BEF1000F04D194F87900B0FA80F055
:10D1D000400994F88CE0BEF1000F05D194F88DE081
:10D1E000BEF1000F08BF012094F8A0E0BEF1000FCF
:10D1F00040F0A18694F8A1E0BEF1000F40F09B86BC
:10D20000002B40F0AB85099B002B41F0538141B1CD
:10D210006B7933B9049921B9069803681593159968
:10D22000A965D9F80030A979002E41F02F8159B1B4
:10D2300095F8540028B9002B01F0AD83C9F80060BF
:10D240003346002685F85460E979BCF1000F41F0BF
:10D25000B28261B195F8540030B9012B14BF01239B
:10D260004FF0FF33C9F80030002685F85460287A63
:10D27000B8F1000F41F0AF8068B195F8546036B94D
:10D28000022B14BF02234FF0FF33C9F800304FF0D8
:10D29000000C85F854C0002A01F08A80697A89B9A7
:10D2A0002A6D002AC1F25A83032A01F05783C4F879
:10D2B000EC2F032601224FF0FF31C4F8F06F84F801
:10D2C000E82F296594F80780B8F1000F00F04F8728
:10D2D000E878002840F04B8794F805C0BCF1000FB7
:10D2E0000AD041F23C0200204FF0020E0121A0546E
:10D2F00084F8E8EF85F85510591C01F03C80227A3B
:10D30000002A40F044872E7906B3A87A002841F01D
:10D3100043809E00F01804EB800E9EF87B100429D9
:10D3200001F00A839EF87800002841F0FE829EF802
:10D3300079004FF47276B0FA80F106FB0346480993
:10D340008EF879004FF0010E86F861E4A17B002988
:10D3500001F02880A87A0A4680B903EB830E04EB1B
:10D360008E0696F87B10042901F0F28232B196F80D
:10D370007820B2FA82F0410986F87810296D4A1CAB
:10D3800000F0B087E37B002B00F00887EA7A82B9CF
:10D3900095F8C2606EB941F21D01635C002B01F08B
:10D3A000A68241F21C0E14F80E1081F0010304F85D
:10D3B0000E30296D4E1C40F0F186049A26792AB968
:10D3C000A87818B14FF0000E85F8C0E0B8F1000F52
:10D3D00003D1EB78002B40F08087BCF1000F03D124
:10D3E000697809B185F8C3C0002E40F0B88443F6CF
:10D3F0001850235C002B00F0B28485F8C26000F066
:10D40000AEBCF4F76FF82DE5F4F78CF8FAE4F4F716
:10D4100069F810E5F4F766F818E5C8F800B00AE511
:10D420007B6D002B14BFB0EE6C0AB0EE490A30469B
:10D43000F6F7F8FC5DE5C8F800B0E3E4002914BF96
:10D44000B0EE6C0AB0EE490A3046F6F7EBFCD4E4D5
:10D450007B6D002B14BFB0EE6C0AB0EE490A30466B
:10D46000F6F7E0FCE2E4796D002914BFB0EE6C0A37
:10D47000B0EE490A3046F6F7D5FC21E50AF5834EB1
:10D4800098F87A00114B124ACEF854200AF58445D8
:10D490000AF5834CDFED0F7A9FED0F0A53F82070E9
:10D4A000CCF8587000212961C5ED027A85ED030A98
:10D4B000B2E5817800290CBF0021022184F85210C6
:10D4C000FFF7F5B8D446FFF7DBB800BF8022FF1F97
:10D4D00010DC002000000043000000000AD7233CBD
:10D4E0000AD7A33C642001F03FFE069A5FED059A3F
:10D4F00017681C9700EE900AB8EE601A5FED081AE4
:10D500001C9CE34821EE295AE5EE219A14B90568DE
:10D510001D951D9C9FEDE3CADFEDDECA0AF5834E23
:10D520002046CEF8504005F0B7FC3046F8F7C0FC76
:10D53000049B079A0398CDF824A00AF58341F5EEE1
:10D54000C09A4FF493664C31F1EE10FA06FB0327B4
:10D55000C8BFC1ED009ACDF82880CDF82CB00025C9
:10D56000F1EE08BABAEE0EBAF2EE04AAB5EE00AACF
:10D57000F7EE009A80468A46BB4606EE905A9AED30
:10D58000006AF8EEE65A013525EE862A12EE100AF8
:10D5900004F02AFF06460F4647EC106B04F030FDFE
:10D5A00053EC102B10EE100A1946CDE9002304F0BD
:10D5B000F7FFDDE90023C4B23946304604F0B4FD7C
:10D5C0005C4405F035F804F57F5102EE900A0E7BBD
:10D5D0004F7B06F0030304EE103A07F00302F8EE67
:10D5E000C47A05EE102AB0EE4B3AF0EE690AA2EECC
:10D5F000AB3A3407E7EE8A0AB8EEC56AF0EE695A2C
:10D60000E6EE0A5AF0EE6A3AB0EE601A72EEE96A95
:10D61000E2EE833A62EEA24A4CBF20EEE21A22EE1C
:10D62000811A380724EEA20A4CBF65EEE66A66EE60
:10D63000A56A60EE231A76EEC12AA1EEA21AB4EE14
:10D64000EC1AF1EE10FAB4EE4C1AD8BFF0EE41CA63
:10D65000F1EE10FAC8BFB0EE41CA802DA8EC011A55
:10D660008BD1039DDFED8CAAD5ED00BADDF824A0A7
:10D67000DFED8A3ADDF82880DDF82CB03BEEECBA1D
:10D680003CEE6CCA2BEE2AAA0AF58840CAEE0C9A28
:10D690002C462030411B0E1FC6F3810339EEE37A7E
:10D6A000A4EC017A84427AD0ABB3012B21D0022BB7
:10D6B0000FD094ED004ADFED787A9FED781A74EE82
:10D6C0006C4A24EEA70AC0EE0C0A70EEC11AE4EC14
:10D6D000011A94ED005ADFED706ADFED702A35EE25
:10D6E0006C6A66EE265A85EE8C2A32EE623AA4EC1B
:10D6F000013AD4ED00BADFED68AADFED683A3BEEFF
:10D70000ECBA2BEE2AAACAEE0C9A39EEE37AA4EC14
:10D71000017A844243D094ED004ADFED5F7A9FEDB9
:10D720005F1ADFED5D6ADFED5D2ADFED5BAADFEDFD
:10D730005B3A74EE6C4AA64624EEA70ADFED567AF1
:10D74000C0EE0C0A103470EEC11A9FED541AEEECC4
:10D75000011A14ED035A35EE6C6A66EE265A85EE10
:10D760008C2A32EE623A04ED033ADEED01BA3BEE6A
:10D77000ECBA2BEE2AAACAEE0C9A39EEE37A8EEDB9
:10D78000017A14ED014A74EE6C4A24EEA70AC0EE49
:10D790000C0A70EEC11A44ED011A8442BBD1039DFC
:10D7A0009FED3FCA0AF5884C00222E46CCF828206F
:10D7B000CCF82C20F6EC01CA2CEE8C5A411BBDEEA5
:10D7C000C56A0B1F8DED006ABDF90070CBF8C870FB
:10D7D0008642C3F382050BF1C80E00F0D980002DFC
:10D7E00072D0012D62D0022D45D0032D37D0042DEB
:10D7F00029D0052D1BD0062D0DD0F6EC016A66EE62
:10D800008C5A0BF1CC0EBDEEE52A8DED002ABDF948
:10D810000020CBF8CC20F6EC012A22EE8C3AFDEE6B
:10D82000C3BACDED00BABDF900404EF8044FB6ECD6
:10D8300001BA6BEE0CAABDEEEAAA8DED00AABDF905
:10D8400000104EF8041FF6EC019A69EE8C3ABDEE1A
:10D85000E37A8DED007ABDF900304EF8043FB6EC66
:10D86000014A64EE0C4AFDEEE47ACDED007ABDF992
:10D8700000704EF8047FB6EC010A60EE0C0ABDEEB3
:10D88000E01A8DED001ABDF900504EF8045F0DE06E
:10D89000B4DE0120FFFF7F7F6666E63F6666663F77
:10D8A00000FEFF460000000000F07F45F6EC011A84
:10D8B00061EE8CCA8642BDEEEC5A8DED005ABDF980
:10D8C00000204EF8042F63D0B446BCEC016A66EE2B
:10D8D0000C6A2036FDEEE65ACDED005ABDF9004047
:10D8E000CEF8044016ED072A62EE0C2ABDEEE23AAD
:10D8F0008DED003ABDF90010CEF80810DCED01BA4C
:10D900002BEE8CBAFDEECBAACDED00AABDF900300E
:10D91000CEF80C3016ED05AA6AEE0C9AFDEEE93A47
:10D92000CDED003ABDF90070CEF8107016ED047A16
:10D9300027EE0C4AFDEEC44ACDED004ABDF9005079
:10D94000CEF8145056ED037A27EE8C0AFDEEC00A8D
:10D95000CDED000ABDF90020CEF8182016ED021A10
:10D9600061EE0C1AFDEEE1CACDED00CABDF9004032
:10D97000CEF81C4016ED015A25EE0C6A8642FDEEEB
:10D98000C66ACDED006ABDF900104EF8201F9BD18C
:10D990001FED3CCA1FED3C2A00200BF24C46CBF891
:10D9A00048040AF5884E86ED00CADEED075AF7EE08
:10D9B000002A35EEA23AF6EE00BA23EE02BA0127AB
:10D9C0006BEE2BAA0BF2844CBCEEEAAA8DED00AAFA
:10D9D000BDF8003009EE903AF8EE693ACCED003A25
:10D9E0008BF888048BF880048BF860748BF8617472
:10D9F0008BF88174FFF7B8BA97E80700C04E089615
:10DA000005F1440C8CE8070000223260FEF7BABE34
:10DA100041F23C0B14F80B10002900F0B880C2460C
:10DA2000FEF718BE41F23C0104F1780814F801A099
:10DA3000B8E80F000DF1740BABE80F00D8F8002028
:10DA4000BDF87460CBF80020BAF1000F40F0A5805B
:10DA5000B6F5807F00F09E8684F849A01EB94FF08D
:10DA6000010E84F848E004F18C0BBBE80F001DAEFA
:10DA70000FC6BDF87430DBF800103160B3F5807F5D
:10DA800000F08386002584F84A5013B9012284F8F7
:10DA9000482004F1A00CBCE80F000DF1740EAEE8B4
:10DAA0000F00BDF87460DCF80030CEF80030B6F539
:10DAB000807F00F06586002184F84B1016B901259F
:10DAC00084F8485004F1B408B8E80F000DF1740B65
:10DAD000ABE80F00BDF87400D8F80060CBF8006028
:10DAE000B0F5807F00F04786002384F84C3010B9F1
:10DAF000012184F848104FF0000CFEF7C1BD84F8F6
:10DB00005260FEF7D4BD4FF480427E4805F072F9B2
:10DB100094F8E83F04F574501430032B00F2D984D4
:10DB2000DFE813F0D30105020102BE0140F23332F7
:10DB300075497648F3F7A0FE2A6BA36B696B606B9F
:10DB4000E66BD7ED002A95ED113AD7ED013A95ED48
:10DB5000127A97ED024A95ED138A801A5A1AAB6B26
:10DB6000616C1043F61A0643EB6B206CC21A2B6CE7
:10DB700046EA0200C91A72EEC3AA33EEC7BA74EEBF
:10DB800048BAE36D267940EA0108FEF7A4BF8A4649
:10DB900084F848800B46FEF765BD04F18C0CBCE8A8
:10DBA0000F000DF1740EAEE80F0004F1A00ADCF8CE
:10DBB0000000CEF80000BAE80F000DF17408BDF8BF
:10DBC0007450A8E80F00B6F5807FBDF87430DAF81D
:10DBD0000010C8F800100CBF01260026B5F5807FA4
:10DBE0000CBF01250025B3F5807F0CBF0123002366
:10DBF00004F1B40B84F84B30BBE80F0084F84960A3
:10DC00001DAE84F84A500FC6BDF87450DBF80020F2
:10DC10003260B5F5807F00F0C885002084F84C00A4
:10DC2000FEF726BDEB78002B3EF420AFD4F8EC1FB6
:10DC3000069BD4F8F06F1868199001EB810204EB91
:10DC4000820E0EF1780CBCE80F0006EB860804EBA0
:10DC5000880678360FC61999DCF800303360012049
:10DC6000C4F8F41F84F8FC0F39B1069A16681796A9
:10DC7000179B591AB1F5C87F0DD8D4F8F80F0028B2
:10DC80003EF4FFAE069A16681696169B191AB1F561
:10DC9000C87F7EF6F6AE2A6B696BA36B606BE66B92
:10DCA00097ED003AD5ED113A97ED014AD5ED124ABC
:10DCB000D7ED029A95ED13AA801A5A1AAB6B40EA77
:10DCC0000201F61AE86B626C0E43216C0B1A286C89
:10DCD00000211E43121A46EA020873EE63AA34EECC
:10DCE00064BA79EECABA84F8FC1FC4F8F41FC4F809
:10DCF000F81F84F8E81FE36D2679FEF7ECBE00BF3D
:10DD00000431FF1F0831FF1F40BC0100E8BD0100C6
:10DD10002A6BA36B696B606BE66B97ED006AD5EDC0
:10DD2000115A97ED012AD5ED122A97ED027A95ED59
:10DD3000138A801A5A1AAB6B40EA0201E86B226C14
:10DD4000F61A3143121AFEF7BCBE002643F66D5296
:10DD500085F8C460A35C002B00F0DA812679D9F83D
:10DD60000030581C00F0A681616B2A6BB1EB020CED
:10DD700040F057814FEA830808EB030904EB890C54
:10DD800043F658529CF87800A258616C002840F085
:10DD9000E28004208646B1EB02090ED0059A08EB1A
:10DDA000030C02EB8C012431CA784A44724500F31B
:10DDB0009783002A80F2F885C87008EB030104EB12
:10DDC000810EBEF878C0BCF5807F04D0206CEA6B71
:10DDD000821A40F0AD83E16BAA6B8A1A40F0888307
:10DDE000A06B696BB0EB010C40F0DE80606B2B6BBD
:10DDF000E046C3EB000C216E002940F0AF8043F6F3
:10DE0000705E04F5755054F80E2090ED09CAD7EDF8
:10DE100002CA531C00F0C4847CEECCBAF7EE007A40
:10DE2000B0EEEB0AB4EEE70AF1EE10FA05DD069A61
:10DE300013681493149A44F80E20069908681390F6
:10DE4000139B40F2DC5E991A714540F2E48043F680
:10DE500070504FF0FF3222504FF0000EA86B236C31
:10DE6000E96BE26BD7ED000A95ED111AD7ED011AB7
:10DE7000D5ED128A121A581A636C296C10435A1A7B
:10DE8000024341F23C0042EA0C0343EA080804F86A
:10DE900000E070EEC1AA31EEE8BAE36DFEF71BBEFA
:10DEA000069ADBF8008011681B911B9EC8EB060EDA
:10DEB000BEF5FA7F80F0CD8394F8E93F002B40F067
:10DEC000C88341F21801012666540599F6F774FEDD
:10DED00094F8E85F032D00F0708304F560554FF46B
:10DEE0000056EE632C3528461521F4F7C5FD28466B
:10DEF0000021F4F7C1FD28463F21F4F7BDFD284677
:10DF00007521F4F7B9FD28460021F4F7B5FD04F5B5
:10DF1000BD5628467F211036F4F7AEFD3046F4F7A3
:10DF200049FFFEF78ABE0599F7F7D6FDD0E70599B8
:10DF3000F7F792F9CCE794F8B4E0BEF1000F05D101
:10DF400094F8B5E0BEF1000F3FF45AA900283FF461
:10DF500002AFFFF755B9032086461CE7A86B236C78
:10DF6000E96BE26B97ED025A97ED006AD5ED116A05
:10DF700097ED019AD5ED125A121A581A636C296C52
:10DF8000024304F5755E581A02439EED092AE36DBB
:10DF900042EA0C0242EA080875EE42BA76EE66AA38
:10DFA00039EE65BAFEF797BD6279002A00F0E18389
:10DFB00043F6DB5001210CEB8C02215402FA01FEE6
:10DFC000984404EB8800D0F884107144622900F36F
:10DFD000C98311F1620FC0F2BD831433C0F88410FD
:10DFE00045F83310002940F0DC84002005EBC30322
:10DFF000626B1871296BE046C1EB020CFBE6069BD5
:10E00000D4F8F41F1E6818961898C4F8F80F012267
:10E0100084F8FC2F28E612F1010E18BF4FF0010E14
:10E020001CE705992A6D03EB8300830001EB0308CD
:10E03000511C08F1340846D12344002E00F0E3813E
:10E04000D3F8881000292FDBB1F5007F40F39A84C4
:10E05000B1F5806F40F39184B1F5C06F40F39684C1
:10E06000B1F5006FC0F2848440F2FE7291421BDD74
:10E07000B1F5206FC0F2F68340F6FE13994213DD2E
:10E08000B1F5406FC0F2E98340F6FE3081420BDD0E
:10E09000B1F5606FC0F2DC8340F6FE5E714503DDD2
:10E0A000B1F5805FC0F2B8834FF0000C012085F815
:10E0B000C20012E02A6D511C21D0616B2B6BB1EBB9
:10E0C000030C00F04F8402EB8208059A012002EB5A
:10E0D000880E0EF1340885F85400D8F8001040F688
:10E0E000FE738C449C45D4BF2CEAEC7340F6FF735E
:10E0F000C8F80030D9F800305A1C7FF43BAE606B92
:10E10000296BA26B6B6BC1EB000CC3EB020872E6D0
:10E1100094F80DE0A079A67A94F80BC094F80C80DE
:10E1200004907246FFF77DB8617A00293FF444A855
:10E13000697900297FF440A82B6D591C00F0D28129
:10E1400003EB830E04EB8E0191F87810002940F068
:10E15000C9814FF4727E0EFB03414FF0010E81F82E
:10E1600080E4734685F855E07146FFF728B894F8C7
:10E1700005C0BCF1000F3FF4BFA86E78002E7FF4FD
:10E18000BBA8B8F1000F3FF4B7A8FFF7AAB8A27B6D
:10E19000002A3FF4F3A8A87AFFF7DEB82679E6B99B
:10E1A00043F61850235CC3B1EA7AB2B901EB81009F
:10E1B00004EB800E0120DEF88830C4F88830DEF8E9
:10E1C0008820C4F89C20DEF88830C4F8B030DEF82F
:10E1D0008820C4F8C42085F85400BCF1000F1AD17F
:10E1E0006878C0B12B7BB3B901EB810204EB820EDE
:10E1F0000120DEF88430C4F88430DEF88420C4F8CE
:10E200009820DEF88430C4F8AC30DEF88420C4F8FE
:10E21000C02085F854000498002840F0B280AB7804
:10E22000C3B16A7BB2B901EB810004EB800E01201F
:10E23000DEF88030C4F88030DEF88020C4F8942006
:10E24000DEF88030C4F8A830DEF88020C4F8BC20A6
:10E2500085F85400B8F1000F7FF4B2A8E8780028E0
:10E2600000F09480AB7BA3BBB4F87820B2F5807F3C
:10E2700006D001EB810004EB800EDEF87C30E36712
:10E28000B4F88C20B2F5807F07D001EB810004EB5D
:10E29000800EDEF87C30C4F89030B4F8A020B2F5DF
:10E2A000807F07D001EB810004EB800EDEF87C302C
:10E2B000C4F8A430B4F8B420B2F5807F06D001EBE6
:10E2C000810104EB8100C36FC4F8B830012285F8E6
:10E2D0005420049900293FF473A8002285F8C12036
:10E2E000FFF77BB8B8F1000F10D1E87870B1AE7BC2
:10E2F00066B995F8C1204AB903EB830E04EB8E0191
:10E30000C86F002840F0C9826322CA67BCF1000FC1
:10E3100014D1697891B12E7B86B995F8C30068B99C
:10E320004FEA830E0EEB030204EB8201D1F8846006
:10E33000002E40F0A6826322C1F88420049AD2B94C
:10E34000A978C1B16E7BB6B995F8C00098B94FEA0B
:10E35000830A0AEB030104EB8100D0F88010002946
:10E3600000F0E182632900F0C9821146534404EBB6
:10E370008303C3F88010E07B00283FF41AA8FFF75E
:10E3800005B8B8F1000F7FF428A867E704990029C1
:10E390007FF423A8FFF714B8A17B00293FF4FBAE5C
:10E3A000FEF7ECBF2E79002E7FF4F5AEFEF7E6BF48
:10E3B0006A7A002A3EF486AF95F8540030B9032BF0
:10E3C0000CBF4FF0FF330323C9F80030002685F857
:10E3D0005460FEF777BF00287EF45DAF296D0029F9
:10E3E000C0F24B82022900F04882C4F8EC1F0226DA
:10E3F0004FF001084FF0FF31C4F8F06F84F8E88F58
:10E400002965FEF748BFDFF83CE4D3F888000EF139
:10E41000E00A2EE01168884202DB5368984231DD41
:10E420005168884202DB936898422BDD91688842EC
:10E4300002DBD368984225DDD168884202DB13698C
:10E4400098421FDD1169884202DB5369984219DD49
:10E450005169884202DB9369984213DD91698842D1
:10E4600002F11C0E02DBD36998420BDDF24500F08D
:10E470000182724652F8041B8842CBDBDEF804307E
:10E480009842C7DC581A0CFB00FC26E600297EF4F3
:10E49000DBAE286D002840F3EA814FF0010E4FF00B
:10E4A000FF36C4F8EC0FC4F8F01F84F8E8EF2E65CF
:10E4B000FEF7CABE00297EF4B4AE697900293EF4A5
:10E4C000B0AE41F23C008AF0010A04F800A0FEF769
:10E4D000A8BE40F2D712D649D648F3F7CDF9F7E4F3
:10E4E000002069E443F66D530121E35CFEF767BE4B
:10E4F000A07938B143F6D85E012102EB820204F81C
:10E500000E108A4008EB030C04EB8C00D0F880104E
:10E510000A44622A4EDC002A40DC03F10C0E002182
:10E52000C0F8801045F83E1005EBCE02117157E49B
:10E53000E17939B143F6D95E012002EB820204F899
:10E540000E00824008EB030104EB810CDCF87C0038
:10E550000244622A1ADC12F1620F0EDB03F1100E84
:10E56000CCF87C2045F83E20002A40F06F81002046
:10E5700005EBCE0C8CF804002DE403F1100E6FF0C7
:10E580006201CCF87C1045F83E10F0E703F1100E64
:10E590006322CCF87C2045F83E20E8E7012108EB17
:10E5A000030E04EB8E0C03F10C0ECCF8802045F822
:10E5B0003E20B9E700216322F1E7DBF800800698EE
:10E5C00003680C930C9AC8EB0201B1F5FA7F7FF651
:10E5D00084AC41F21400235833B141F2180214F80C
:10E5E00002A0BAF1000F68D0656E93484FF48042E4
:10E5F000032DCCBFFF21002104F5605604F0FAFB87
:10E600004FF40050F0632C3630461521F4F734FAFD
:10E6100030460021F4F730FA30463F21F4F72CFA67
:10E6200030467521F4F728FA04F5BD55304600212F
:10E63000F4F722FA103530467F21F4F71DFA41F243
:10E6400018082846F4F7B6FB002304F80830FEF754
:10E65000F4BA069D606E2A681A9241F208010428F5
:10E66000754E63581A9DB4BF4FF000094FF0FF0973
:10E6700049464FF080023046A5EB0305B4BF4FF08A
:10E68000FF0A4FF0000A04F0B5FB4946802206F16C
:10E69000800004F0AFFB6948A0FB053BCBF3860389
:10E6A00041F2100941F2140CCBF3462206F803A004
:10E6B00044F8092044F80C3081E741F2100104F5D8
:10E6C0006055665C701CC3B29A1B9101E9632C35DE
:10E6D00028461521F4F7D0F951462846F4F7CCF92D
:10E6E00028463F21F4F7C8F928467521F4F7C4F904
:10E6F00031462846F4F7C0F93146284604F5BD56A0
:10E700001036F4F7B9F909E4DFF83C814C4E84F88F
:10E71000E8CFB8E80F000FC6B8E80F000FC6D8F86A
:10E7200000103160A6F12C026146A2F134000123F1
:10E73000FAF734FA04F1C80C04F6E87084453EF4A4
:10E7400079A901228CF899230CF5727C6045F9D1E6
:10E75000FEF770B914336FF06201C0F8841045F809
:10E76000331042E414336322C0F8842045F8332088
:10E770003BE4E64624E4012584F84C50FFF7BBB99E
:10E78000012284F84B20FFF79DB9012084F84A004C
:10E79000FFF77FB94FF0010884F84980FFF763B9AC
:10E7A0008E467CEECCBAFFF759BB4FF0010C84F8D3
:10E7B0004CC0FDF75DBF00297EF459AD296D0029DD
:10E7C00032DB012930D00126C4F8EC1F4FF0FF31B5
:10E7D000C4F8F06F84F8E86F2965FEF748BD286B30
:10E7E000626B696BA36B97ED006AD5ED115A97EDDB
:10E7F000012AD5ED122A97ED027A95ED138A121AA5
:10E800005B1A1643A86BE26BE96B1E43236C121A6A
:10E810003243591AFEF755B940F6FF7140F6FF52E0
:10E820008B1A0CFB03FC41E401202865FEF71FBD99
:10E83000A803020018BE01000831FF1F4FECC44EB0
:10E84000F0C3FF1F78BE01006471FF1F01208FE637
:10E8500040F6FF5140F6FF32E2E740F6FF3140F666
:10E86000FF12DDE740F6FF1140F2FF72D8E729659D
:10E87000FEF7EABC4FF0000C2FE402202865FEF7FB
:10E880000ABD632E1DD016F163000DD09E4404EB2B
:10E890008E010020C1F8840050E5632823D0633046
:10E8A00014D00022CA6731E504EBC30043F6BC5222
:10E8B000865C002EEAD043F6B8528658C1F88460D0
:10E8C0003CE56FF06200C1F8840037E504EBC30259
:10E8D00043F69C56905D0028E3D043F6985E52F8CC
:10E8E0000E60CE6712E56FF06200C8670EE5D24A8F
:10E8F00045F6E4461E209051FEF75BBD04EBC306CF
:10E9000043F67C5E16F80EE0BEF1000F3FF42DAD2D
:10E9100043F67852B658C0F88060622E3FF726ADB5
:10E9200026EAE67122E5632120E59EF87A10B1FA25
:10E9300081F041098EF87A10A07B00283FF42BACBF
:10E94000F21804EB820696F87B1004297EF40FADD2
:10E95000B94E042286F84820FEF710BD0320286532
:10E96000FEF7B0BCA16B6A6BC2EB0108FFF743BABC
:10E9700040F2FF714FF4C06252E74FF480614FF4F0
:10E9800000724DE74FF40071002249E74FF4C06177
:10E990004FF4806244E74FF0FF33C9F80030FEF7D0
:10E9A00050BC0120FFF722BBD0B2FFF705BA4FF0F1
:10E9B000FF312965FEF7C4BBD4F8F41FFFF754B943
:10E9C000FDF7C4FC95F85530FFF7C5B9606E3044CB
:10E9D000062800F36381994A20EAE07602EBC60E2E
:10E9E000B4469EF80430DFF850E2666643F6440110
:10E9F00002EBCC000EF8013090F805C0666BA06BFE
:10EA00002B6B6A6BD7ED008A97ED019A97ED026A3E
:10EA100095ED115AD5ED126A95ED138A821A43F6D7
:10EA20004501F61A1643AB6BE26B0EF801C043F6D4
:10EA3000460C0121D21AE86B236C0EF80C10616CA5
:10EA400032431E1A1643C8EB010246EA0208E36D80
:10EA5000267978EEC5AA39EE66BA76EE48BAFEF7A0
:10EA60003AB8E06D626BD7ED005A95ED112AD7EDFB
:10EA7000012A95ED127A97ED023AD5ED133A30441A
:10EA80000428CABF052320EAE0701846E065296B18
:10EA9000A2EB010146EA0106D8BF0346696BA06BF1
:10EAA000E26B401A216C0491A96B0643521A32435F
:10EAB000E86B049E301A42EA000875EEC2AA32EEF4
:10EAC000C7BA73EE63BA2679FEF705B8206E626B9B
:10EAD000A36B97ED006AD5ED115A97ED012AD5ED9C
:10EAE000122A97ED027A95ED138A30440028D4BF9C
:10EAF000002001202066296B686B521A1B1A1643EE
:10EB0000A96BE26BE86B1E43236C511A46EA0102C3
:10EB1000191AFDF7D6BF04EE106ADFED499A94ED9D
:10EB20001BAAF8EEC44AB1EE04BAA4EEA9AAB4EE48
:10EB3000CBAAF1EE10FA08D5B7EE00BAB4EECBAA24
:10EB4000F1EE10FAC8BFB0EE4ABA606BA26B2B6B45
:10EB500084ED1BBA696B97ED006AD5ED115A97EDFC
:10EB6000012AD5ED122A97ED027A95ED138AC01A83
:10EB700040EA0608E36B206C561AAA6B48EA0601C5
:10EB8000EE6B9B1A1943821BFDF79BBF0BEE906A3D
:10EB9000DFED2BCAD4ED1A7AB8EEEBCAF1EE040A17
:10EBA000ECEE2C7AF4EEE07AF1EE10FA08D5F7EEFE
:10EBB000000AF4EEE07AF1EE10FAC8BFF0EE670A50
:10EBC0002B6B606BA26BC4ED1A0AC3E701EE106AEF
:10EBD000DFED1B8A94ED165AF8EEC11AF1EE046AC5
:10EBE000A1EEA85AB4EEE65AF1EE10FA08D5F7EE07
:10EBF000006AB4EEE65AF1EE10FAC8BFF0EE456ACC
:10EC00002B6B606BA26BC4ED166AA3E7606F97ED88
:10EC1000006AD5ED115A97ED012AD5ED122A97ED2C
:10EC2000027A95ED138A626BA36B30440028D4BF3F
:10EC30000020012060675EE71071FF1F5003020093
:10EC4000CDCCCC3D216F97ED006AD5ED115A97EDF3
:10EC5000012AD5ED122A97ED027A95ED138A626B9F
:10EC6000A36B31440029D4BF00210121216742E771
:10EC7000616D97ED006AD5ED115A97ED012AD5ED3A
:10EC8000122A97ED027A95ED138A626BA36B3144D9
:10EC90000029D4BF0021012161652CE74FF0070C4A
:10ECA000014A66465F239EE65003020008B502480B
:10ECB000FDF79AFB08BD00BF1071FF1F70B50E4B2A
:10ECC0000E4C0022802120460126FF251A605A6042
:10ECD000DA601A61DE621D729A621A755A759A615B
:10ECE000DA6119625962FAF763FF2046044A05495E
:10ECF000BDE8704003F07EB910CEFF1F1071FF1FFA
:10ED00007822FF1F9D12000010B54FF400742246B8
:10ED10000749084800F062FA22460749074800F010
:10ED20005DFA22460649074800F058FA10BD00BFB8
:10ED3000980B040040D20020980D040040D0002021
:10ED4000980F040040CE002010B54FF480342246C6
:10ED50000449054800F042FA22460449044800F0FC
:10ED60003DFA10BDC803020010DC0020C8030300F8
:10ED700040CEFF1F08B54FF4FA620249024800F086
:10ED80002DFA08BDC803040040D40020F0B50D469C
:10ED900086460C460FCD0EF124060FC604F114076B
:10EDA0000FCF2D6835600EF1380C04F12806ACE861
:10EDB0000F000FCE3F68CCF800700EF14C050FC568
:10EDC00004F13C0C33682B60BCE80F000EF16006C8
:10EDD0000FC6503494E807000EF57D67DCF800405C
:10EDE000346087E807007046F0BD00BF03684A6AD8
:10EDF0009A4210B473D04FF0010C8B6B426993426E
:10EE00005AD04FF0010CCC6C836A9C4241D04FF039
:10EE1000010C0A6EC46BA24228D04FF0010C01F520
:10EE20007D6191ED007AD0ED147AB4EE677AF1EE5F
:10EE300010FA17D190ED150AD1ED010AB4EE600A6F
:10EE4000F1EE10FA0ED190ED161AD1ED021A5DF81E
:10EE5000044BB4EE611AF1EE10FA0CBF60464CF0B0
:10EE60000100704701205DF8044B70474A6E036C47
:10EE70009A42D2D18C6E426C9442CED1CC6E836CCD
:10EE80009C42CAD10A6FC46CA24218BF4CF0010C5C
:10EE9000C5E70A6DC46AA242B9D14A6D036B9A42B2
:10EEA000B5D18C6D426B9442B1D1CC6D836B9C42D9
:10EEB00018BF4CF0010CACE7CC6B83699C42A0D12D
:10EEC0000C6CC26994429CD14B6C046AA34298D1E9
:10EED0008B6C426A934218BF4CF0010C93E78C6A2A
:10EEE00043689C4287D1CA6A8468A24283D10A6B74
:10EEF000C3689A427FF47FAF4A6B0469B2EB040C9B
:10EF000018BF4FF0010C78E7F0B501F124058646F3
:10EF10000C460FCD76460FC604F138070FCF2D688B
:10EF200035600EF1140C04F14C06ACE80F000FCE66
:10EF30003F68CCF800700EF128050FC504F1600C95
:10EF400033682B60BCE80F000EF13C060FC604F5D9
:10EF50007D6494E80700DCF8007037600EF150051E
:10EF600085E807007046F0BD034B186810B10168D2
:10EF70000A681047704700BF7CDD0120034B5868CA
:10EF800010B101680A681047704700BF7CDD01209E
:10EF9000034B186810B101680A681047704700BF3A
:10EFA00084DE0120034B586810B101680A681047DD
:10EFB000704700BF84DE0120034B986810B10168E0
:10EFC0000A681047704700BF84DE0120034BD868F1
:10EFD00010B101680A681047704700BF84DE012045
:10EFE000034600201972DA60704700BF0A4A0B4BD3
:10EFF0000B480C4910B5002414601A6802601A60AE
:10F000000B6823B1186810B101680C68A047064866
:10F010000022027010BD00BF38100B4030100B40B2
:10F02000A0DE01209CDE0120A4DE0120F0B572B636
:10F0300099B904688CB102790F2A0ED843490B881C
:10F0400043FA02F5EF070AD502F1007606F590675C
:10F05000B4EB471F03D162B6F0BD3C490B8813F0F7
:10F06000010226D09E0757D55D0757D51C0757D5F7
:10F07000DA0657D59F0657D55E0657D51D0657D5D4
:10F08000DC0557D59A0557D55F0557D51E0557D5C9
:10F09000DD0457D59C0457D55A0409D5DA0B08BFAF
:10F0A0000F2206D062B60024102204600271F0BD67
:10F0B0000E22012595402B430B8062B6244E254D30
:10F0C000254FDFF89CE0D1B20171336843F00204B0
:10F0D000346002F1007C2A68A6F5802642F0020422
:10F0E0002C600CF59063283EDFF878C01B4C5B0168
:10F0F00040F28245CEF8005039708CF8001000279D
:10F100003170217003601F605F609F60DF601F616E
:10F110005F619F61DF61F0BD0122CAE70222C8E79B
:10F120000322C6E70422C4E70522C2E70622C0E79D
:10F130000722BEE70822BCE70922BAE70A22B8E79D
:10F140000B22B6E70C22B4E70D22B2E7ACDE0120B9
:10F15000408004403C8004401A8000401F800040F2
:10F16000008000401E80004030B314490B6833B962
:10F17000134B0B60B3FBF0FC00FB1C30704770B40A
:10F18000104C114A114E84FB035C9C44DD17C5EB07
:10F190002C4402FB143206FB04F444F2A71303FBD5
:10F1A0000245002D02DA05F10046751E0D60B5FB23
:10F1B000F0F100FB115070BC704700BFB0DE0120C1
:10F1C00042CE0C1F5F0B4E831DF30100ECF4FFFFDA
:10F1D00008B5FCF75DFDFFF769FDFCE7844641EAF1
:10F1E000000313F003036DD1403A41D351F8043BBF
:10F1F00040F8043B51F8043B40F8043B51F8043B11
:10F2000040F8043B51F8043B40F8043B51F8043B00
:10F2100040F8043B51F8043B40F8043B51F8043BF0
:10F2200040F8043B51F8043B40F8043B51F8043BE0
:10F2300040F8043B51F8043B40F8043B51F8043BD0
:10F2400040F8043B51F8043B40F8043B51F8043BC0
:10F2500040F8043B51F8043B40F8043B51F8043BB0
:10F2600040F8043B51F8043B40F8043B403ABDD21F
:10F27000303211D351F8043B40F8043B51F8043BC1
:10F2800040F8043B51F8043B40F8043B51F8043B80
:10F2900040F8043B103AEDD20C3205D351F8043B50
:10F2A00040F8043B043AF9D2043208D0D2071CBF1C
:10F2B00011F8013B00F8013B01D30B880380604645
:10F2C000704700BF082A13D38B078DD010F00303BB
:10F2D0008AD0C3F10403D21ADB071CBF11F8013B2B
:10F2E00000F8013B80D331F8023B20F8023B7BE77A
:10F2F000043AD9D3013A11F8013B00F8013BF9D2A5
:10F300000B7803704B7843708B788370604670473E
:10F3100008B5104C08E0206841050DD421680A05A5
:10F320000FD42268D30411D423685803F3D500F016
:10F33000E1FE20684105F1D502F0AEF921680A0529
:10F34000EFD502F0B7FA2268D304EDD502F0C0FB86
:10F35000EAE700BF3480044008B5FFF7D9FF00BFDB
:10F36000014B10221A80704700200540704700BFF3
:10F37000094908B50B6830B16A461844A2F5005C2B
:10F38000604502D20860184608BD03F0A7F90C21B9
:10F3900001604FF0FF3008BD3C24FF1F0078B0FA39
:10F3A00080F14809704700BF01230370704700BF18
:10F3B000084A1378802B01D0002070470649074B7C
:10F3C00007480860002119701378802BFCD00120B9
:10F3D000704700BF03E007404480044001E007405D
:10F3E000000028220A4A1378012B01D00020704720
:10F3F00003F1804000F5FC2C60218CF8001013789C
:10F40000802BFCD10348044A02600120704700BFF2
:10F4100003E00740448004400000060203F08CB97A
:10F4200003F092B9704700BF3F28F0B445D8042AD2
:10F4300043D8DFE802F0474A4D0344004FF410255B
:10F440002D4C04EBC0035B681A6812F4E06648D0E8
:10F450002A4A2B4E2B4CC2F8306103F1404CACF5DC
:10F4600092262948294FC2F82C417C2E284CC2F8FC
:10F470003401C2F83871C2F83C412CD9ACF5942261
:10F480007C2A2AD9ACF596207C2828D9ACF5982777
:10F490007C2F2ED9ACF59A247C2C0ED81D4E72B63A
:10F4A0001A6822F4702747F08070C3F3840C284355
:10F4B0001F6046F82C10186062B6F0BC70474FF41D
:10F4C0003025BDE74FF40025BAE74FF44025B7E7F4
:10F4D0004FF42025B4E7104EE1E7104EDFE7104E61
:10F4E000DDE754F830704FF4807087F88062186060
:10F4F000AEE70C4ED3E700BF141304000002FF1F59
:10F50000F921FF1F2922FF1FC921FF1F9921FF1F7A
:10F510006921FF1F8825FF1F4024FF1FB824FF1FFC
:10F520001825FF1F4825FF1F30B4054B054D064C1D
:10F53000002210211A602A602060196030BC7047D8
:10F5400014D0034004D0034000D003402DE9F84319
:10F55000944B9548954D964E964C9749DFF87CC252
:10F56000DFF87CE2954F4FF000621A604FF0805256
:10F570001A604FF000521A604FF080421A604FF04C
:10F5800000421A600022026028234EF6FF70CCF879
:10F59000000006F50028CEF8003005F5002C2360A9
:10F5A0000EF5012E0B6033602B603B60A36207F504
:10F5B00000278B6204F5012401F501210EF11006EC
:10F5C00008F6E8790CF6E87507F57F681031203405
:10F5D000C9F800302B603360C8F800300B6023603E
:10F5E000774CC8F81830A8F5002C04F58057ACF11A
:10F5F000200E08378B610921216007F5FD28CEF820
:10F6000000203860CEF80830FB600EF5FE2708F2C7
:10F61000FC7404374EF8041C22603860A360FB6061
:10F6200044F8041C083404F6FC7CC7F8FC2FCCF822
:10F630000000ACF5E120A0F2DC78C9F800302B60C6
:10F64000C7F8F81FD8F800105E4841F40074C8F8F5
:10F650000040016806F57F4606F1E80E41F00074AF
:10F6600007F5883709F5803905F58035564E046071
:10F67000CEF8002047F6FF7008223860C9F8003045
:10F680002B60326001F04CFF72B6504B504C514F22
:10F690001E682568396862B6490102D5322E88BFD6
:10F6A0000135C6F52F3C0CF21F304B4FDFF81C9193
:10F6B000DFF8208183084FF47A72A7FB031602FB60
:10F6C00005F505EB9605322672B6D9F800102268CA
:10F6D000D8F800E062B6C1F52F3C0CF21F30830869
:10F6E000A7FB030C1EF0806FC5EB9C034FF47A70F0
:10F6F00002D0322988BF013200FB0231B1F57A7F96
:10F7000004D3013E05D005F57A75DDE701F020FD53
:10F71000DAE701F041FA72B62C4B2E4A18682668D7
:10F72000116862B64A0102D5322888BF0136C0F599
:10F730002F3E0EF21F35284FDFF89090DFF89480AF
:10F74000AB084FF47A7202FB06F6A7FB031006EB38
:10F7500090054FF4AF7672B6D9F800102268D8F849
:10F7600000E062B6C1F52F3C0CF21F339808A7FBEE
:10F77000000C1EF0806FC5EB9C034FF47A7002D032
:10F78000322988BF013200FB0231B1F57A7F04D300
:10F79000013E05D005F57A75DDE701F0D9FCDAE721
:10F7A000BDE8F88304E100E0048003402C800340BE
:10F7B00024800340148003401C80034034800340B5
:10F7C000008003400480044000900C4018E000E0FA
:10F7D000B4DE012004ED00E0176CC1160880034080
:10F7E0000C800340A0F14203012B51D911B93F28ED
:10F7F00064D9704710B4A04A92F800C0012202FAFE
:10F800000CF4A14250D2C31E012B40F2BD81A0F1E5
:10F810001D02012A40F2BF810E2800F28A8044F2C4
:10F820008414C440E20740F18480944A146804FBC5
:10F83000011323FA0CF3A0F1020CBCF1240F00F227
:10F840008381DFE81CF07A01730111010A010301D1
:10F85000FC00F500EE00E700810181018101E0007C
:10F860008101D900D20081018101CB00C400BD001B
:10F87000B60081018101810181018101AF00A800F1
:10F880008101810181018101A1009A0093008C0016
:10F89000794B1A780B2A0CD8C2F10C0399404228F4
:10F8A000084624D001F0CABE3F2822D95DF8044B97
:10F8B00070470C2A1CBF0C3AD140F0E7704B53F84C
:10F8C000302092F8801203EBC00C59B30120DCF811
:10F8D000043082F800014FF0010C4FF4A27182F85D
:10F8E00080C219601A6822F020001860704701F089
:10F8F00087BE634B53F8301091F8804203EBC00C85
:10F9000044BBDCF804301A6842F00300186001249C
:10F910004FF4A27281F880421A60196821F0200029
:10F920001860C3E7DCF80430186820F002011960A1
:10F93000D1E7A0F12303032B7FF677AFA0F11002EC
:10F94000012A94BF4F4A504A146804FB011323FA5A
:10F950000CF370E781F88020DCF80430D7E74B49DE
:10F960004B480B604FF4517202609FE7494C4A4983
:10F9700023604FF451730B6098E74848484A03608E
:10F980004FF45174146091E7464947480B604FF4B7
:10F99000517303608AE7454C454A23604FF4517127
:10F9A000116083E74348444C03604FF45173236074
:10F9B0007CE74249424A0B6040F24440106075E7E0
:10F9C000404C4149236040F244430B606EE73F489E
:10F9D0003F4A036040F24444146067E73D493E48B3
:10F9E0000B6040F24443036060E73C4C3C4A2360B8
:10F9F00040F24461116059E73A483B4C036040F2E1
:10FA00004463236052E73949394A0B6040F244406D
:10FA100010604BE7374C3849236040F244430B6099
:10FA200044E73648364A036040F2444414603DE7F8
:10FA3000344935480B6040F24443036036E7334CA9
:10FA4000334A236040F2444111602FE73148324C81
:10FA5000036040F24443236028E73049304A0B609A
:10FA600040F24440106021E72E4C2F4923604FF4B0
:10FA700051730B601AE700BFF425FF1F08900B407D
:10FA80001413040008900C400880034048900B4079
:10FA90002CB0044040900B4028B0044038900B40FC
:10FAA00024B0044030900B4020B0044018800B403C
:10FAB0004CA0044010800B4048A004401880034034
:10FAC00008B004401080034004B00440408003406C
:10FAD00018C004403880034014C0044018900C4003
:10FAE00004A0044010900C4000A0044018900B406B
:10FAF00004C004402880034010B00440208003402C
:10FB00000CB0044028900B400CC0044020900B40E7
:10FB100008C004403080034010C0044048800340C7
:10FB20001CC0044018900340349004402348244AE9
:10FB300003604FF451741460B8E6224922480B6008
:10FB400040F244430360B1E63F283FF6AFAE1F4C9E
:10FB500054F8302092F8803223B37F294FF0010C03
:10FB60004FEAC0038CBF82F880C082F800C12344F2
:10FB700001245B6882F880424FF4A2721A60186810
:10FB800020F02001196091E6114A146804FB01136A
:10FB900023FA0CF34FE60F4A146804FB011323FA0F
:10FBA0000CF348E6C300E0187F29406801688CBF69
:10FBB00041F0030121F002010160D8E710900340F9
:10FBC0003090044010900B4000C004401413040017
:10FBD0000890034008800B4038B1102828BF10203F
:10FBE000044AC3B2107813707047024A0123107898
:10FBF00013707047F425FF1FA0F11002D2B2012A42
:10FC000070B440F2A280DFED647A6449B4EEE70A92
:10FC1000F1EE10FA47F612234EBF10210B460821D1
:10FC200000EE903A9FED5E7AB8EEE01A61EE076A58
:10FC3000B4EEE60AF1EE10FA80F29E805C0801EE66
:10FC4000104AB8EEC11A61EE071AB4EEE10AF1EEFD
:10FC500010FA80F293809E0802EE106AB8EEC21A83
:10FC600061EE072AB4EEE20AF1EE10FA80F2888023
:10FC7000DC0803EE104AB8EEC31A61EE073AF4EE60
:10FC8000C03AF1EE10FA7DD91E0904EE106AB8EE02
:10FC9000C41A61EE074AB4EEE40AF1EE10FA73DA20
:10FCA0005C0905EE104AB8EEC51A61EE075AB4EECB
:10FCB000E50AF1EE10FA69DA9E0906EE106AB8EE6E
:10FCC000C61A61EE070AB4EEE00AF1EE10FAA8BF18
:10FCD000062505DADD0907EE905AB8EEE71A072582
:10FCE00081EE007A4FF6FF7CC31EB6EE000A77EE77
:10FCF000406AFCEEE61A11EE904A644528BF64465D
:10FD0000012B35D917280ED9A0F11D03012B3FD99E
:10FD10000E281DD9233803281FD9012A13D8214BB7
:10FD2000214E22481CE0224EC64006F0010383F01B
:10FD30000106002BE8D01F4B1F48204A1E602943B4
:10FD400006601460196070BC70471D4B082167E79E
:10FD500044F28416C640F307DCD51A4B1A4E1B48F2
:10FD6000294300251D6035600460196070BC704730
:10FD7000174B184E1848F3E70025B1E70125AFE708
:10FD80000225ADE70325ABE70425A9E70525A7E78D
:10FD9000124B134E1348E3E7C0E1E440008793039E
:10FDA0000000803700900C4004900C4008900C40FC
:10FDB0006006F00000800340048003400880034098
:10FDC0000024F40000900B4004900B4008900B407E
:10FDD00000900340049003400890034000800B40D3
:10FDE00004800B4008800B403F2806D8044B53F892
:10FDF000300090F80012C8B270470020704700BF72
:10FE0000141304003F2820D81B4A02EBC003012929
:10FE10005B680FD004291DD052F83000002280F812
:10FE2000802299B1022923D003290DD14FF4817189
:10FE30001960704752F830004FF4A27280F88012B7
:10FE40001A60196821F020021A6070474FF4807020
:10FE50001860704752F830104FF0010C4FF4A27246
:10FE600081F880C21A60186840F02001196070475C
:10FE700040F203121A6070471413040072B60D4961
:10FE80000D4A0E4B1B680868116862B64A0102D51C
:10FE9000322B88BF0130C3F52F3C0CF21F320849CA
:10FEA00093084FF47A72A1FB031C02FB00F000EBF5
:10FEB0009C007047B4DE012004ED00E018E000E093
:10FEC000176CC1162DE9F843054672B6224B234F35
:10FED000234A18683C68116862B64A0102D5322884
:10FEE00088BF0134B5B3C0F52F3606F21F331D4E5F
:10FEF000DFF86490DFF8688098084FF47A72A6FB08
:10FF0000001C02FB04F404EB9C0472B6D9F8001048
:10FF10003A68D8F800E062B6C1F52F3303F21F301B
:10FF20008308A6FB030C1EF0806FC4EB9C034FF408
:10FF30007A7002D0322988BF013200FB0231B1F55C
:10FF40007A7F04D3013D05D004F57A74DDE701F032
:10FF5000FFF8DAE7BDE8F88318E000E0B4DE01203E
:10FF600004ED00E0176CC116013803280BD872B6F7
:10FF7000074B53F8201041B1002049680130002997
:10FF8000FBD162B67047002070470846F9E700BF12
:10FF900064DF012030B472B62F4A13781D0706D5EE
:10FFA0002E4B196A00293BD09C6A002C48D055780A
:10FFB0002C0706D5294B196C002947D09C6C002CC6
:10FFC00041D092F802C05FEA0C7105D5234B1D6E3B
:10FFD000002D3DD0996E99B1D278130709D51F4BEA
:10FFE000D3F88040002C35D0D3F888504FF0110C56
:10FFF00045B162B61A4B0021197030BC00F06EBEDC
:020000021000EC
:100000004FF00D0C164C174D217843F83C5003EB84
:10001000CC0308304A1E5860227062B630BC70476C
:1000200004220F4C104D94F800C043F8325003EBFB
:10003000C20108300CF1FF334860237062B6EDE76F
:100040004FF0050CDEE74FF0090CDBE70822E8E78C
:100050000C22E6E71022E4E7141504000000FF1F5D
:100060008DDF0120C800400088004000431E032BA4
:100070001FD81C4A400140F0100030B4104472B642
:10008000194C14F803C0BCF1030F1BD8DFE80CF0C7
:100090000212151703220D88E25410F0080F14BF46
:1000A000C823882343EA054308310360416062B6F0
:1000B00030BC704708300222EDE70522EBE708303C
:1000C0000422E8E7094C54F8230038B1084A52F8F2
:1000D0002350696042F8231062B6E9E744F8231020
:1000E000034AF7E70000FF1F9CDF012064DF0120C7
:1000F00074DF01202DE9F04FDFF82093DFF820A313
:10010000DFF820B385B044E0B24D9E0805EBC6078A
:1001100008F1FF3C7A6803F008015FFA8CF4A2F161
:10012000080001F0FF0E002940F0068155F8363036
:100130001B0C1FFA83F822F8088C002B00F0F380C8
:10014000A54922F806EC51F8243042F804EC002BC3
:1001500000F0C282A14951F824205060A04A41F821
:10016000240032F814E0F04422F8148000F096FDE8
:10017000002800F0AA829B4B9B4C17F0080F00F15F
:10018000080018BF1C46786045F83640082189F8F9
:10019000001099F80040E6B275071CD5934B18780B
:1001A000B0B193490A7802F0FF0522B16F1EFCB28C
:1001B0000C7004B900BE8F48017801F0FF0839B116
:1001C00008F1FF3C5FFA8CF30370002B00F05282C1
:1001D000042289F8002006F0080505F0FF02002D32
:1001E00000F0D2809AF80000C3B25FEA13188BD1F6
:1001F0009808DFF8E08158F8305008EBC006C5F3E6
:1002000083077A1E71680C2A00F28980DFE802F009
:100210007D7D8787878787874587878707000F6862
:10022000754E704B4C6848F83030BDB240F2816C6E
:10023000724873497460002201246545376002608A
:10024000C8F81020C8F818200C70624F00F2F08037
:10025000B5F5D06F80F03B83B5F5817F00F0F48277
:1002600000F28C82802D00F06983822D40F0F282B2
:10027000B38803F07F01042900F2EC82614D6248EB
:100280008F003D440270427095F800E05FEA8E7581
:1002900040F14B840470022434E3584E326842B378
:1002A000DFF884C1564BBCF80010584F1C783878E2
:1002B00040290D4628BF4025491B002C40F0020E66
:1002C00084F0010489B21C70ACF800100CBF8824C3
:1002D000C82408EBCE0C80F0010044EA0543CCF8BA
:1002E000042048F83E302A443870002900F0468146
:1002F0003260414EB6F80080B8F5A06F0FD1444D82
:10030000B278002777702A7009E03B4C238842F2CC
:100310002106B34200F03681324C48F830400120CB
:100320008BF8000032E72F4A2F4817F0080F18BF4C
:10033000104645F8360029E700F0D0FC354A52F85F
:100340002430002B00F0CC81DFF8E0E058681EF884
:1003500004C042F8240003F108027A60BCF1030FE4
:1003600007D8DFE80CF032022E2A4FF002080EF810
:1003700004801C8817F0080F0CBF8823C82343EAA9
:10038000044345F8363001E7F00700F17681310685
:1003900000F1B681B20708D51F4D204A95F80090AC
:1003A00002275FFA89F32B701770F30602D51B4EF4
:1003B0001024347005B0BDE8F08F04210EF804104D
:1003C000D7E705200EF80400D3E74FF0030C0EF832
:1003D00004C0CEE70000FF1F10DF0120BCDE0120BB
:1003E00008E30120C80040008800400098DF012099
:1003F00021DF0120A0DF012084DF0120B8DE012001
:1004000020DF0120C020074090DF01208CDF012089
:100410009820074064DF01208820074080200740A3
:100420009020074094200740CCDE01209CDF012073
:1004300042F22100854200F0198100F2CE80B5F52C
:10044000086F00F05B82B5F5106F40F003823D6AE3
:10045000B049B6780E702C0600F1F782D8F8284023
:10046000AD4A200600F1EB82D8F83000AA49020616
:1004700000F1DF82D8F83860A74F330600F1D3824D
:10048000D8F84020A44B170600F13083D8F8485024
:10049000A1492E0600F12483D8F850709E4C3D06E9
:1004A00000F11883D8F858309B481C0600F10C83E3
:1004B000D8F860609849300600F10083D8F86840A9
:1004C000954B220600F1F482D8F87000924D030695
:1004D00000F1C782D8F878708F493F0600F1BB82DF
:1004E000D8F880308C4A1E0600F11983D8F888505D
:1004F000894E2D0600F10C83D8F8904086492406D9
:1005000000F1FF82D8F89820834D100600F1F382A5
:10051000824C834E8349844F0394002501960291B7
:100520002C46386828B1466800F0D8FB3046002ECB
:10053000F9D1019B7D4A18683C6042F8254028B1FA
:10054000466800F0CBFB3046002EF9D10298039BA1
:1005500090F800E0019943F8044B754A0C60AEF145
:10056000020C039322F81540BCF1030F00F2258121
:10057000DFE81CF067011F0167011F01402D18BF54
:100580000022B5E66B4F0A784C788D78CB783A70BC
:100590007C70BD70FB703E680A794C7989793A713C
:1005A000862E7C71B97100F08E81634B634C93F899
:1005B00000C021784CF0020200298CF001061E7068
:1005C0000CBF8823C82348F8323008EBC20381F0FF
:1005D0000107002527705D609EE642F221239D42BF
:1005E00040F0B781564F574B5749B0783E681E6070
:1005F0000870002101918C468E4608464E4E357893
:1006000045F0020708EBC703002C58600CBF882098
:10061000C82040EA0C0348F83730484BDFF818C1CF
:100620001A7085F001003070002940F01A81BEF187
:10063000400F1BD140F0020C08EBCC030198DFF80F
:10064000D8E05860002A40F021810F0447F088026A
:100650003A4B4EF83C2008441C7035700746402940
:1006600004D10021394C3A4E2180376001258BF8A6
:10067000005054E600F046FDAAE5274B35482E49C8
:100680001A614FF0020E80F800E0334F0A703349D0
:1006900019609960324E334D334C9A610D21397097
:1006A000FF213170DFF8D0E0297022702F4D304AE1
:1006B0008EF800104FF09F0A012706F804AC5D6029
:1006C0000770DA6005B0BDE8F08F2A4F45F83600B4
:1006D0003D7801353D7059E541F8240013493DE569
:1006E000104E305D032800F2E78001A151F820F0A0
:1006F0008D0101008D010100AD070100A707010078
:10070000154F184C0D208021B207387021707FF5ED
:100710004CAE41E698DF01200000FF1F74DF01208E
:1007200064DF01209CDF012010DF0120BCDE0120FE
:1007300008E3012010E301208CDF012020DF0120ED
:10074000B4DE012018E30120B0DF0120CCDE01205F
:10075000B8DE012094200740C020074088004000F8
:10076000882007408020074098200740D0DE0120E5
:1007700024DF01208DDF01208C20074040F202326F
:10078000954240F0E080B08800F07F03042B61D8F0
:100790007288002A5ED1B64E99000E44357845F035
:1007A0000207377025E701213155EFE4002737555F
:1007B000ECE4029E4FF001003070019B029A01357B
:1007C00004330132042D07F10407019302927FF4F0
:1007D000A8AEA84CA84D2778A84800263A072E7046
:1007E000077000F1F5806078A549A64F08700023D6
:1007F000C8F83030C8F83830030700F1D480A37847
:10080000A14AA04E137000211F07C8F85010C8F865
:10081000581000F1F380E7789C499A4C0F70002340
:100820003E07C8F87030C8F8783000F1A4809849C5
:100830000C78002384F00102C8F89030C8F8983092
:10084000D7E602990C70B8E7B28802F07F03042B58
:1008500040F28480864A0F25157001258BF80050E0
:100860005DE540297FF6E6AE864E019F40F0020826
:1008700006EBC8004760A2B18CF80050814D854E50
:100880001C704039403745F83860EBE60804804B6F
:10089000019F1C7040F0C80235700F444EF83C2098
:1008A000DDE61C70019F774C7B4A8CF80050403984
:1008B000403744F83820D5E617F0080F0CBF022067
:1008C0000320305562E4754F0F253D706DE6744F7F
:1008D00078680028BED07488B58803E00C37786843
:1008E0000028B7D03A88A242F8D17B88AB42F5D134
:1008F000240A032C0CBF04783C8903E0694A6A4847
:1009000017780770B6F806C0A44580F03581674EA9
:10091000357845F0020708EBC701BCF1400FE64609
:1009200028BF4FF0400E486070440190CEEB0C01A0
:1009300000224FEA0E4C0124C8206AE65A480224DD
:1009400002704270DEE7B5F5A06F83D1002201246A
:100950004FE642F22136B542F8D07BE77288002A92
:100960007FF478AF42489E00304490F800C02CF0ED
:10097000020101703DE600F091F9002800F0EF80DF
:100980000830C4F884004448C8F8800000F086F9B4
:100990003C4E002800F0DD8008303E4DC6F88C004B
:1009A000C6F8885043E700F079F9002800F0C480C9
:1009B000083078643848C8F8400000F06FF9314ECC
:1009C000002800F0B4800830324FF064B76416E7B6
:1009D00000F064F9002800F0CB800830C8F824004B
:1009E0002D48C8F8200000F059F9264B002800F0E7
:1009F000BA800830274ED8629E62F4E600F04EF9C5
:100A0000002800F0A280083070662348C8F8600013
:100A100000F044F91B4B002800F0928008301D4E76
:100A2000D8669E66F7E6FC6BA4F1080000F056F964
:100A300026E54D6BA5F1080000F050F91AE5D36AE0
:100A4000A3F1080000F04AF90EE57F6AA7F108005B
:100A500000F044F902E5CC6FA4F1080000F03EF983
:100A60003EE56E6FA6F1080000F038F932E500BFF0
:100A7000C0200740141504008DDF0120C42007406A
:100A8000C82007400000FF1FCC200740D0200740AF
:100A900020DF0120C80040008800400021DF012045
:100AA0001815040098DF012090DF01208CDF012061
:100AB000DA6EA2F1080000F011F905E54F6EA7F11A
:100AC000080000F00BF9F9E4C56DA5F1080000F08D
:100AD00005F9EDE4626DA2F1080000F0FFF8E1E431
:100AE000CE6CA6F1080000F0F9F8D5E4586C08388F
:100AF00000F0F4F8CAE4D5F89C00083800F0EEF8ED
:100B000006E5D1F89430A3F1080000F0E7F8F9E425
:100B1000D6F88C70A7F1080000F0E0F8ECE4D2F809
:100B20008400083800F0DAF8E0E40224EAE62978E4
:100B3000B064481C287062E62A7801322A703AE7CD
:100B40002A789866501C287065E62F7801372F7038
:100B50005CE72F78C6F88800781C287067E62A784A
:100B600001322A7010E72A789862571C2F703AE6F3
:100B700029780131297034E7402CA64628BF4FF070
:100B8000400ECEEB040100EB0E0401944FEA0E4C34
:100B90000022012432E500BF2DE9F04101F090F977
:100BA000324C334B3348DFF8E880DFF8E8C0324E90
:100BB000324FDFF8E4E000221A605A609A60DA608F
:100BC0001A615A619A61DA611A625A629A62DA6249
:100BD0001A635A639A63DA631A645A649A64DA6429
:100BE0001A655A659A65DA651A665A669A66DA6609
:100BF0001A675A679A67DA67C3F880202168C3F8D2
:100C0000842041F48025256001681D4D41F040712C
:100C10000160032088F80000C3F30721C3F30740F5
:100C200004F528341B0E4FF0A0088CF80080CC345B
:100C30003170387013492B70FF238EF80030124D3D
:100C40000CF8B83C11480B704FF0010C06F808CCBA
:100C5000227070264FF40014102207F82CCC2E704E
:100C6000046081F8F820BDE8F08100BF34800440C2
:100C70000000FF1F00D800409C200740B020074024
:100C8000B42007401020074035E400E004E100E014
:100C900044210740402107408020074072B60D489C
:100CA0000268B2FA82F30B2B10DC4FF00041D940FE
:100CB00022EA0102026062B6074803EBC303DB00CD
:100CC000C2180021C15010465160704762B6002022
:100CD000704700BFF825FF1FD003FF1F0D4B0E4AC2
:100CE000C11AA2FB01231B090B2B0CD80B4A11784C
:100CF00051B972B60A484FF0004C02682CFA03F35F
:100D00001A43026062B67047064A11780029F0D093
:100D1000FFF740B9D003FF1F398EE3388DDF012084
:100D2000F825FF1F98DF0120044B054A19689088B9
:100D300019B10A884B88D11A08447047ACDF0120EA
:100D400008E301202DE9F04FA74A83B00123137077
:100D50000191002900F0B0800E46A449A44F04463A
:100D60000868002800F03581A24DB0F802E0CEF10D
:100D70004003B34228BF33460EEB030291B200F1A9
:100D800008084FF0000BF61A418003F1FF3C08EB16
:100D90000E0285F800B0002B00F086800EF1080BE3
:100DA0000EF10C0101448344251DAB4538BF8C4234
:100DB0002CBF01210021092B94BF002101F001016A
:100DC000002900F0B18044EA0B095FEA897140F024
:100DD000AB80191F4FEA910E0EF1010ABCF1020F10
:100DE0004FEA8A0940F29E8059464FF00108256873
:100DF00041F8045BC2450EF00705A6463AD9002D1E
:100E000061D0012D2ED0022D26D0032D1ED0042D11
:100E100016D0052D0ED0062D06D05EF8045FCBF857
:100E2000045004314FF002085EF8045F41F8045B9F
:100E300008F101085EF8045F41F8045B08F101085D
:100E40005EF8045F41F8045B08F101085EF8045F96
:100E500041F8045B08F101085EF8045F41F8045BA7
:100E600008F1010808F101085EF8045F41F8045B2D
:100E7000C24528D84B454A44C9EB0C0C04EB090881
:100E800000F02B8198F800101170BCF1000F47D0D2
:100E900098F801505570BCF1010F41D098F802103C
:100EA0009170234441881C463F292FD8524D05217B
:100EB0002970002E7FF455AF01984B4F00263E70ED
:100EC00003B0BDE8F08F9B460D46DEF8043045F8D0
:100ED000043BDEF808304B60DEF80C306B60DEF867
:100EE0001050CD60DEF814300B61DEF818504D6103
:100EF000DEF81C308B6108F108085EF8205FCD61D8
:100F0000C24501F12001DFD85B46B3E740220280F1
:100F100001460420FFF7AAF8344B00201860C5E70B
:100F20002344BFE7A046ADE72146234411F801ABB7
:100F300008F80EA0E4431C44994204F00705B1D020
:100F40004DB3012D21D0022D1BD0032D15D0042D22
:100F50000FD0052D09D0062D1CBF11F8015B02F83A
:100F6000015F11F8018B02F8018F11F8019B02F863
:100F7000019F11F801CB02F801CF11F801BB02F873
:100F800001BF11F8014B02F8014F11F8015B02F8A3
:100F9000015F994286D08A4608311AF8014B547095
:100FA0009AF80050957011F8064CD47011F8055C51
:100FB000157111F8044C547111F8035C957111F816
:100FC000024CD47111F8015C02F8085F9942E2D139
:100FD00068E73D78002D00F08980DFF820A0054DFE
:100FE0004FF0010940E000BFA1DF0120A4DF012094
:100FF00098DF0120A8DF0120A0DF012021480100A7
:10100000BAF101086BD02878002868D100F0A0F868
:101010003B78002B6AD00420FEF7A6FF072835D9BD
:10102000287800285BD100F093F83A78002A5DD048
:101030000420FEF799FF072835D9287800284ED1DB
:1010400000F086F83978002950D00420FEF78CFF94
:10105000072835D92878A8F1030A00283FD100F0E5
:1010600077F83B78002B41D00420FEF77DFF07285E
:10107000C6D8224B83F80090FFF710FE204A10607C
:1010800000287FF472AE1D490870B9E71B4A82F848
:101090000090FFF703FE1A49086000287FF465AE50
:1010A000164B1870BCE7154981F80090FFF7F6FD64
:1010B000134B186000287FF458AE104A1070BCE73C
:1010C0000E4B83F80090FFF7E9FD0D4A10600028F1
:1010D0007FF44BAE09490870BCE74346E2E60124C1
:1010E0004FF0FF302C7003B0BDE8F08F034C0020B0
:1010F00020704FF0FF3003B0BDE8F08FA1DF01207A
:10110000A4DF012038B50F4B187880B90E4C216848
:1011100071B1B1F802C0A1F800C000F0FF050420D1
:10112000FEF7A4FF256038BD084901220A7038BDCA
:10113000FFF7B4FD0028F7D00146BDE83840042091
:10114000FEF794BFA1DF0120A4DF0120A0DF012072
:1011500038B52C4C237803B138BD01202070FFF73F
:10116000E3FD002842D100F087FA00283BD100F0CF
:1011700091FB002834D100F09BFC70BB00F018FDFF
:1011800040BB00F095FD10BB00F012FEE0B900215D
:101190002170EFF30582002ADED1EFF3108172B6E1
:1011A000194B186828B3194C227812BB45691D6089
:1011B000012323700DB3AA6101B962B600254577FA
:1011C000816888472570C7E700F0A8F9DFE700F0DD
:1011D000A3F9D9E700F09EF9D3E700F099F9CDE73C
:1011E00000F094F9C7E700F08FF9C0E700F0DAFEED
:1011F000B9E70029B0D162B638BD054A15600029AB
:10120000DCD1DAE7B1DF0120C4DF0120C8DF012033
:10121000C0DF012010B4047F4160022C0346C2608D
:1012200010D0EFF3108172B6427F32B9007F0128EF
:101230000CD0032814D00120587701B962B65DF8AC
:10124000044B704783685DF8044B1847114C2068C5
:10125000A0B1114C5A6122689A6123605361EAE798
:101260000E4C206880B10E4C5A6122689A6123604E
:1012700053610C4C4FF080502060DCE7064A586107
:10128000986123601360D6E7054A5861986123602E
:101290001360EEE7C4DF0120C0DF0120B4DF0120CE
:1012A000B8DF012004ED00E070B5EFF3108272B6F4
:1012B0000C4C206880B10C4E00254369236073B14B
:1012C0009D6102B962B6457781688847EFF3108265
:1012D00072B620680028F0D102B962B670BD3360E2
:1012E000EFE700BFB4DF0120B8DF01202DE9F843AC
:1012F000794E3468002C31D0206800282CD1DFF8DA
:10130000EC91764FDFF8E8810546A36803B1DD6014
:1013100020693360016825750B684B456AD1027FEF
:101320004560022AC46069D0EFF3108272B6437F31
:1013300043B9017F012900F09080032900F09980D2
:101340000121417702B962B66368002B3FD134684E
:1013500024B120680028D8D0471E2760EFF31085FD
:1013600072B65F4B00211868196005B962B6002893
:1013700000F0AD804FF000093568CC464FF0020E0A
:101380000EE0CC1A8560C0F80CC001462C60E86005
:101390004FF0010980F814E00D463846002F51D077
:1013A0008768002D53D0036829688B42E9D32C4607
:1013B00003E011688B42144635D3A2685B1A0360C0
:1013C000002AF6D18260C4602946A060E2E7306856
:1013D000414A2360002868D001688B4211D2CB1AA1
:1013E000A060E5600360C46014602046022222759C
:1013F0000446AEE7224600219847A5E78268904759
:10140000A2E7864603E011688B4296463ED3DEF89B
:1014100008205B1A2360002AF5D1A260C4F80CE012
:10142000CEF80840E2E7D268C2608460E060C2683B
:10143000CB1A294690600D46236080F814E03846A8
:10144000002FADD1B9F1000F43D1BDE8F88385601D
:10145000C56001464FF001099CE7DFF898E0DEF82F
:10146000001039B31F4943610B68836108605861FC
:1014700066E7396829B31C4943610B6883610860DA
:1014800058614FF08051C8F8001059E7D268E26007
:10149000C4F808E0CEF80C40E268CB1A0221946050
:1014A000CEF800302175044653E7A060E060146078
:1014B00020469BE70B4B41618161CEF8000018602C
:1014C0003EE7094B4161816138601860D9E7BDE8AA
:1014D000F8833160BDE8F883BCDF0120B4DF012070
:1014E000CCDF0120C0DF0120B8DF01201512010090
:1014F00004ED00E0C4DF0120024A136801331360E9
:10150000FFF7F4BEB4DE0120704700BF704700BF94
:10151000704700BF704700BF704700BF704700BFF3
:1015200030B42948294A2A4B2A4D6024E12104700D
:1015300011701B78284C082B30D00A2B27482849DB
:1015400037D00C2B0CBF35225D2212232A6023607A
:1015500002600B60234D24482C782449BCB1012241
:1015600002600A60224B234C1D782348012D26D9A6
:10157000042D0FD9082D1ED9102D94BF862587253F
:10158000256005601D4D01242C7030BC704704603F
:101590000C60E7E7842222600260F3E700F58E200A
:1015A0000F490830212213232A60236002600B6058
:1015B000D0E73922F7E7852121600160E2E7802347
:1015C00023600360DEE700BF0040074001400740A2
:1015D000FC25FF1F08B003400CB0034008B00B40CF
:1015E0000CB00B40D1DF012020B0034020B00B40F5
:1015F000FD25FF1F24B0034024B00B40D0DF0120A5
:101600000A4A0B49136843F4805313600A7842B9BD
:101610000849C0230B70084B80F30C0000B21880FF
:101620007047044980220A70F5E700BF2C8004400F
:10163000D1DF012021C00C4000C00C400A4A0B49F8
:10164000136843F4005313600A7842B90849C02371
:101650000B70084B80F30C0000B2188070470449EF
:1016600080220A70F5E700BF2C800440D1DF012002
:1016700021D00C4000D00C40054A064B1078197858
:10168000C2B2CBB29A4238BF4032D01A704700BFC4
:101690005CE00120D9DF0120F0B574490B7913F02B
:1016A000300F08D072B68A7D02F0FF0CD2B9402606
:1016B000CA794E7462B66D4FF878C2B2150600F161
:1016C000AF8052060DD5694D2879430609D5684A81
:1016D000684E13680027377003B11F70634C3C21BC
:1016E000E170F0BD62B6644E644834780778644DAA
:1016F000E2B2531C402BCC79F8B228BF00230CF186
:10170000FF3783425FFA84FE07F0030402D005F836
:1017100003E01A460CF1FF3C1CF0FF036ED067B2E9
:1017200097B3012F1FD0022F0ED0541C402C91F8DC
:1017300007C028BF002484425FFA8CF703F1FF330F
:101740001CBF2F552246DBB2541C402C91F807C019
:1017500028BF002484425FFA8CF703F1FF331CBFDB
:101760002F552246DBB2541C402C91F807C028BFED
:10177000002484425FFA8CF703F1FF331CBF2F551E
:10178000224613F0FF0339D0541C402C91F807C0B7
:1017900028BF002484425FFA8CF71CBF22462F55D5
:1017A000541C013B402C5FFA83FC28BF0024CB79FA
:1017B0008442DFB201D02F552246541CCF79402CF1
:1017C00028BF00248442FFB21CBF2F5522460CF1D3
:1017D000FF3C541C5FFA8CF303F1FF3C402CCF79A3
:1017E00028BF00245FFA8CF3844203F1FF3CFBB274
:1017F0001CBF2B5522461CF0FF03C5D121490D68A3
:10180000D4B23470002D3FF456AF824236BFC0F1DF
:101810004000121A1218272AC4BF01222A704AE770
:1018200097F804C05FEA0C647FF54BAF164B174E78
:1018300019783578CCB2EBB29C420ED0144901E055
:10184000A3420AD00133402B28BF00233879C85C5B
:10185000C5B2FD71387D0728F2D9044CDFB237706C
:101860002179080644BF7C21E1702AE700A00640E8
:1018700060E00120D8DF01205CE00120D9DF0120F9
:101880001CE00120D4DF012064E001205DE00120A4
:10189000DCDF0120054A064B10781978C2B2CBB2C2
:1018A0009A4238BF4032D01A704700BFD8E00120BA
:1018B0006DE00120F0B574490B7913F0300F08D0BA
:1018C00072B68A7D02F0FF0CD2B94026CA794E74F6
:1018D00062B66D4FF878C2B2150600F1AF805206BD
:1018E0000DD5694D2879430609D5684A684E1368B5
:1018F0000027377003B11F70634C3C21E170F0BDCD
:1019000062B6644E644834780778644DE2B2531C82
:10191000402BCC79F8B228BF00230CF1FF3783426B
:101920005FFA84FE07F0030402D005F803E01A46CC
:101930000CF1FF3C1CF0FF036ED067B297B3012F90
:101940001FD0022F0ED0541C402C91F807C028BF86
:10195000002484425FFA8CF703F1FF331CBF2F553C
:101960002246DBB2541C402C91F807C028BF00244B
:1019700084425FFA8CF703F1FF331CBF2F552246D8
:10198000DBB2541C402C91F807C028BF00248442CD
:101990005FFA8CF703F1FF331CBF2F55224613F07B
:1019A000FF0339D0541C402C91F807C028BF0024F5
:1019B00084425FFA8CF71CBF22462F55541C013B12
:1019C000402C5FFA83FC28BF0024CB798442DFB22D
:1019D00001D02F552246541CCF79402C28BF00241B
:1019E0008442FFB21CBF2F5522460CF1FF3C541C11
:1019F0005FFA8CF303F1FF3C402CCF7928BF002421
:101A00005FFA8CF3844203F1FF3CFBB21CBF2B5501
:101A100022461CF0FF03C5D121490D68D4B23470B1
:101A2000002D3FF456AF824236BFC0F14000121A7B
:101A30001218272AC4BF01222A704AE797F804C067
:101A40005FEA0C647FF54BAF164B174E197835786B
:101A5000CCB2EBB29C420ED0144901E0A3420AD0B2
:101A60000133282B28BF00233879C85CC5B2FD712B
:101A7000387D0728F2D9044CDFB237702179080687
:101A800044BF7C21E1702AE700B00640DCE0012081
:101A90006CE00120D8E001206DE0012098E00120F9
:101AA00068E00120E0E00120D9E0012070E00120A1
:101AB000054A064B10781978C2B2CBB29A4238BFA9
:101AC0004032D01A704700BF54E10120E9E0012004
:101AD00030B42D4B1A79940621D52C48DC79057841
:101AE0002B4901353F2D0B78C8BF00259D42E2B23E
:101AF00005D0284C5FFA85FC625580F800C0264866
:101B0000036863B1254A1478E1B28D4236BFC1F152
:101B100040016D1A6D18272DC4BF01251D701A4D87
:101B2000E8785FFA80FC5FEA0C6012D45FEA4C62EE
:101B30000DD5154B1D796B0609D5194C194920682F
:101B400000220A7000B102700F4B2C25DD7030BCF2
:101B500070472B791906E9D5134A10481478017893
:101B6000CBB29C420DD05A1C272A84BF00231A46B0
:101B70000E4D054CA95C98BFD3B2CAB2E271037096
:101B8000D4E76C20E870D1E700C0064054E10120A2
:101B9000E9E0012014E10120E4E0012055E1012009
:101BA00058E10120E8E001205CE10120ECE00120A7
:101BB000054A064B10781978C2B2CBB29A4238BFA8
:101BC0004032D01A704700BFD0E1012065E101200A
:101BD00030B42D4B1A79940621D52C48DC79057840
:101BE0002B4901353F2D0B78C8BF00259D42E2B23D
:101BF00005D0284C5FFA85FC625580F800C0264865
:101C0000036863B1254A1478E1B28D4236BFC1F151
